:020000040800F2
:1000000000000824F9380008952F0008972F0008F1
:10001000992F00089B2F00089D2F0008000000006A
:100020000000000000000000000000009F2F0008FA
:10003000A12F000800000000A32F0008A52F000832
:100040004939000849390008493900084939000888
:100050004939000849390008493900084939000878
:10006000493900084939000849390008AD2F00080E
:100070004939000849390008493900084939000858
:100080004939000849390008BD2F000849390008DE
:100090004939000849390008493900084939000838
:1000A0004939000849390008CD2F0008DD2F000824
:1000B00049390008ED2F000849390008493900087E
:1000C0004939000849390008493900084939000808
:1000D00049390008FD2F000849390008493900084E
:1000E0004939000849390008000000000D300008B7
:1000F00049390008493900084939000849390008D8
:1001000049390008493900084939000849390008C7
:1001100049390008493900084939000849390008B7
:1001200049390008493900084939000849390008A7
:100130004939000849390008493900084939000897
:1001400000000000000000000000000000000000AF
:100150004939000849390008493900084939000877
:100160004939000849390008493900084939000867
:100170004939000849390008493900084939000857
:100180004939000849390008493900084939000847
:100190004939000849390008493900084939000837
:1001A0004939000849390008493900084939000827
:1001B0004939000849390008493900084939000817
:1001C0004939000849390008493900084939000807
:1001D00049390008493900084939000849390008F7
:1001E00049390008493900084939000849390008E7
:1001F00049390008493900084939000849390008D7
:1002000049390008493900084939000849390008C6
:1002100049390008493900084939000849390008B6
:100220004939000849390008493900080000000030
:100230004939000849390008000000004939000820
:100240004939000849390008493900084939000886
:100250004939000849390008493900084939000876
:100260004939000849390008493900084939000866
:1002700049390008493900084939000800000000E0
:1002800049390008493900084939000800000000D0
:080290000000000049390008DC
:1002C00010B5054C237833B9044B13B10448AFF390
:1002D00000800123237010BDDC0900240000000011
:1002E000A430010808B5034B1BB103490348AFF321
:1002F000008008BD00000000E0090024A4300108CF
:1003000081F0004102E000BF83F0004330B54FEAC6
:1003100041044FEA430594EA050F08BF90EA020F33
:100320001FBF54EA000C55EA020C7FEA645C7FEAC6
:10033000655C00F0E2804FEA5454D4EB5555B8BFE9
:100340006D420CDD2C4480EA020281EA030382EA5A
:10035000000083EA010180EA020281EA0303362DEC
:1003600088BF30BD11F0004F4FEA01314FF4801CBF
:100370004CEA113102D0404261EB410113F0004FD1
:100380004FEA03334CEA133302D0524263EB430388
:1003900094EA050F00F0A780A4F10104D5F1200E26
:1003A0000DDB02FA0EFC22FA05F2801841F1000181
:1003B00003FA0EF2801843FA05F359410EE0A5F155
:1003C00020050EF1200E012A03FA0EFC28BF4CF086
:1003D000020C43FA05F3C01851EBE37101F000453C
:1003E00007D54FF0000EDCF1000C7EEB00006EEB49
:1003F0000101B1F5801F1BD3B1F5001F0CD34908D3
:100400005FEA30004FEA3C0C04F101044FEA445229
:1004100012F5800F80F09A80BCF1004F08BF5FEAB0
:10042000500C50F1000041EB045141EA050130BD90
:100430005FEA4C0C404141EB0101013C28BFB1F5A2
:10044000801FE9D291F0000F04BF01460020B1FAED
:1004500081F308BF2033A3F10B03B3F120020CDAC0
:100460000C3208DD02F1140CC2F10C0201FA0CF09E
:1004700021FA02F10CE002F11402D8BFC2F1200C03
:1004800001FA02F120FA0CFCDCBF41EA0C019040B9
:10049000E41AA2BF01EB0451294330BD6FEA040402
:1004A0001F3C1CDA0C340EDC04F11404C4F12002ED
:1004B00020FA04F001FA02F340EA030021FA04F3FF
:1004C00045EA030130BDC4F10C04C4F1200220FA56
:1004D00002F001FA04F340EA0300294630BD21FA94
:1004E00004F0294630BD94F0000F83F4801306BF5A
:1004F00081F480110134013D4EE77FEA645C18BF4E
:100500007FEA655C29D094EA050F08BF90EA020FE4
:1005100005D054EA000C04BF1946104630BD91EADC
:10052000030F1EBF0021002030BD5FEA545C05D1DF
:100530004000494128BF41F0004130BD14F580041E
:100540003CBF01F5801130BD01F0004545F0FE4192
:1005500041F470014FF0000030BD7FEA645C1ABFC7
:10056000194610467FEA655C1CBF0B46024650EAFE
:10057000013406BF52EA033591EA030F41F400212A
:1005800030BD00BF90F0000F04BF0021704730B5B0
:100590004FF4806404F132044FF000054FF0000185
:1005A00050E700BF90F0000F04BF0021704730B546
:1005B0004FF4806404F1320410F0004548BF40421B
:1005C0004FF000013EE700BF42004FEAE2014FEA70
:1005D00031014FEA02701FBF12F07F4393F07F4F4B
:1005E00081F06051704732F07F4208BF704793F04E
:1005F0007F4F04BF41F40021704730B54FF4607461
:1006000001F0004521F000411CE700BF50EA010263
:1006100008BF704730B54FF000050AE050EA01020C
:1006200008BF704730B511F0004502D5404261EB7C
:1006300041014FF4806404F132045FEA915C3FF4BD
:10064000D8AE4FF003025FEADC0C18BF03325FEA5A
:10065000DC0C18BF033202EBDC02C2F1200300FA0B
:1006600003FC20FA02F001FA03FE40EA0E0021FA30
:1006700002F11444BDE600BF4FF0FF3C06E000BFAE
:100680004FF0010C02E000BF4FF0010C4DF804CD1B
:100690004FEA410C7FEA6C5C4FEA430C18BF7FEADB
:1006A0006C5C1BD001B050EA410C0CBF52EA430C09
:1006B00091EA030F02BF90EA020F0020704710F189
:1006C000000F91EA030F58BF994208BF90422CBF18
:1006D000D8176FEAE37040F0010070474FEA410C11
:1006E0007FEA6C5C02D150EA013C07D14FEA430C2F
:1006F0007FEA6C5CD6D152EA033CD3D05DF8040BA0
:10070000704700BF8446104662468C4619466346D1
:1007100000E000BF01B5FFF7B7FF002848BF10F1A8
:10072000000F01BD4DF808EDFFF7F4FF0CBF0120ED
:1007300000205DF808FB00BF4DF808EDFFF7EAFF69
:1007400034BF012000205DF808FB00BF4DF808ED24
:10075000FFF7E0FF94BF012000205DF808FB00BF19
:100760004DF808EDFFF7CEFF94BF012000205DF8A3
:1007700008FB00BF4DF808EDFFF7C4FF34BF0120B0
:1007800000205DF808FB00BF4FEA410C7FEA6C5C7B
:1007900002D150EA013C0AD14FEA430C7FEA6C5C7B
:1007A00002D152EA033C02D14FF0000070474FF0F3
:1007B000010070474FEA410212F5001215D211D51F
:1007C0006FF47873B3EB625212D94FEAC12343F04E
:1007D000004343EA505311F0004F23FA02F018BFD0
:1007E000404270474FF00000704750EA013005D199
:1007F00011F0004008BF6FF0004070474FF000005C
:10080000704700BF80F0004002E000BF81F000416F
:1008100042001FBF5FEA410392EA030F7FEA226CA6
:100820007FEA236C6AD04FEA1262D2EB1363C1BF36
:10083000D218414048404140B8BF5B42192B88BFA5
:10084000704710F0004F40F4000020F07F4018BFC8
:10085000404211F0004F41F4000121F07F4118BFE8
:10086000494292EA030F3FD0A2F1010241FA03FC90
:1008700010EB0C00C3F1200301FA03F100F0004378
:1008800002D5494260EB4000B0F5000F13D3B0F140
:10089000807F06D340084FEA310102F10102FE2AAF
:1008A00051D2B1F1004F40EBC25008BF20F001001F
:1008B00040EA03007047490040EB0000013A28BFBE
:1008C000B0F5000FEDD2B0FA80FCACF1080CB2EB41
:1008D0000C0200FA0CF0AABF00EBC25052421843BF
:1008E000BCBFD0401843704792F0000F81F4000164
:1008F00006BF80F400000132013BB5E74FEA410337
:100900007FEA226C18BF7FEA236C21D092EA030FA2
:1009100004D092F0000F08BF0846704790EA010F1C
:100920001CBF0020704712F07F4F04D1400028BF49
:1009300040F00040704712F100723CBF00F500002B
:10094000704700F0004343F0FE4040F40000704761
:100950007FEA226216BF08467FEA2363014642020D
:1009600006BF5FEA412390EA010F40F48000704720
:100970004FF0000304E000BF10F0004348BF4042C6
:100980005FEA000C08BF704743F0964301464FF002
:1009900000001CE050EA010208BF70474FF000035E
:1009A0000AE000BF50EA010208BF704711F000439F
:1009B00002D5404261EB41015FEA010C02BF84466F
:1009C0000146002043F0B64308BFA3F18053A3F5CE
:1009D0000003BCFA8CF2083AA3EBC25310DB01FA15
:1009E00002FC634400FA02FCC2F12002BCF1004F99
:1009F00020FA02F243EB020008BF20F0010070472A
:100A000002F1200201FA02FCC2F1200250EA4C007D
:100A100021FA02F243EB020008BF20EADC707047C3
:100A20004FF0FF0C1CEAD0521EBF1CEAD15392EAD1
:100A30000C0F93EA0C0F6FD01A4480EA010C4002AD
:100A400018BF5FEA41211ED04FF0006343EA501007
:100A500043EA5111A0FB01310CF00040B1F5000F49
:100A60003EBF490041EAD3715B0040EA010062F1F8
:100A70007F02FD2A1DD8B3F1004F40EBC25008BFE2
:100A800020F00100704790F0000F0CF0004C08BF00
:100A900049024CEA502040EA51207F3AC2BFD2F1CD
:100AA000FF0340EAC250704740F400004FF00003DB
:100AB000013A5DDC12F1190FDCBF00F00040704715
:100AC000C2F10002410021FA02F1C2F1200200FA53
:100AD00002FC5FEA310040F1000053EA4C0308BF1A
:100AE00020EADC70704792F0000F00F0004C02BF6B
:100AF000400010F4000F013AF9D040EA0C0093F0E6
:100B0000000F01F0004C02BF490011F4000F013B3F
:100B1000F9D041EA0C018FE70CEAD15392EA0C0FAD
:100B200018BF93EA0C0F0AD030F0004C18BF31F018
:100B3000004CD8D180EA010000F00040704790F0EE
:100B4000000F17BF90F0004F084691F0000F91F092
:100B5000004F14D092EA0C0F01D142020FD193EA58
:100B60000C0F03D14B0218BF084608D180EA0100E0
:100B700000F0004040F0FE4040F40000704740F0BC
:100B8000FE4040F4400070474FF0FF0C1CEAD0528A
:100B90001EBF1CEAD15392EA0C0F93EA0C0F69D0E6
:100BA000A2EB030280EA010C49024FEA402037D051
:100BB0004FF0805343EA111143EA10130CF0004048
:100BC0008B4238BF5B0042F17D024FF4000C8B4238
:100BD00024BF5B1A40EA0C00B3EB510F24BFA3EB18
:100BE000510340EA5C00B3EB910F24BFA3EB9103E8
:100BF00040EA9C00B3EBD10F24BFA3EBD10340EA42
:100C0000DC001B0118BF5FEA1C1CE0D1FD2A3FF687
:100C100050AF8B4240EBC25008BF20F0010070473C
:100C20000CF0004C4CEA50207F32C2BFD2F1FF03DF
:100C300040EAC250704740F400004FF00003013A10
:100C400037E792F0000F00F0004C02BF400010F4B4
:100C5000000F013AF9D040EA0C0093F0000F01F0C8
:100C6000004C02BF490011F4000F013BF9D041EAEA
:100C70000C0195E70CEAD15392EA0C0F08D142021D
:100C80007FF47DAF93EA0C0F7FF470AF084676E7F0
:100C900093EA0C0F04D14B023FF44CAF08466EE7C9
:100CA00030F0004C18BF31F0004CCAD130F0004297
:100CB0007FF45CAF31F000437FF43CAF5FE700BFEF
:100CC00042000ED2B2F1FE4F0BD34FF09E03B3EBB6
:100CD000126209D44FEA002343F0004323FA02F0E2
:100CE00070474FF00000704712F1610F01D14202CE
:100CF00002D14FF0FF3070474FF00000704700BF47
:100D000053B94AB9002908BF00281CBF4FF0FF3172
:100D10004FF0FF3000F074B9ADF1080C6DE904CE6E
:100D200000F006F8DDF804E0DDE9022304B07047C6
:100D30002DE9F047089E0D4604468846002B4DD10C
:100D40008A42944668D9B2FA82F252B101FA02F3A9
:100D5000C2F1200120FA01F10CFA02FC41EA030879
:100D600094404FEA1C45210CB8FBF5FE1FFA8CF7A6
:100D700005FB1E8341EA03430EFB07F199420BD9A1
:100D80001CEB03030EF1FF3080F01E81994240F20C
:100D90001B81AEF1020E63445B1AA4B2B3FBF5F003
:100DA00005FB103344EA034400FB07F7A7420AD9C6
:100DB0001CEB040400F1FF3380F00881A74240F2ED
:100DC000058164440238E41B40EA0E4000211EB154
:100DD000D4400023C6E90043BDE8F0878B4208D920
:100DE000002E00F0EE800021C6E900050846BDE8AF
:100DF000F087B3FA83F100294AD1AB4202D3824291
:100E000000F2F980841A65EB030301209846002E56
:100E1000E2D0C6E90048DFE702B9FFDEB2FA82F2AB
:100E2000002A40F09180A1EB0C054FEA1C471FFA05
:100E30008CFE0121B5FBF7F307FB1350250C45EAA7
:100E400000450EFB03F0A84208D91CEB050503F191
:100E5000FF3802D2A84200F2CB8043462D1AA4B23A
:100E6000B5FBF7F007FB105544EA05440EFB00FE06
:100E7000A64508D91CEB040400F1FF3502D2A645B3
:100E800000F2BB802846A4EB0E0440EA03409EE734
:100E9000C1F120078B4022FA07FC4CEA030C20FA30
:100EA00007F405FA01F31C43FD404FEA1C4900FA20
:100EB00001F3B5FBF9F8200C1FFA8CFE09FB18555D
:100EC00040EA054508FB0EF0A84202FA01F20BD9F0
:100ED0001CEB050508F1FF3A80F08880A84240F23B
:100EE0008580A8F1020865442D1AA4B2B5FBF9F07B
:100EF00009FB105544EA054500FB0EFEAE4508D936
:100F00001CEB050500F1FF346CD2AE456AD90238FE
:100F1000654440EA0840A0FB0294A5EB0E05A542FB
:100F2000C846A64656D353D05EB1B3EB080265EB74
:100F30000E0505FA07F722FA01F3CD401F43C6E973
:100F400000750021BDE8F087C2F1200320FA03F10B
:100F50000CFA02FC25FA03F395400D434FEA1C47B7
:100F60001FFA8CFEB3FBF7F107FB11302B0C43EAA1
:100F7000004301FB0EF0984204FA02F408D91CEB7E
:100F8000030301F1FF382FD298422DD9023963446F
:100F90001B1AADB2B3FBF7F007FB103345EA03456C
:100FA00000FB0EF3AB4208D91CEB050500F1FF383E
:100FB00016D2AB4214D902386544ED1A40EA014119
:100FC00038E73146304607E78646E5E61846FAE652
:100FD0004B45A9D2B9EB020864EB0C0E0138A3E72C
:100FE0004046EAE7204694E74146D1E7D0467BE712
:100FF000023B654432E7084609E76444023842E7A9
:10100000704700BF844641EA000313F003036DD12B
:10101000403A41D351F8043B40F8043B51F8043BBB
:1010200040F8043B51F8043B40F8043B51F8043BC2
:1010300040F8043B51F8043B40F8043B51F8043BB2
:1010400040F8043B51F8043B40F8043B51F8043BA2
:1010500040F8043B51F8043B40F8043B51F8043B92
:1010600040F8043B51F8043B40F8043B51F8043B82
:1010700040F8043B51F8043B40F8043B51F8043B72
:1010800040F8043B51F8043B40F8043B51F8043B62
:1010900040F8043B403ABDD2303211D351F8043B02
:1010A00040F8043B51F8043B40F8043B51F8043B42
:1010B00040F8043B51F8043B40F8043B103AEDD2B1
:1010C0000C3205D351F8043B40F8043B043AF9D202
:1010D000043208D0D2071CBF11F8013B00F8013BD5
:1010E00001D30B8803806046704700BF082A13D3E2
:1010F0008B078DD010F003038AD0C3F10403D21AFA
:10110000DB071CBF11F8013B00F8013B80D331F82D
:10111000023B20F8023B7BE7043AD9D3013A11F8AD
:10112000013B00F8013BF9D20B7803704B78437018
:101130008B7883706046704700000000000000005C
:10114000A2EB0300704700BF02780B78012A28BF8A
:101150009A42F5D16DE9044540EA0104CDE9026700
:101160006FF0000C4FEA447212B380EA010414F0ED
:10117000070F6AD100F0070420F0070004F0030510
:1011800021F007014FEAC505F0E8042314F0040F2D
:10119000F1E804670CFA05F462EA040266EA040660
:1011A0000AD063EA0403624667EA0407664603E07E
:1011B000F0E80423F1E8046782FA4CF582EA0604B9
:1011C000A4FA8CF46CBB83FA4CF583EA0705A5FA04
:1011D0008CF595B950E9022351E9026782FA4CF582
:1011E00082EA0604A4FA8CF483FA4CF583EA070534
:1011F000A5FA8CF52543DBD09CB92DBAB5FA85F458
:1012000024F0070427FA04F1DDE9026723FA04F366
:1012100003F0FF0001F0FF01FDE80445A0EB010031
:10122000704724BAB4FA84F424F0070426FA04F1CF
:10123000DDE9026722FA04F202F0FF0001F0FF018B
:10124000FDE80445A0EB0100704714F0030F3CD10A
:1012500010F0030428D150F8082B51F8083B82FA0B
:101260004CF582EA0305A5FA8CF55DB950F8042C1B
:1012700051F8043C82FA4CF582EA0305A5FA8CF594
:10128000002DE8D02DBAB5FA85F424F0070423FA2E
:1012900004F122FA04F202F0FF0001F0FF01FDE880
:1012A0000445A0EB010070474FEAC40420F003009E
:1012B00050F8082B21F0030151F8083B0CFA04F414
:1012C00062EA040263EA0403C9E710F003041AD0D7
:1012D000A1EB040120F00300E40750F8042B06D032
:1012E0000FD28B785FFAA2F4E41A06D12BB1CB7837
:1012F0005FFAB2F4E41A00D11BB920465DF8104B36
:10130000704701F1040150F8042BCC0721F00301D0
:1013100051F8043B48D824D222F07F4482FA4CF59D
:1013200094EA1325A5FA8CF50AD165B951F8043B66
:1013300084EA0204B4EB036F0ED150F8042BEBE700
:101340004FEA132355E035F07F454DD10878FDE88D
:101350000445C0F1000070474FEA126203F0FF033A
:1013600047E002EA1C4482FA4CF594EA1345A5FAD8
:101370008CF50AD165B951F8043B84EA0204B4EB58
:10138000034F0CD150F8042BEBE74FEA134330E046
:1013900015EA1C4528D10B884FEA124229E04FEA92
:1013A000124203EA1C4324E002F0FF0482FA4CF5E7
:1013B00094EA1365A5FA8CF50AD165B951F8043B96
:1013C00084EA0204B4EB032F09D150F8042BEBE7B5
:1013D0004FEA13630DE015F0FF0F05D10B684FEADC
:1013E000122223F07F4304E04FF00000FDE80445A3
:1013F000704712BA1BBA82FA4CF482EA0304A4FAC8
:101400008CF5B5FA85F402FA04F203FA04F34FEA14
:101410001260FDE80445A0EB136070470000000077
:1014200000000000000000000000000000000000BC
:1014300000000000000000000000000000000000AC
:1014400090F800F06DE9024520F007016FF0000C04
:1014500010F0070491F820F040F049804FF00004AC
:101460006FF00700D1E9002391F840F000F1080087
:1014700082FA4CF2A4FA8CF283FA4CF3A2FA8CF3BF
:101480004BBBD1E9022382FA4CF200F10800A4FA26
:101490008CF283FA4CF3A2FA8CF3E3B9D1E904237A
:1014A00082FA4CF200F10800A4FA8CF283FA4CF3B1
:1014B000A2FA8CF37BB9D1E9062301F1200182FA6B
:1014C0004CF200F10800A4FA8CF283FA4CF3A2FA71
:1014D0008CF3002BC6D0002A04BF04301A4612BA7F
:1014E000B2FA82F2FDE8024500EBD2007047D1E982
:1014F000002304F00305C4F100004FEAC50514F011
:10150000040F91F840F00CFA05F562EA05021CBFE1
:1015100063EA050362464FF00004A9E700000000FB
:1015200001F0FF01102A2BDB10F0070F08D010F894
:10153000013B013A8B422DD010F0070F42B3F6D198
:10154000F0B441EA012141EA014122F007047FF0B1
:1015500000070023F0E80256083C85EA010586EA08
:10156000010685FA47F5A3FA87F586FA47F6A5FA44
:1015700087F68EB9EED1F0BC01F0FF0102F0070250
:1015800032B110F8013B013A83EA010313B1F8D1FB
:101590000020704701387047002D06BF35460338DC
:1015A000073815F0010F07D1013015F4807F02BF15
:1015B000013015F4C03F0130F0BC0138704700BF66
:1015C00070B54FF0FF0C4CF4E06C1CEA11541DBFD9
:1015D0001CEA135594EA0C0F95EA0C0F00F0DEF8A4
:1015E0002C4481EA030621EA4C5123EA4C5350EA89
:1015F000013518BF52EA033541F4801143F48013DA
:1016000038D0A0FB02CE4FF00005E1FB02E506F06A
:101610000042E0FB03E54FF00006E1FB03569CF0BF
:10162000000F18BF4EF0010EA4F1FF04B6F5007FC5
:1016300064F5407404D25FEA4E0E6D4146EB060637
:1016400042EAC62141EA55514FEAC52040EA5E50C0
:101650004FEACE2EB4F1FD0C88BFBCF5E06F1ED86A
:10166000BEF1004F08BF5FEA500E50F1000041EBA1
:10167000045170BD06F0004646EA010140EA02004E
:1016800081EA0301B4EB5C04C2BFD4EB0C0541EA70
:10169000045170BD41F480114FF0000E013C00F385
:1016A000AB8014F1360FDEBF002001F0004170BDA9
:1016B000C4F10004203C35DA0C341BDC04F11404C2
:1016C000C4F1200500FA05F320FA04F001FA05F24E
:1016D00040EA020001F0004221F0004110EBD3701B
:1016E00021FA04F642EB06015EEA430E08BF20EA47
:1016F000D37070BDC4F10C04C4F1200500FA04F3EA
:1017000020FA05F001FA04F240EA020001F000417B
:1017100010EBD37041F100015EEA430E08BF20EAEE
:10172000D37070BDC4F1200500FA05F24EEA020E36
:1017300020FA04F301FA05F243EA020321FA04F065
:1017400001F0004121FA04F220EA020000EBD3701C
:101750005EEA430E08BF20EAD37070BD94F0000F1C
:101760000FD101F00046400041EB010111F4801F50
:1017700008BF013CF7D041EA060195F0000F18BF01
:10178000704703F00046520043EB030313F4801F3D
:1017900008BF013DF7D043EA0603704794EA0C0FF7
:1017A0000CEA135518BF95EA0C0F0CD050EA41060D
:1017B00018BF52EA4306D1D181EA030101F000418A
:1017C0004FF0000070BD50EA410606BF10461946B2
:1017D00052EA430619D094EA0C0F02D150EA0136BE
:1017E00013D195EA0C0F05D152EA03361CBF1046FF
:1017F00019460AD181EA030101F0004141F0FE419E
:1018000041F470014FF0000070BD41F0FE4141F421
:10181000780170BD70B54FF0FF0C4CF4E06C1CEA21
:1018200011541DBF1CEA135594EA0C0F95EA0C0FD6
:1018300000F0A7F8A4EB050481EA030E52EA033591
:101840004FEA013100F088804FEA03334FF08055B2
:1018500045EA131343EA12634FEA022245EA1115DF
:1018600045EA10654FEA00260EF000419D4208BF90
:10187000964244F1FD0404F5407402D25B084FEA3D
:101880003202B61A65EB03055B084FEA32024FF4E9
:1018900080104FF4002CB6EB020E75EB030E22BF46
:1018A000B61A754640EA0C005B084FEA3202B6EB06
:1018B000020E75EB030E22BFB61A754640EA5C00B5
:1018C0005B084FEA3202B6EB020E75EB030E22BF45
:1018D000B61A754640EA9C005B084FEA3202B6EB46
:1018E000020E75EB030E22BFB61A754640EADC0005
:1018F00055EA060E18D04FEA051545EA16754FEA67
:1019000006164FEAC30343EA52734FEAC2025FEA84
:101910001C1CC0D111F4801F0BD141EA00014FF013
:1019200000004FF0004CB6E711F4801F04BF0143E4
:101930000020B4F1FD0C88BFBCF5E06F3FF6AFAE00
:10194000B5EB030C04BFB6EB020C5FEA500C50F190
:10195000000041EB045170BD0EF0004E4EEA113113
:1019600014EB5C04C2BFD4EB0C0541EA045170BD1A
:1019700041F480114FF0000E013C90E645EA060E5E
:101980008DE60CEA135594EA0C0F08BF95EA0C0F8C
:101990003FF43BAF94EA0C0F0AD150EA01347FF4D4
:1019A00034AF95EA0C0F7FF425AF104619462CE7AB
:1019B00095EA0C0F06D152EA03353FF4FDAE10460E
:1019C000194622E750EA410618BF52EA43067FF45F
:1019D000C5AE50EA41047FF40DAF52EA43057FF4EF
:1019E000EBAE12E74A0011D212F5001211D20DD55A
:1019F0006FF47873B3EB62520ED44FEAC12343F015
:101A0000004343EA505323FA02F070474FF00000BE
:101A1000704750EA013002D14FF0FF3070474FF06D
:101A20000000704738B505460C462846214600227E
:101A30000023FEF781FE28B928462146BDE838403C
:101A400000F00AB8284604F1004100F005F84042D1
:101A500061EB410138BD00BFD0B50C4B00220646FA
:101A60000F46FFF7ADFDFFF7BDFF0446FEF78AFD09
:101A7000074B0022FFF7A4FD02460B4630463946CD
:101A8000FEF742FCFFF7AEFF2146D0BD0000F03D5F
:101A90000000F04120B310B58646002301E0013379
:101AA0009BB28B4209D21EF803C0BCF1550FF6D190
:101AB0000EEB03025278AA2AF1D18B4209D0C91A3F
:101AC0008CB222460EEB03017046FFF79BFA2046CC
:101AD00010BD0A460021704609F066FF0020F7E7B6
:101AE000004870470CFEFFFF00B586464FF0000C23
:101AF000604611E00133DBB2072B09D800F0010288
:101B00004008002AF6D048F20842424090B2F1E77D
:101B10000CF1010C1FFA8CFC8C4504D21EF80C3021
:101B200058400023E8E75DF804FB0000F8B5002BFF
:101B300018BF002824D004461E460378552B21D117
:101B40004378AA2B20D1837893421FD1B0F8033079
:101B50009D1EADB206392F46A94219DDD91C89B2A6
:101B6000FFF7C2FF6B1DE35A984214D115B9002745
:101B70003846F8BD2A46611D3046FFF743FAF7E7BD
:101B8000064FF5E7064FF3E7054FF1E7054FEFE79F
:101B90006FF0C707ECE7044FEAE700BF0CFEFFFF5A
:101BA000D4FEFFFF70FEFFFFA8FDFFFF08B5014652
:101BB000014809F057FF08BDC030010810B53C4B83
:101BC0001B68B3F5026F02DB3A4B01221A603A4BF5
:101BD0001B68B3F5007F23DB384B1B6803B300237E
:101BE000364A136009E0364A32F81300354951F895
:101BF0002320024441F823200133B3F5007FF2DBB8
:101C0000314B1C68314B1B6893FBF4F204FB12331D
:101C1000A3B12F4B01221A602C4A136801331360C1
:101C20002C4B1A682C4B1B689A4202DD294B002270
:101C30001A60204B1B68012B21D010BDB3F5007F2B
:101C40000CDA204951F82320B2FBF4F2234820F8A3
:101C50001320002241F823200133EFE7204CFF231B
:101C6000237063704FF480621C49A01CFFF7CAF90F
:101C700040F2024221461B4807F0DCFFC9E7144B43
:101C80001B68012BD9D172B6124A13680133136055
:101C90000023074A1360144A1360074A136062B6B0
:101CA000044A13600A4A1360044B01221A60C4E715
:101CB000F80900240C0A0024FC0900240800002470
:101CC000A81B00242012002400000024040A002481
:101CD0000400002430290024080A0024200E0024D7
:101CE000100A00247C2A0024000A00244FF07E50B1
:101CF0007047000010B500F0EDFE04464368012B6C
:101D000011D0A368012B11D0E368012B11D02369F6
:101D1000012B11D06369012B11D02368012B11D045
:101D2000207EC8B910BD00F051F8EAE700F05CF879
:101D3000EAE700F069F8EAE700F076F8EAE700F091
:101D400083F8EAE7FFF7D2FFFEF73EFC02460B46B8
:101D5000034809F087FEE3E7FFF728FFE2E700BF4B
:101D6000CC300108F8B5154B1988B3F90030002BB9
:101D700003DB134B00221A70F8BDC9B2114E0025C7
:101D800075548CB221463046FFF784FE0E4F3B4619
:101D90002A4621463046FFF7C9FE384600F0EEFDE0
:101DA000064B1D80C82422462946304609F0FCFD1A
:101DB00022462946384609F0F7FDDDE7002A0024CF
:101DC0001800002438290024201A002408B5044BE8
:101DD000044A07CA83E80700184609F0A5FE08BDB3
:101DE000001B0024E030010810B5054C054A2346CD
:101DF00007CA03C31A70204609F096FE10BD00BF43
:101E00000C1B0024EC30010810B5054C054A234694
:101E100007CA03C31A70204609F086FE10BD00BF32
:101E2000F41A0024F830010808B5054B054A92E879
:101E3000030018601971184609F076FE08BD00BF4E
:101E4000EC1A00240431010808B50348034B036071
:101E500009F06AFE08BD00BFE81A002435313200DF
:101E600010B58AB000230793089309930093019358
:101E7000029303930493059306932648264A02602F
:101E80004FF4802242608360C360042202610375C4
:101E9000012242758261037743628362C3624FF419
:101EA00080520263436380F8383002F0DDFB38BBB8
:101EB0000023079307A9174802F00EFD18BB174B24
:101EC0000093062301930023029340F2FF720392D2
:101ED0000422049205938DF8193069460D4801F0EB
:101EE000ABFF98B90B4C6946204601F0A5FF204690
:101EF00002F080FA0A21204601F096FD0AB010BDDA
:101F000000F0A3FED4E700F0A0FED8E700F09DFEAD
:101F1000E8E700BF181B0024002002400008302E14
:101F200010B5B8B004460021339134913591369103
:101F30003791C02202A809F037FD22681F4B9A4250
:101F400001D038B010BD4FF400220023CDE90223A8
:101F50004FF400332B9302A805F014FA58BB184B2A
:101F6000D3F8D82042F02002C3F8D820D3F8D820E4
:101F700002F020020092009AD3F8E02042F004021E
:101F8000C3F8E020D3F8E03003F004030193019B91
:101F900002233393032334930024359433A909484F
:101FA00004F0AAF922462146122002F059FD12201F
:101FB00002F08CFDC5E700F048FED0E700200240AB
:101FC0000044025800080258002918BF002826D0F3
:101FD00000B586468C4688420BD100201DE002F1F8
:101FE00020010FE0814217D1DAB10EF1010E0CF1A0
:101FF000010C9EF800200C4BD35C03F00303012B73
:10200000EDD011469CF80000074BC35C03F00303BE
:10201000012BE7D12030E5E7081A5DF804FB012029
:1020200070470020F9E700BFC53201082E20704735
:102030008446002318460AE0A1F14102D2B2052AE3
:1020400011D808443738022B00D800010133032B84
:1020500011D81CF80310A1F13002D2B2092AEBD832
:1020600008443038EFE7A1F16102D2B2052A03D863
:1020700008445738E7E7704700207047F8B50B1A57
:10208000052B60DD06460F4615460230FFF7D0FFF0
:102090000446A0F55C43B3F5806F56D3A0F55843D2
:1020A000B3F5806F1CD2B11D7F1A052F4FDDB379B8
:1020B0005C2B4ED1F379752B4DD106F10800FFF75B
:1020C000B7FFA0F55C43B3F5806F46D2254B03EA1A
:1020D0008424C0F30900204300F580340C2000E084
:1020E00006207F2C0BD9B4F5006F0DD3B4F5803FDB
:1020F0000DD3B4F5881F32D2F027042601E0002763
:102100000126731EDBB20EE0C0270226F9E7E027A6
:102110000326F6E704F03F012A6841F08001D1541C
:10212000A409013BDBB2002BF4D1012E06D92B68A8
:102130003C431C702B6833442B6005E02B6804F093
:102140007F041C70F6E70020F8BD0020FCE70020AB
:10215000FAE70020F8E70020F6E70020F4E7002087
:10216000F2E700BF00FC0F002DE9F04182B00E46FF
:102170000F688B685D1C3D440022019207EB030C45
:10218000FB5C222B40F0858080462C46104600E008
:102190000134E11B726891420AD22378222B07D0C6
:1021A0005C2BF5D10134E31B934272D20130EFE78F
:1021B00091426ED22378222B6BD1A4EB0C0CACEBAA
:1021C0000000336901309847074600285DD0019030
:1021D0002BE0631B002B58DD6B78752B55D85C2BDF
:1021E00011D35C3B192B50D8DFE803F0114F4F4F50
:1021F0004F4F184F4F4F2B4F4F4F4F4F4F4F324F67
:102200004F4F394F4047222B01D02F2B3DD1019BFF
:102210005A1C01926A781A70022305E0019B5A1C2D
:10222000019208221A7002231D44A54239D22B784C
:102230005C2BCED0019B5A1C019215F8012B1A7011
:10224000F3E7019B5A1C01920C221A700223EBE760
:10225000019B5A1C01920A221A700223E4E7019B97
:102260005A1C01920D221A700223DDE7019B5A1CB1
:10227000019209221A700223D6E701AA21462846B4
:10228000FFF7FCFE03460028CED117B1736938462C
:102290009847ADB13368ED1AB560002002B0BDE8D3
:1022A000F081019B00221A701023C8F80C30C8F886
:1022B00010703368E41AB4600134B4600120EDE7B3
:1022C0000020EBE70246D0B110B40468ACB18368DB
:1022D0004068834202D30AE00133936093689842D6
:1022E00002D9E15C2029F7D99368984202D01046C0
:1022F00010BC7047013B9360F9E72246F7E770474F
:1023000010B5036828209847044618B128220021F8
:1023100009F04AFB204610BD38B5044678B1006884
:1023200078B1A5687DB92B1D6268934207D203225C
:102330000649284409F028FF08B90335A56020465E
:1023400038BD0446FBE70024F9E700BF0C31010863
:102350002DE9F04393B005460C4600231193FFF797
:1023600065FE002C00F099802368002B00F0978018
:10237000002331E0652A29D048336B44002203F85A
:10238000442C0DF1040911A948460AF0D5FE064671
:102390000F46DDF84480C84500F08380C5E9066734
:1023A00041A3D3E90023FEF7DBF9002864D06FF0E6
:1023B00000436B610823EB6001ABA8EB0308A36843
:1023C0004344A360012013B0BDE8F08303F148014A
:1023D000694401F8442C01333E2BCDD8A2681A443D
:1023E00061688A42C8D221688A5C452AC2D82B2AF1
:1023F000C2D3A2F12B011A29BED801A656F821F0AA
:10240000CD23000879230008CD2300086D2400089F
:1024100079230008CD230008CD230008CD23000830
:10242000CD230008CD230008CD230008CD230008CC
:10243000CD230008CD230008CD2300087923000810
:1024400079230008792300087923000879230008FC
:1024500079230008792300087923000879230008EC
:102460007923000879230008CD23000803F14802EE
:102470006A4402F8440CAEE700220D4B3046394660
:10248000FEF764F918B14FF000436B6192E73046F4
:102490003946FEF78FF968618CE7002093E700204A
:1024A00091E700208FE700BF0000C0FFFFFFDF4182
:1024B0000000E0C138B5002918BF00281AD00D4629
:1024C00084680AB90AE024687CB1216A69B12846A7
:1024D000FEF73AFE0028F6D107E024682CB1216A05
:1024E0002846FFF771FD0028F7D12CB1236A2BB1E4
:1024F000204638BD0024FBE70024F9E70024F7E775
:1025000038B5044616E0E36813F4807F04D12069EF
:1025100010B10F4B5B689847E36813F4007F04D158
:10252000206A10B10A4B5B689847094B5B682046EC
:1025300098472C4654B12568E36813F4807FE2D1B4
:10254000A0680028DFD0FFF7DBFFDCE738BD00BF65
:102550000C000024CB68B3F57A7F80F08B802DE9E6
:10256000F04106460C460133CB60002900F0848020
:102570008B684A68934280F081800A68D25C7B2A2B
:1025800002D00020BDE8F08101338B600846FFF7E0
:1025900099FEA3686268934203D22268D35C7D2BC4
:1025A00059D0A3686268934204D2013BA36000251E
:1025B0002F4634E0013BA3600020E3E70746A36811
:1025C0000133A3602046FFF77DFE21462846FFF732
:1025D000CBFD002839D02046FFF774FE2B692B6213
:1025E00000232B61A368626893422ED22268D25CDA
:1025F0003A2A2AD10133A3602046FFF763FE214621
:10260000284600F03FF800B32046FFF75BFEA368C2
:102610006268934211D22268D35C2C2B0DD1A8465C
:1026200004F11000FFF76CFE054670B1002FC5D015
:10263000C8F80000C0F80480C1E7A368626893424C
:1026400003D22268D35C7D2B07D0CFB13846FFF789
:1026500057FF002096E700252F46E368013BE36023
:1026600007B17D604023F360B760A3680133A360C6
:10267000012087E700207047002083E7002081E7E2
:1026800000207FE7002975D070B506460C460D681E
:10269000002D71D08868021D4B689A4206D804222A
:1026A0003749284409F070FD00283AD0A068421D3F
:1026B00063689A4206D805223249284409F064FD2D
:1026C000002835D0A068021D63689A4206D804220B
:1026D0002D49284409F058FD00282FD0A3686268CE
:1026E000934202D2EB5C222B30D0A3686268934203
:1026F00007D2EA5CA2F13003DBB22D2A18BF092B06
:1027000029D9A3686268934202D2EB5C5B2B27D085
:10271000A3686268934231D2EB5C7B2B25D000200A
:102720002DE00423F360A3680433A360012026E0B6
:102730000120F060A2680532A26020E00223F3606D
:1027400001207061A2680432A26018E02146304680
:10275000FFF70AFD13E021463046FFF7F9FD0EE0D2
:102760002146304600F012F809E021463046FFF7D6
:10277000F1FE04E000207047002000E0002070BD62
:10278000103101083031010838310108CB68B3F548
:102790007A7F6DD22DE9F04106460C460133CB60BD
:1027A0000A688B68D25C5B2A02D00020BDE8F08109
:1027B00001338B600846FFF785FD3CB1A368626872
:1027C000934203D22268D35C5D2B48D044B1A36806
:1027D0006268934204D2013BA36000252F461EE0AD
:1027E000A368013BA3600020E0E7C8F80000C0F840
:1027F0000480A3680133A3602046FFF763FD2146F0
:102800002846FFF73FFF68B32046FFF75BFDA3684C
:10281000626893420ED22268D35C2C2B0AD1A84660
:1028200004F11000FFF76CFD0546D8B1002FDCD194
:102830000746DEE7A3686268934213D22268D35C3E
:102840005D2B0FD1E368013BE36007B17D6020237E
:10285000F360B760A3680133A3600120A6E70025F9
:102860002F46EFE737B13846FFF74AFE00209DE7D5
:1028700000207047002099E7F0B58BB015461E4642
:1028800000240394049405940694079408940994EE
:102890002B4B1C605C600446002918BF002817D130
:1028A000002C4AD0019400230293059A049B9A427B
:1028B0003ED2029215B1029B23442B60204B01AA09
:1028C00092E8030083E80300002738460BB0F0BD10
:1028D000039004911B4B93E807000AAF07E9070038
:1028E0001846FFF70DFD0746E0B103A8FFF714FDFA
:1028F000FFF7E8FC01463846FFF7C4FE90B136B951
:10290000002DE2D0039B059A13442B60DDE703A85A
:10291000FFF7D8FC059B049A934203D2039AD35C39
:10292000002BEDD0002FBBD03846FFF7E9FDB7E70D
:10293000002BBFD0013B0293BCE72746C5E700BF91
:102940007C1B00240C00002470B5044648B10D46E1
:102950001646FEF775FD33462A46411C2046FFF712
:102960008BFF70BD08B500221146FFF7EDFF08BDD3
:1029700008B50022FFF79EFD08BD00002DE9F84FC5
:1029800004460146414809F06DF82046FFF7EAFF8A
:10299000002874D004463E49FFF7EAFF05463D494A
:1029A0002046FFF7E5FF06463B492046FFF7E0FFDC
:1029B00080463A492046FFF7DBFF07463849204664
:1029C000FFF7D6FF824637492046FFF7D1FF814601
:1029D00035492046FFF7CCFF8346002D18BF002E57
:1029E00045D03B1E18BF0123B8F1000F3FD0002B8C
:1029F0003DD0B9F1000318BF0123BAF1000F36D062
:102A0000002B34D0002832D06969284809F02AF810
:102A10007169274809F026F8D8F81410254809F0FC
:102A200021F87969244809F01DF8DAF814102348D0
:102A300009F018F8D9F81410214809F013F8DBF858
:102A40001410204809F00EF8D8F814201E4B9A6094
:102A500072695A606A691A607A69DA60DAF8142071
:102A60001A61D9F814205A61DBF814201A76174B32
:102A700001221A702046FFF743FDBDE8F88F144885
:102A800009F052F8114B00221A70F6E740310108A4
:102A900054310108603101086431010868310108CE
:102AA00078310108883101089C310108B4310108EE
:102AB000C8310108D0310108D8310108EC310108D2
:102AC0000032010818320108841B00241800002479
:102AD0003432010800487047841B002400B583B0DD
:102AE0000B4BD3F8D82042F00102C3F8D820D3F81A
:102AF000D83003F001030193019B002211460B2003
:102B000001F0AEFF0B2001F0E1FF03B05DF804FB24
:102B1000004402582DE9F0418AB00024059406943F
:102B2000079408940994304BD3F8E02042F08002D7
:102B3000C3F8E020D3F8E02002F080020092009A6F
:102B4000D3F8E02042F00402C3F8E020D3F8E020FC
:102B500002F004020192019AD3F8E02042F001024F
:102B6000C3F8E020D3F8E02002F001020292029ABA
:102B7000D3F8E02042F01002C3F8E020D3F8E020C0
:102B800002F010020392039AD3F8E02042F002020E
:102B9000C3F8E020D3F8E03003F002030493049B71
:102BA000DFF848802246C621404603F0B9FC104DAC
:102BB00022463021284603F0B3FCC62305930127A3
:102BC000069707940226089605A9404603F094FB51
:102BD0003023059306970794089605A9284603F025
:102BE0008BFB0AB0BDE8F081004402580000025897
:102BF0000008025810B584B0002400940194029497
:102C0000039401F085FF01238DF800308DF8014019
:102C10004FF01052019212228DF808208DF80940D1
:102C20008DF80A4003228DF80B208DF80C408DF8AA
:102C30000D308DF80E308DF80F40684601F086FF9C
:102C4000042001F073FF04B010BD72B6FEE700006F
:102C500000B59FB04C2200210BA808F0A5FE202251
:102C6000002103A808F0A0FE022003F05FFC00236F
:102C700000933A4BDA6A22F00102DA62DB6A03F06F
:102C800001030093364B9A6942F440429A619B6972
:102C900003F440430093009B314B9B6913F4005FA6
:102CA000FAD0304BD3F8F42042F00202C3F8F420FB
:102CB000D3F8F43003F002030193019B0023029345
:102CC000274B9A6942F440429A619B6903F440435E
:102CD0000293224BDA6A42F00102DA62DB6A03F005
:102CE00001030293029B1E4B9B6913F4005FFAD011
:102CF00003230B934FF480330C9301230E93402353
:102D00000F930223149315931693F022179218939E
:102D100019931A9308231B9300231C931D930BA84C
:102D200003F02EFCB0B93F23039303230493002345
:102D30000593082306934023079308934FF480627A
:102D400009920A93042103A804F080F820B91FB067
:102D50005DF804FBFFF779FFFFF777FF00040058E9
:102D6000004802580044025800B5B1B0C02200210A
:102D7000684608F019FE4FF000420023CDE9002319
:102D8000684604F0FFFA10B931B05DF804FBFFF7B4
:102D90005CFF000008B5FFF72DFF394B5B6913F4AA
:102DA000003F13D1BFF34F8FBFF36F8F344B00221F
:102DB000C3F85022BFF34F8FBFF36F8F5A6942F4AD
:102DC00000325A61BFF34F8FBFF36F8F2C4B5B699B
:102DD00013F4803F27D12A4B0022C3F88420BFF38D
:102DE0004F8FD3F88040C4F34E3000E01846C4F350
:102DF000C90243F6E07303EA401343EA82732049B1
:102E0000C1F860321346013A002BF2D1431E00286C
:102E1000ECD1BFF34F8F4B6943F480334B61BFF369
:102E20004F8FBFF36F8F00F0B9FDFFF711FFFFF772
:102E30009BFFFFF76FFEFFF751FE00F081F900F0F6
:102E400083FB00F061FC0F4800F022F800F02EFA3E
:102E5000FFF706F800F0D0F900210B4806F0C6FC99
:102E600006E0FEF747FF094B00221A70FEF7A6FEA8
:102E7000FEF778FF054B1B78002BF2D1F6E700BF79
:102E800000ED00E07C2A002498280024180000248B
:102E900008B5054B1860054B186800230222194637
:102EA000806809F053F808BDA01B00242C00002402
:102EB000022801D80120704708B508F08BFA0923D1
:102EC0000360002008BD000010B5013801280AD8B1
:102ED00014464FF0FF3392B20748006807F098FF9E
:102EE00040B9204610BD08F075FA092303604FF081
:102EF000FF30F7E70520F5E7A01B0024022801D8E2
:102F00000020704708B508F065FA092303604FF008
:102F1000FF3008BD08B508F05DFA092303604FF0E3
:102F2000FF3008BD08B548B94FF0FF33012208480B
:102F3000006807F0D5FF40B9012008BD08F04AFA43
:102F4000092303604FF0FF30F7E70520F5E700BFE6
:102F5000A01B002408B5022804D84FF400534B608E
:102F6000002008BD08F036FA09230360F8E70000E6
:102F700082B0074BD3F8F42042F00202C3F8F420E9
:102F8000D3F8F43003F002030193019B02B07047C1
:102F900000440258FEE7FEE7FEE7FEE7FEE7704763
:102FA0007047704708B500F027FD08BD08B5024816
:102FB00002F006FE08BD00BF042A002408B502483E
:102FC00000F0CEFD08BD00BF181B002408B5024864
:102FD00005F0ADFF08BD00BF0028002408B5024879
:102FE00005F0A5FF08BD00BF0028002408B5024871
:102FF00005F09DFF08BD00BFE428002408B5024885
:1030000006F0DAFE08BD00BF7C2A002408B502489D
:1030100005F08DFF08BD00BF4C280024012070473B
:1030200008B508F0D7F9162303604FF0FF3008BD4C
:1030300008B54FF0FF31FFF7F3FFFEE710B5034689
:103040000C4A0D490D48006840B10C480068034423
:10305000521A934206D8094A136010BD0748084C1B
:103060000460F2E708F0B6F90C2303604FF0FF307C
:10307000F3E700BF0000082400040000A41B0024A4
:10308000602B0024244B1B6803F00F03062B06D88B
:10309000214A136823F00F0343F0070313601F4B0B
:1030A0001A6842F001021A6000221A6119681C4A6B
:1030B0000A401A60184B1B6813F0080F06D0164A16
:1030C000136823F00F0343F007031360134B002230
:1030D0009A61DA611A62134999621349D9621349F4
:1030E00019635A639963DA6319645A64196821F49D
:1030F000802119601A660E4B1A680E4B1340B3F10B
:10310000005F03D20C4B0122C3F808210B4B43F2A2
:10311000D2021A60704700BF0020005200440258DB
:103120007FEDF6EA000202020000FF0180020101C9
:103130000010005C0000FFFF0080005100400052C2
:1031400000B58DB000230793089309930A930B935E
:1031500004930593069300930193029303932448E9
:10316000244A02601722426083604FF6FF72C260F9
:1031700003614361836106F029F850BB1C4806F0E7
:1031800085F848BB04230793502308930023099331
:103190000B9307A9164806F0F1FA00BB002304932D
:1031A0000593069304A9124806F0ACFCD0B900229E
:1031B0000092012301930292039269460C4806F0A3
:1031C000C7F990B900210A4806F0C4FB0DB05DF8BC
:1031D00004FBFFF73AFDD1E7FFF737FDD2E7FFF732
:1031E00034FDDBE7FFF731FDE1E7FFF72EFDE9E70F
:1031F000002800240000014000B58DB00023079393
:10320000089309930A930B930493059306930093F1
:103210000193029303932348234A026017224260DA
:1032200083604FF6FF72C2600361836105F0CEFFD9
:1032300048BB1C4806F02AF840BB042307935023E0
:103240000893002309930B9307A9164806F096FAF2
:10325000F8B900230493069304A9124806F052FC1F
:10326000D0B9002200920123019302920392694691
:103270000C4806F06DF990B900210A4806F06AFB87
:103280000DB05DF804FBFFF7E0FCD2E7FFF7DDFCD3
:10329000D3E7FFF7DAFCDCE7FFF7D7FCE1E7FFF75E
:1032A000D4FCE9E7E42800240004004000B58DB018
:1032B00000230793089309930A930B9304930593B0
:1032C000069300930193029303932448244A0260D7
:1032D0001722426083604FF6FF72C2600361836110
:1032E00005F074FF58BB1D4805F0D0FF50BB042308
:1032F0000793502308930223099300230B9307A9F4
:10330000164806F03BFA00BB00230493069304A979
:10331000124806F0F7FBD8B902230093012301936A
:1033200000220292039269460C4806F011F990B906
:1033300000210A4806F00EFB0DB05DF804FBFFF714
:1033400084FCD0E7FFF781FCD1E7FFF77EFCDBE7E9
:10335000FFF77BFCE0E7FFF778FCE9E74C28002467
:103360000018004000B58DB000230793089309931F
:103370000A930B9303684C4A934208D04B4A9342FA
:103380003AD04B4A934262D00DB05DF804FB494BF2
:10339000D3F8F02042F00102C3F8F020D3F8F02077
:1033A00002F001020192019AD3F8E02042F01002EB
:1033B000C3F8E020D3F8E03003F010030293029B3F
:1033C0004FF4007307930223089301230B9307A97B
:1033D000394802F091FF002211461A2001F040FB0B
:1033E0001A2001F073FB002211461B2001F038FB6C
:1033F0001B2001F06BFBC7E72E4BD3F8E82042F00F
:103400000202C3F8E820D3F8E82002F00202039297
:10341000039AD3F8E02042F00402C3F8E020D3F886
:10342000E03003F004030493049B4023079302233A
:1034300008930B9307A9214802F05EFF0022114672
:103440001D2001F00DFB1D2001F040FB9CE7194BF6
:10345000D3F8E82042F04002C3F8E820D3F8E8208F
:1034600002F040020592059AD3F8E02042F00202F1
:10347000C3F8E020D3F8E03003F002030693069B84
:103480004FF480430793022308930B9307A90C483A
:1034900002F032FF002211462B2001F0E1FA2B202E
:1034A00001F014FB70E700BF000001400004004081
:1034B000001800400044025800100258000802584A
:1034C000000402580368B3F1804F00D0704782B007
:1034D000074BD3F8E82042F00102C3F8E820D3F804
:1034E000E83003F001030193019B02B0704700BF75
:1034F0000044025800B587B0002301930293039360
:10350000049305930368B3F1804F02D007B05DF8D0
:1035100004FB0B4BD3F8E02042F00102C3F8E0209B
:10352000D3F8E03003F001030093009B01230193E3
:1035300002220292059301A9024802F0DDFEE5E7AE
:10354000004402580000025800B58BB000230793D6
:1035500008930993009301930293039304930593B3
:10356000069318484FF08042026017224260836041
:103570006422C2600361836105F058FEC8B900236C
:103580000793099307A90F4806F0BCFAA0B9602376
:103590000093322301930022029204926946094863
:1035A00005F0EEFE58B90748FFF7A4FF0BB05DF831
:1035B00004FBFFF74AFBE2E7FFF747FBE7E7FFF70C
:1035C00044FBF0E79828002438B504460268434BD2
:1035D0009A4204D02268424B9A424FD038BD037FB2
:1035E000012BF7D13F4B1B6833B33E4B1B68012BBC
:1035F00028D03D4B1A683D4B1B689A4234DA394B50
:103600001B68012B04DD374B1B68B3F5C87F1FDB3C
:10361000344B1B68B3F5C87F04DB324B1B68B3F532
:10362000AF6F1BDB01224021314802F079FF2D4AA8
:10363000136801331360CDE7012204212C4802F006
:103640006FFFD2E700220421294802F069FFD0E78A
:1036500001224021264802F063FFE8E700224021D2
:10366000234802F05DFFE2E71E4B1B68012BDEDD05
:10367000012240211E4802F053FFD8E7237F012B8F
:10368000ACD11C4800F066FA1B4A11681B4B23F8AA
:103690001100126833F812204EF660239A4206D9C0
:1036A000154B1A68154B4EF6602123F81210124B79
:1036B0001A68124C34F81210114A1568090A114898
:1036C00041551D681168013114F8154044541168C2
:1036D000023111601A6801321A607FE70000014070
:1036E00000040040F809002430290024080A0024BE
:1036F00000000258181B0024FC090024A81B002409
:10370000000A0024E01F002408B51A481A4B036081
:103710004FF46123436000238360C36003610C2284
:1037200042618361C36103624362836207F0C8FC44
:1037300098B900210F4807F003FE88B900210D4811
:1037400007F023FE78B90B4807F0DBFD70B90122C2
:103750000A49084807F086FD08BDFFF776FAE8E752
:10376000FFF773FAEAE7FFF770FAECE7FFF76DFA95
:10377000EDE700BF7C2A002400100140342900241A
:1037800030B5B9B00446002133913491359136916A
:103790003791C02202A808F007F922682F4B9A42FD
:1037A00001D039B030BD01220023CDE9022302A8A7
:1037B00003F0E8FD00284AD1294BD3F8F02042F06D
:1037C0001002C3F8F020D3F8F02002F010020092AB
:1037D000009AD3F8E02042F00102C3F8E020D3F8C9
:1037E000E03003F001030193019B4FF4C063339376
:1037F000022334930025359536930723379333A955
:10380000184802F079FD1848184B03602A234360DA
:1038100040238360C5604FF4806303614561856127
:10382000C5614FF480330362456201F0D3FB88B970
:103830000D4BE3679C6300221146252001F010F92F
:10384000252001F043F9E06F01F0C4FBA9E7FFF781
:10385000FCF9B1E7FFF7F9F9EAE700BF0010014012
:103860000044025800000258042A002410000240BC
:1038700008B502681A4B9A4200D008BD194A13884D
:10388000B2F90020002A09DB13F4804F11D0164A48
:1038900012780A2A08D0134B00221A8001221249FA
:1038A000124807F0DFFCE8E7114A1A430D4B1A8073
:1038B000F4E70D4A12780D2A0DD0C3F30D010D481F
:1038C000425401339BB2074A1380C72BE6D91346F3
:1038D00000221A80E2E743F48043024A1380DDE7C6
:1038E00000100140002A0024342900247C2A0024EE
:1038F0000080FFFF38290024DFF834D0FFF7C2FB37
:103900000C480D490D4A002302E0D458C45004333A
:10391000C4188C42F9D30A4A0A4C002301E0136010
:103920000432A242FBD307F05BFDFFF733FA704786
:103930000000082400000024DC090024D03801081D
:10394000DC0900245C2B0024FEE70000104B1B78F0
:103950000BB90120704710B504464FF47A70B0FBE4
:10396000F3F30C4A1068B0FBF3F001F0BDF868B94E
:103970000F2C01D901200AE0002221464FF0FF3030
:1039800001F06EF8044B1C60002000E0012010BD27
:10399000240000241C0000242800002410B503206B
:1039A00001F04CF803F046F90F498B69C3F3032388
:1039B0000E4AD35C03F01F03D8408B6903F00F035A
:1039C000D35C03F01F0320FA03F3094A1360094B89
:1039D00018600F20FFF7BAFF10B10124204610BD78
:1039E0000446FFF7C5FAF9E700440258843201089B
:1039F000200000241C000024034B1B78034A11689C
:103A00000B441360704700BF24000024102B0024D7
:103A1000014B1868704700BF102B0024014B186839
:103A2000000C70470010005C2DE9F04104460E4682
:103A300003684549454A934218BF8B4213D102F5AA
:103A40000072976807F01F072569082D12D0052F0F
:103A500018BF002F09D0092F07D0936813F4404FE7
:103A60002DD1042506E03A4AEBE7DB6813F0010F9D
:103A70001FD10425FFF7CCFF804623681A682A422D
:103A800023D1B6F1FF3FF8D0FFF7C2FFA0EB08004B
:103A9000B04201D8002EF0D123681B682B42ECD134
:103AA000636D43F004036365002384F85030032002
:103AB00045E0636D43F02003636501203FE0636DE3
:103AC00043F020036365012039E0626D42F4007227
:103AD0006265DA6812F4406F11D1627D7AB91A68B2
:103AE00012F0080F0BD0626D22F480726265626D75
:103AF00012F4805F03D1626D42F001026265134AE5
:103B000093420CD01A4693420CD0052F14BF0021CB
:103B100001213FB131B9092F04D0D26803E0A2F5E9
:103B20008072F0E7DA68082D06D012F4804F08D1D1
:103B30000C221A60002002E008221A600020BDE872
:103B4000F0810020FBE700BF00200240002102407E
:103B5000006302580368186C7047704770477047DD
:103B6000F8B5044603681D685E689649964A934214
:103B700018BF8B4240D1954B9F6807F01F0715F087
:103B8000020F10D016F0020F0DD0636D13F0100F5E
:103B900003D1636D43F400636365204600F09AFE31
:103BA000236802221A6015F0040F02D016F0040FE9
:103BB00005D115F0080F4FD016F0080F4CD0636DEB
:103BC00013F0100F03D1636D43F400736365236832
:103BD000DA6812F4406F39D17B4A93420ED01A460C
:103BE00093420ED0052F14BF002101214FB141B9DE
:103BF000092F06D0D26805E0754BBDE7A2F58072AB
:103C0000EEE7DA6812F4005F20D11A6812F0080FAC
:103C10001CD09A6812F0040F10D15A6822F00C02DE
:103C20005A60636D23F480736365636D13F4805F82
:103C30000CD1636D43F00103636507E0636D43F0EE
:103C400010036365A36D43F00103A3652046FFF7EE
:103C500084FF23680C221A6015F0200F02D016F0A2
:103C6000200F05D115F0400F63D016F0400F60D043
:103C7000636D13F0100F03D1636D43F4005363655C
:103C80002368DA6C12F4C07F19D10121DA6812F4CA
:103C9000406F16D101204C4A934214D01A469342E9
:103CA00014D0062F14BF4FF0000C4FF0010C6FB171
:103CB000BCF1000F0AD1072F08D0D26807E000211D
:103CC000E4E70020E7E7A2F58072E8E7DA6851B39D
:103CD00012F0007F03D030B312F4005F23D11968D3
:103CE00011F0400F1FD012F4001F1CD19A6812F07F
:103CF000080F10D15A6822F060025A60636D23F4F5
:103D000080536365636D13F4807F0CD1636D43F062
:103D10000103636507E0636D43F010036365A36D02
:103D200043F00103A365204600F0D0FD2368602224
:103D30001A6015F0800F02D016F0800F36D115F4FE
:103D4000807F02D016F4807F44D115F4007F02D02A
:103D500016F4007F4AD115F0100F20D016F0100F86
:103D60001DD0236B6BB1002F4ED023681549164A26
:103D7000934218BF8B4245D1144B9B6813F4404FBC
:103D80000AD0636D43F480636365A36D43F002035F
:103D9000A3652046FFF7E3FE236810221A6015F49E
:103DA000806F02D016F4806F34D1F8BD636D43F498
:103DB000803363652046FFF7D1FE236880221A60B6
:103DC000BDE700BF00200240002102400023024066
:103DD00000630258636D43F400336365204600F0CE
:103DE00077FD23684FF480721A60AEE7636D43F489
:103DF00080236365204600F06CFD23684FF4007259
:103E00001A60A8E70B4BB8E72368DB6813F0030FD1
:103E1000C2D0B6E7636D43F480436365A36D43F09E
:103E20000803A36523684FF480621A60204600F0FF
:103E30004EFDBAE700630258F0B583B0002201924C
:103E400090F85020012A00F055820346012280F8A4
:103E500050200068826812F0040F09D05A6D42F0B9
:103E600020025A650120002283F8502003B0F0BDE3
:103E70000A68C2F31304002C4ED1C2F384620124F9
:103E80009440C2692243C2611D684C683035220AE1
:103E9000920002F00C02A85804F01F0E1F2404FA2E
:103EA0000EF420EA04000C68C4F3846C0CFA0EFCD7
:103EB00040EA0C00A8501C68A26812F0040200D06E
:103EC0000122A06810F0080000D0012002432FD08A
:103ED0001868826812F0010F40F008820A68CD6805
:103EE000D0F8C040C2F3130624EA060405F0180C0B
:103EF000B24D25FA0CF52A40C2F313022243C0F852
:103F0000C020C868AE4A904200F0B0800A68002A1B
:103F1000C0F26B810020A6E792FAA2F232B1B2FAA7
:103F200082F202F01F0201249440AAE72022F8E75F
:103F30000F688D681434780E800000F00400265855
:103F4000C7F3045E4FF0070C0CFA0EFC26EA0C0CCB
:103F500005FA0EF54CEA050525509A48006800F070
:103F60007040B0F1805F0BD01C68E06810F0100F5B
:103F700039D14869E468C4F382046400A04006E0D3
:103F800048691C68E468C4F382046400A0400D69B9
:103F9000042D36D01F680E68603757F8254004F0AE
:103FA000004406F0F8463043204347F825001868DF
:103FB0000E694C7E012C1ED01546603050F826400C
:103FC00024F000442C4340F826401D680C69087E0C
:103FD000012813D0286920F4F04004F01F04A24007
:103FE00002432A6174E74869E468A40804F0040401
:103FF0006400A040CBE74FF00045DEE74FF40062DD
:10400000E8E71868026E02F0F8420C68B2EB846FC1
:104010001DD01868426E02F0F8420C68B2EB846F53
:104020001AD01868826E02F0F8420C68B2EB846F06
:1040300017D01868C26E02F0F8420C68B2EB846FB9
:104040007FF446AFC26E22F00042C26640E7026EC5
:1040500022F000420266DCE7426E22F00042426635
:10406000DFE7826E22F000428266E2E71C680A689F
:10407000C2F31305002D34D1900E013000F01F0063
:1040800009288CBF00200120002861D0002D37D1E5
:10409000900E0130800600F0F840002D3CD1960EC5
:1040A000013606F01F070126BE403043002D41D1E6
:1040B000920E013202F01F0202EB4202120502438D
:1040C00088681434550EAD0005F004056659C2F336
:1040D00004520727974026EA070690403043605174
:1040E00014E792FAA2F048B1B0FA80F0013000F083
:1040F0001F0009288CBF00200120C5E72020F5E71C
:1041000092FAA2F030B1B0FA80F00130800600F0EF
:10411000F840C2E72020F8E792FAA2F646B1B6FAD4
:1041200086F6013606F01F06012707FA06F6BCE7F9
:104130002026F6E792FAA2F242B1B2FA82F20132F6
:1041400002F01F0202EB42021205B8E72022F6E756
:10415000CDB9900E0130800600F0F840FDB9960E02
:10416000013606F01F070126BE40304365BB920EA4
:10417000013202F01F0202EB42021E3A120542F027
:10418000007202439CE792FAA2F030B1B0FA80F0DC
:104190000130800600F0F840E0E72020F8E792FACE
:1041A000A2F646B1B6FA86F6013606F01F060127DA
:1041B00007FA06F6D9E72026F6E700BFFFFF0F0053
:1041C0000000FF470010005C92FAA2F25AB1B2FA66
:1041D00082F2013202F01F0202EB42021E3A120585
:1041E00042F00072CDE72022F3E719684248434CC1
:1041F000A14218BF81420CBF0120002021D1404EB6
:10420000B56805F0E077F0B13B48806810F0010038
:1042100000D00120394CA46814F0010400D001241E
:1042200020430CBF01200020002859D0354882428D
:1042300012D03548824231D0344882423FD00020EB
:1042400011E6334EDCE73348806810F0010000D0FF
:10425000012080F00100E7E715F4000FE9D12D4AB5
:10426000914201D00020FEE547F40002B16821F040
:10427000E0710A43B260284A126892092749A1FBFB
:104280000212920901325200019202E0019A013AAF
:104290000192019A002AF9D10020E4E515F0807F0F
:1042A000CAD11C4A914201D00020DCE547F080725F
:1042B000B16821F0E0710A43B2600020D3E515F443
:1042C000800F15D1134A914201D00020CBE547F46D
:1042D0008002B16821F0E0710A43B2600020C2E5BB
:1042E0005A6D42F020025A650120BCE50020BAE573
:1042F0000020B8E50220B9E500200240002102407C
:1043000000230240000084CB000052C70000B8CF59
:1043100000630258006002581C000024632D3E0513
:1043200038B503689A6812F0010F56D104469968AF
:104330002B4A114209D0436D43F010034365836D4E
:1043400043F001038365012048E09968254A0A404B
:1043500042F001029A60FFF75BFB054623682249A1
:10436000224A934218BF8B420DD102F50072926827
:1043700002F01F021D498B4207D01946994207D00F
:1043800032B100202AE01A4AF1E7A1F58071F5E781
:1043900023681A6812F0010F1DD19A6812F0010FFC
:1043A00005D199680F4A0A4042F001029A60FFF76E
:1043B0002FFB401B0228EBD923681B6813F0010F69
:1043C000E6D1636D43F010036365A36D43F0010311
:1043D000A365012002E0002000E0002038BD00BFFE
:1043E0003F000080C0FFFF7F00200240002102400C
:1043F0000063025838B5044603683E493E4A93427A
:1044000018BF8B4252D102F50072956805F01F0566
:104410009B6813F0040F69D194F85030012B67D0DA
:10442000012384F850302046FFF77AFF002859D145
:10443000626DA0F60273134043F4807363652368D2
:104440002D4A934234D01A46934200D01DB9626D72
:1044500022F480126265626D12F4805F2BD0A26D2F
:1044600022F00602A2651C221A60002384F8503054
:104470002368214A934221D01A46934221D0052D28
:1044800014BF00210121E5B1D9B9092D19D0636DFF
:1044900043F480136365D36813F0007F27D0636D06
:1044A00023F4405343F48053636520E0134AACE7A0
:1044B000A2F58072C8E70022A265D4E7A2F5807257
:1044C000DBE7DA6812F0007F05D0626D22F440521B
:1044D00042F4805262659968094A0A4042F0040237
:1044E0009A6004E0002384F8503000E0022038BDD8
:1044F0000220FCE700200240002102400063025835
:10450000C0FFFF7F38B5044603684F494F4A9342C6
:1045100018BF8B4223D14E4B9B6813F4403F14BF0E
:10452000012300234BB302F0DBFD05466368B3F5BE
:10453000003F1CD0B3F5403F1DD0B3F5803F16D0EF
:10454000FFF76CFA41F20303984258D8414B9D4261
:104550004FD92268936843F48073936038BD3E4B13
:104560009B6813F4403F14BF01230023DAE71B0CC0
:10457000B5FBF3F5E4E78508E2E74FF400200021FE
:1045800003F0A6FF05466368B3F5101F2DD022D8AF
:10459000B3F5E01F27D004D9B3F5001FD0D14509EA
:1045A000CEE7B3F5801F0DD006D9B3F5A01F09D013
:1045B000B3F5C01F06D0C3E7B3F5002F02D0B3F5A3
:1045C000402F04D19B0C5B00B5FBF3F5B8E7B3F5C6
:1045D000802FF7D0B4E7B3F5201F08D0B3F5301F14
:1045E000AED1050AACE70509AAE78509A8E7C50920
:1045F000A6E72268936823F480739360AEE7174BB5
:104600009D4205D82268936823F440739360A5E720
:10461000134B9D4207D82268936823F4407343F4F8
:10462000807393609AE70F4B9D4207D82268936886
:1046300023F4407343F4007393608FE72268936818
:1046400043F44073936089E7002002400021024058
:1046500000230240002D31010063025821BCBE003E
:1046600041787D0181F0FA0230B583B000230193D7
:10467000002800F010810446436DEBB123689A686E
:1046800012F0005F03D09968844A0A409A60236858
:104690009A6812F0805F1CD19968814A0A4042F002
:1046A00080529A607F4B1B689B097F4AA2FB0323C1
:1046B0009B090133019309E0FDF732FC0023A36558
:1046C00084F85030DAE7019B013B0193019B002BFA
:1046D000F9D12268936813F0805F40F09C80636D8D
:1046E00043F010036365A36D43F00103A365012547
:1046F000936813F0040300D00123616D11F0100FD3
:1047000040F0C180002B40F0BE80636D23F48173C4
:1047100043F002036365936813F0010F21D16349ED
:10472000634B9A4218BF8A420CBF0122002274D107
:104730008B6813F0010300D001235D49896811F0F3
:10474000010100D001210B430CBF0123002343B121
:10475000002A6BD0574963688A6822F47C1213439D
:104760008B60FFF75BF941F20303984202D9A3681B
:10477000102B5DD0627D236B43EA4233A268134362
:10478000227F43EA0243227F012A5CD0626A22B17F
:1047900002F47872A16A0A4313432168C868464A42
:1047A00002401343CB6021688B6813F0040300D0F0
:1047B00001238A6812F0080200D0012213431BD1A2
:1047C000227DE36A43EA8232C8683C4B03401343CC
:1047D000CB6094F83830012B3AD02268136923F06B
:1047E000010313612268136923F07043616B0B436B
:1047F00013612046FFF786FEE368012B3AD022685A
:10480000136B23F00F031363636D23F0030343F073
:10481000010363653CE000256AE7294B9B6813F0C0
:10482000010300D0012383F0010390E7254992E7BB
:10483000617D226B42EA41321343227F43EA024305
:1048400043F00C039FE7226A013A43EA42439DE7A3
:10485000206802691C4B1340E26B511E226C42EA35
:104860000142616C0A43A16C0A43134343F0010304
:104870000361B7E721680B6B23F00F03A269013ACC
:1048800013430B63C0E7636D43F0100363650125B9
:10489000284603B030BD0125FAE700BFC0FFFF5F27
:1048A000C0FFFF6F1C000024632D3E050020024066
:1048B000002102400023024003C0F0FFFCBFFFFFC5
:1048C00000600258006302581EF800FC70477047F1
:1048D000704770477047000090F85020012A00F0A0
:1048E000A18030B49AB00346012280F85020002203
:1048F0001692179200684C4A904242D000220192D0
:10490000019A002A41D0926812F0040200D00122DC
:10491000846814F0040F76D1002A74D1424C434AC3
:10492000904218BFA04239D102F5007208680028F1
:104930003FD0906820F440404C6820439060186855
:10494000394D3A4CA04218BFA84229D1A86810F0AE
:10495000010000D00120354CA46814F0010400D0FF
:10496000012420430CBF01200020002856D0946869
:104970002F4820400C68896821430843906000203C
:1049800046E002F580720192BAE75A6D42F02002C9
:104990005A65002283F8502001203CE0254AC5E7F3
:1049A0002548806810F0010000D0012080F001004F
:1049B000DBE7916821F44041916019681A4C1B486B
:1049C000814218BFA14215D1A16811F0010100D0A8
:1049D00001211648806810F0010000D00120014339
:1049E0000CBF01210021D9B19068114901409160AB
:1049F00000200DE01049896811F0010100D001216B
:104A000081F00101EFE75A6D42F020025A65012062
:104A1000002283F850201AB030BC70470020F7E71E
:104A20000020F5E7022070470020024000210240EC
:104A3000E0F0FFFF00630258006002580649CB68AF
:104A400023F4E0631B041B0C000200F4E06003434A
:104A5000024A1A43CA60704700ED00E00000FA0500
:104A600000B5174BDB68C3F30223C3F1070CBCF19D
:104A7000040F28BF4FF0040C03F1040EBEF1060F23
:104A800014D9033B4FF0FF3E0EFA0CFC21EA0C0157
:104A900099400EFA03F322EA03031943002807DBC7
:104AA0000901C9B2074B19545DF804FB0023E9E77B
:104AB00000F00F000901C9B2034B1954F4E700BF1D
:104AC00000ED00E000E400E014ED00E0002807DB6A
:104AD00000F01F02400901239340024A42F82030AF
:104AE000704700BF00E100E00138B0F1807F0BD2D9
:104AF0004FF0E0235861054AF02182F8231000208E
:104B0000986107221A6170470120704700ED00E0AC
:104B1000BFF35F8F044B5A6A22F480325A6200223C
:104B2000C3F89420704700BF00ED00E040F00100A2
:104B3000054BC3F894005A6A42F480325A62BFF3BC
:104B40004F8FBFF36F8F704700ED00E04278164B38
:104B5000C3F898200378FBB14368134AC2F89C302D
:104B6000017BC37A1B0643EA0173817A43EAC1439E
:104B7000417B43EA8143817B43EA4143C17B43EA72
:104B80000143417A43EA0123017A43EA4103017870
:104B90000B43C2F8A0307047034B0022C3F89C209F
:104BA000C3F8A020704700BF00ED00E0F0B4876DAF
:104BB0000468664E664DAC4218BFB44242D0183508
:104BC000AC423FD01835AC423CD01835AC4239D05D
:104BD0001835AC4236D01835AC4233D01835AC421B
:104BE00030D005F55675AC422CD01835AC4229D0E2
:104BF0001835AC4226D01835AC4223D01835AC421B
:104C000020D01835AC421DD01835AC421AD018351A
:104C1000AC4217D04F4DAC4214D01435AC4211D039
:104C20001435AC420ED01435AC420BD01435AC4226
:104C300008D01435AC4205D01435AC4202D014353E
:104C4000AC4207D1446E856E6560C46E14B1046FCA
:104C5000456F656004683D4E3D4DAC4218BFB4429F
:104C600052D01835AC424FD01835AC424CD0183524
:104C7000AC4249D01835AC4246D01835AC4243D08E
:104C80001835AC4240D005F55675AC423CD01835CD
:104C9000AC4239D01835AC4236D01835AC4233D09E
:104CA0001835AC4230D01835AC422DD01835AC4256
:104CB0002AD01835AC4227D0264E274DAC4218BF1B
:104CC000B44211D0254DAC420ED01435AC420BD0BD
:104CD0001435AC4208D01435AC4205D01435AC4282
:104CE00002D01435AC4224D1C46D04F01F05012458
:104CF000AC407C60046863608368402B20D003680C
:104D000099600368DA6014E0C46D04F01F0C3F245E
:104D100004FA0CF4BC6005682C6824F480242C6030
:104D2000046863608368402B05D00368996003685A
:104D3000DA60F0BC704703689A600368D960F8E7EE
:104D400003689A600368D960F3E700BF100002406F
:104D500028000240085402581C540258305402588B
:104D600003682749274A934218BF8B422FD0183235
:104D700093422CD01832934229D01832934226D035
:104D80001832934223D01832934220D018329342E3
:104D90001DD002F55672934219D01832934216D0A4
:104DA0001832934213D01832934210D018329342E3
:104DB0000DD0183293420AD01832934207D01832DD
:104DC000934204D023F0FF038365806D704710B4D5
:104DD000D9B210390C4AA2FB0142C2F302120B4CA9
:104DE000A25CC2655F2906D9094A1A40043282656D
:104DF000806D10BC7047064A1A408265F8E700BF14
:104E00001000024028000240ABAAAAAA943201086E
:104E100000FCFFFF83699BB9836A012B0AD0022B38
:104E200002D00BB100207047C36A13F0807F2AD1F3
:104E300000207047C36AB3F1C07F26D000207047BE
:104E4000B3F5005F0AD0836A022B26D9032B26D143
:104E5000C36A13F0807F24D100207047836A032B3C
:104E600003D8DFE803F01404140A00207047C36A73
:104E700013F0807F0DD100207047C36AB3F1C07F6B
:104E800009D00020704701207047012070470120A1
:104E900070470120704701207047012070470020B3
:104EA000704701207047000003682249224A93425C
:104EB00018BF8B4228D01432934225D0143293422B
:104EC00022D0143293421FD0143293421CD0143299
:104ED000934219D01432934216D0DAB2103A1749DD
:104EE000A1FB0212120916491944A8291FD9154B12
:104EF00013449B000366144B436602F01F02012318
:104F000003FA02F282667047DBB2083B0F4AA2FB4B
:104F100003230F4A02EB1312920002660D4A426607
:104F2000C3F30413012202FA03F3836670470832C5
:104F3000DDE700BF085402581C540258ABAAAAAAC5
:104F4000F0FBFDBF0082001080080240CDCCCCCC2D
:104F5000009600168058025801794A1E072A2CD85C
:104F600030B40368154D164CA34218BFAB4218D09D
:104F70001434A34215D01434A34212D01434A342E3
:104F80000FD01434A3420CD01434A34209D01434EB
:104F9000A34206D00B4B0B449B00C3660A4B03672E
:104FA00005E00A4B0B449B00C366094B03670123D2
:104FB00003FA02F2426730BC704770470854025847
:104FC0001C5402583F820010400902403F960016D0
:104FD0004059025870B50446FEF71AFD002C00F047
:104FE000B681054623685349534A934218BF8B4202
:104FF0000CBF0122002250D030318B424DD01831ED
:105000008B424AD018318B4247D018318B4244D062
:1050100018318B4241D018318B423ED001F5567188
:105020008B423AD018318B4237D018318B4234D072
:1050300018318B4231D018318B422ED018318B422F
:105040002BD018318B4228D018318B4225D03B49C8
:105050003B4A934218BF8B4200F03181394A934258
:1050600000F02D811432934200F0298114329342D2
:1050700000F025811432934200F0218114329342D2
:1050800000F01D811432934200F0198140236365C2
:10509000032384F8353001204AE0022184F83510DA
:1050A000002184F834107ABB274A93422CD018325E
:1050B000934229D01832934226D01832934223D0FB
:1050C0001832934220D0183293421DD002F5567206
:1050D000934219D01832934216D01832934213D00B
:1050E0001832934210D0183293420DD018329342A6
:1050F0000AD01832934207D01832934204D01A686B
:1051000022F001021A6003E01A6822F001021A601C
:1051100023681A6812F0010F18D0FEF779FC431BC0
:10512000052BF5D920236365032384F8353001204E
:1051300070BD00BF10000240280002400854025811
:105140001C54025830540258400002401A688148EA
:105150001040A168E2680A4321690A4361690A4371
:10516000A1690A43E1690A43216A0A430243616A69
:10517000042900F099807849086878490140B1F124
:10518000005F11D36168A1F12905A1F13F00032857
:1051900088BF052D06D9A1F14700012802D94F3952
:1051A000032901D842F480121A602668756925F037
:1051B0000705636A1D43042B08D1A36A1D43E36AF4
:1051C00023B12046FFF726FE002872D175612046E4
:1051D000FFF7C6FDE36D03F01F023F23934083609A
:1051E00023685F495F4A934218BF8B4242D018320E
:1051F00093423FD0183293423CD01832934239D078
:105200001832934236D01832934233D01832934238
:1052100030D002F5567293422CD01832934229D0E6
:105220001832934226D01832934223D01832934238
:1052300020D0183293421DD0183293421AD018321F
:10524000934217D0484A934214D01432934211D05B
:10525000143293420ED0143293420BD01432934244
:1052600008D01432934205D01432934202D0143243
:10527000934213D12046FFF717FEA368802B59D025
:10528000236E22791A60636EA26E5A606368013BD6
:10529000072B52D90023E36623676367002060650C
:1052A000012384F8353043E7E16A206B01430A4368
:1052B00061E740236365012084F8350038E7022266
:1052C00084F83520002284F834201A6827491140D8
:1052D000A268402A2CD0802A27D00022E06842EA27
:1052E000D002206942EAD002606942EAD002A06995
:1052F00042EAD002E06942EAD002206A42EA101291
:105300000A431A6022681A4B13441A4AA2FB032369
:105310001B099B00E3652046FFF722FDE26D02F0CA
:105320001F0101228A4042605AE74FF48042D5E7CC
:105330001022D3E700236360A2E72046FFF70CFEAC
:10534000E36E00221A60236F626F5A60A6E70120A5
:10535000EEE600BF3F8010FE0010005C0000FFFF83
:105360001000024028000240085402580F00FEFFBF
:10537000F8ABFDA7CDCCCCCC002800F03E8170B5B9
:10538000044690F83400012800F03981012084F8A7
:10539000340094F83500C0B2012807D04FF4006300
:1053A0006365002384F83430012070BD022084F846
:1053B0003500002060652068924E934DA84218BFCA
:1053C000B0422FD01835A8422CD01835A84229D089
:1053D0001835A84226D01835A84223D01835A8423F
:1053E00020D01835A8421DD005F55675A84219D011
:1053F0001835A84216D01835A84213D01835A8423F
:1054000010D01835A8420DD01835A8420AD018354A
:10541000A84207D01835A84204D0056825F0010538
:10542000056003E0056825F0010505602046FFF7EB
:10543000BDFB23687349744A934218BF8B4238D02E
:105440001832934235D01832934232D018329342F8
:105450002FD0183293422CD01832934229D01832D0
:10546000934226D002F55672934222D018329342CC
:105470001FD0183293421CD01832934219D01832E0
:10548000934216D01832934213D01832934210D060
:10549000183293420DD01A6822F00E0242F00A022E
:1054A0001A60236C93B12268136843F004031360FD
:1054B0000CE01A6822F01E0242F016021A60236CF9
:1054C00023B12268136843F00803136023684D4931
:1054D0004D4A934218BF8B4242D0183293423FD07C
:1054E000183293423CD01832934239D0183293424A
:1054F00036D01832934233D01832934230D002F56E
:10550000567293422CD01832934229D018329342CB
:1055100026D01832934223D01832934220D018322A
:1055200093421DD0183293421AD01832934217D0AA
:10553000364A934214D01432934211D0143293421B
:105540000ED0143293420BD01432934208D014324E
:10555000934205D01432934202D0143293420ED1BA
:10556000236E1A6812F4803F03D01A6842F48072E6
:105570001A60E36E1BB11A6842F480721A602368E5
:105580002049214A934218BF8B4230D018329342AF
:105590002DD0183293422AD01832934227D0183295
:1055A000934224D01832934221D0183293421ED015
:1055B00002F5567293421AD01832934217D018321D
:1055C000934214D01832934211D0183293420ED025
:1055D000183293420BD01832934208D018329342BB
:1055E00005D01A6842F001021A600020DDE61A6850
:1055F00042F001021A600020D7E601207047022025
:10560000D3E600BF100002402800024008540258B0
:1056100070B50446FEF7FCF9002C00F091810546B8
:1056200094F83530DBB2022B06D08023636500236B
:1056300084F83430012070BD23688C498C4A934231
:1056400018BF8B4230D0183293422DD0183293427B
:105650002AD01832934227D01832934224D01832DD
:10566000934221D0183293421ED002F556729342D3
:105670001AD01832934217D01832934214D01832ED
:10568000934211D0183293420ED0183293420BD06D
:105690001832934208D01832934205D01A6822F08B
:1056A0000E021A60266809E01A6822F01E021A60CB
:1056B0002268536923F080035361266823686B498D
:1056C0006B4A934218BF8B4242D0183293423FD06C
:1056D000183293423CD01832934239D01832934258
:1056E00036D01832934233D01832934230D002F57C
:1056F000567293422CD01832934229D018329342DA
:1057000026D01832934223D01832934220D0183238
:1057100093421DD0183293421AD01832934217D0B8
:10572000544A934214D01432934211D0143293420B
:105730000ED0143293420BD01432934208D014325C
:10574000934205D01432934202D01432934204D1D2
:10575000226E136823F48073136023684349444A1C
:10576000934218BF8B422FD0183293422CD018325C
:10577000934229D01832934226D01832934223D034
:105780001832934220D0183293421DD002F556723F
:10579000934219D01832934216D01832934213D044
:1057A0001832934210D0183293420DD018329342DF
:1057B0000AD01832934207D01832934204D01A68A4
:1057C00022F001021A6003E01A6822F001021A6056
:1057D000336813F0010F0ED0FEF71AF9431B052BA7
:1057E000F6D920236365032384F83530002384F839
:1057F000343001201FE723681C491D4A934218BF1B
:105800008B4239D01832934236D01832934233D07B
:105810001832934230D0183293422DD0183293422E
:105820002AD01832934227D002F55672934223D0E1
:105830001832934220D0183293421DD0183293422E
:105840001AD01832934217D01832934214D018321B
:10585000934211D0183293420ED0A16DE36D03F044
:105860001F02012393404B600DE000BF1000024077
:105870002800024008540258A16DE36D03F01F0296
:105880003F2393408B6023682E492F4A934218BFD1
:105890008B4242D0183293423FD0183293423CD0D0
:1058A0001832934239D01832934236D0183293428C
:1058B00033D01832934230D002F5567293422CD036
:1058C0001832934229D01832934226D0183293428C
:1058D00023D01832934220D0183293421DD0183270
:1058E00093421AD01832934217D0184A934214D0D8
:1058F0001432934211D0143293420ED01432934298
:105900000BD01432934208D01432934205D0143293
:10591000934202D0143293420BD1636EA26E5A604E
:10592000E36E33B11A6822F480721A60236F626FDB
:105930005A60012384F83530002084F834007AE678
:10594000012078E610000240280002400854025866
:10595000002800F0298108B5024690F83530DBB206
:10596000022B03D080234365012008BD03689048C3
:1059700090498B4218BF83420CBF0121002166D0A1
:105980003030834263D01830834260D01830834275
:105990005DD0183083425AD01830834257D0183027
:1059A000834254D000F55670834250D01830834261
:1059B0004DD0183083424AD01830834247D0183037
:1059C000834244D01830834241D0183083423ED0C5
:1059D000183083423BD0196821F00E01196013681A
:1059E000A0F5956073498B4218BF83426AD0724913
:1059F0008B4267D018318B4264D018318B4261D012
:105A000018318B425ED018318B425BD018318B42FB
:105A100058D001F556718B4254D018318B4251D079
:105A200018318B424ED018318B424BD018318B42FB
:105A300048D018318B4245D018318B4242D01831B2
:105A40008B423FD0196821F0010119603EE004202B
:105A500082F8350081BB584A93422DD018329342C8
:105A60002AD01832934227D01832934224D01832C9
:105A7000934221D0183293421ED002F556729342BF
:105A80001AD01832934217D01832934214D01832D9
:105A9000934211D0183293420ED0183293420BD059
:105AA0001832934208D01832934205D01A6822F077
:105AB00001021A60002058E71A6822F001021A60F9
:105AC000002052E7196821F0010119601368384875
:105AD00038498B4218BF834242D018318B423FD0A5
:105AE00018318B423CD018318B4239D018318B425F
:105AF00036D018318B4233D018318B4230D001F57B
:105B000056718B422CD018318B4229D018318B42E0
:105B100026D018318B4223D018318B4220D0183137
:105B20008B421DD018318B421AD018318B4217D0BE
:105B300022498B4214D014318B4211D014318B4244
:105B40000ED014318B420BD014318B4208D014315B
:105B50008B4205D014318B4202D014318B4217D1C5
:105B6000116E0B6823F480730B60906DD36D03F09E
:105B70001F0101238B404360536E916E5960D36EB9
:105B800033B1196821F480711960136F516F596036
:105B9000012382F83530002382F83430136D2BB1A5
:105BA000104698470020E0E6012070470020DCE620
:105BB00010000240280002404000024008540258F1
:105BC000F0B583B00446002301937D4B1D687D4BE7
:105BD000A3FB0535AD0A876D3E68D7F800C00368A2
:105BE00079497A48834218BF8B420CBF01200020BC
:105BF00061D0774A93425ED0183293425BD018321C
:105C0000934258D01832934255D01832934252D012
:105C1000183293424FD002F5567293424BD018324D
:105C2000934248D01832934245D01832934242D022
:105C3000183293423FD0183293423CD018329342EC
:105C400039D01832934236D06249634A934218BF22
:105C50008B4212D0614A93420FD0143293420CD03F
:105C60001432934209D01432934206D01432934234
:105C700003D01432934240F061821A68E16D01F062
:105C80001F010420884010EA0C0F00F0A78212F0D8
:105C9000040F00F0A382786012F4004F00F05A82E3
:105CA00012F4803F40F05082A36C002B00F046823B
:105CB0002046984742E2E26D02F01F0108228A4026
:105CC000324241D070BB424A93422BD018329342A9
:105CD00028D01832934225D01832934222D018325D
:105CE00093421FD0183293421CD002F55672934251
:105CF00018D01832934215D01832934212D018326D
:105D000093420FD0183293420CD01832934209D0EC
:105D10001832934206D01832934203D01A68C2F365
:105D2000C00202E01A68C2F380026AB11A6822F067
:105D300004021A60E36D03F01F0208239340BB6066
:105D4000636D43F001036365E26D02F01F0226FA02
:105D500002F313F0010F47D023681B481B498B4205
:105D600018BF83423CD018318B4239D018318B4256
:105D700036D018318B4233D018318B4230D01831A5
:105D80008B422DD018318B422AD001F556718B42AF
:105D900026D018318B4223D018318B4220D01831B5
:105DA0008B421DD018318B421AD018318B4217D03C
:105DB00018318B4214D018318B4211D01B6813E07C
:105DC0001C000024B5814E1B100002402800024038
:105DD00040000240085402581C54025830540258E3
:105DE0005B6913F0800F3BD1E36D03F01F030422C6
:105DF00002FA03F3334240D02268964896498A4219
:105E000018BF824235D018318A4232D018318A42C6
:105E10002FD018318A422CD018318A4229D018311B
:105E20008A4226D018318A4223D001F556718A421F
:105E30001FD018318A421CD018318A4219D018312B
:105E40008A4216D018318A4213D018318A4210D0B3
:105E500018318A420DD018318A420AD013680CE0FA
:105E6000012303FA02F2BA60636D43F00203636533
:105E7000BAE7126812F0020F3DD1E36D03F01F0381
:105E8000102202FA03F333425FD02268714872494C
:105E90008A4218BF824234D018318A4231D0183138
:105EA0008A422ED018318A422BD018318A4228D00B
:105EB00018318A4225D018318A4222D001F5567114
:105EC0008A421ED018318A421BD018318A4218D01B
:105ED00018318A4215D018318A4212D018318A42BC
:105EE0000FD018318A420CD018318A4209D012687A
:105EF000C2F3800208E0BB60636D43F00403636596
:105F0000BBE71268C2F3C002FAB1BB6023681A682B
:105F100012F4802F0DD01B6813F4002F04D1236CD2
:105F20009BB12046984710E0A36C73B12046984778
:105F30000BE01A6812F4807F03D11A6822F008027D
:105F40001A60236C0BB120469847E36D03F01F03E2
:105F5000202202FA03F3334200F0928022683D4887
:105F60003D498A4218BF82422ED018318A422BD036
:105F700018318A4228D018318A4225D018318A42F5
:105F800022D018318A421FD018318A421CD001F524
:105F900056718A4218D018318A4215D018318A4277
:105FA00012D018318A420FD018318A420CD01831E1
:105FB0008A4209D018318A4206D018318A4203D069
:105FC0001268C2F3400202E01268C2F30012002A13
:105FD00056D0BB6094F83530DBB2042B0ED023686A
:105FE0001A6812F4802F39D01B6813F4002F2CD1BB
:105FF000636C002B44D02046984741E02268136828
:1060000023F0160313602268536923F08003536161
:10601000236CB3B12268136823F008031360E36DA7
:1060200003F01F023F239340BB60012384F8353007
:10603000002384F83430236D002B7FD0204698470E
:106040007CE0A36C002BE5D1E9E7E36BC3B120460C
:10605000984715E010000240280002401A6812F428
:10606000807F09D11A6822F010021A60012384F897
:106070003530002384F83430E36B0BB12046984769
:10608000636D002B5AD0636D13F0010F52D00423BF
:1060900084F8353023689649964A934218BF8B425C
:1060A0002FD0183293422CD01832934229D0183274
:1060B000934226D01832934223D01832934220D0F4
:1060C000183293421DD002F55672934219D01832FD
:1060D000934216D01832934213D01832934210D004
:1060E000183293420DD0183293420AD0183293429C
:1060F00007D01832934204D01A6822F001021A60C5
:1061000003E01A6822F001021A60019B0133019337
:10611000AB4204D823681B6813F0010FF5D1236844
:106120001B6813F0010F0BD0032384F835300023D4
:1061300084F83430E36C0BB12046984703B0F0BDCF
:10614000012384F83530F2E7236C002BF6D020468B
:106150009847F3E712F0200F3AD123686449654A63
:10616000934218BF8B422FD0183293422CD0183252
:10617000934229D01832934226D01832934223D02A
:106180001832934220D0183293421DD002F5567235
:10619000934219D01832934216D01832934213D03A
:1061A0001832934210D0183293420DD018329342D5
:1061B0000AD01832934207D01832934204D01A689A
:1061C00022F004021A6003E01A6822F008021A6042
:1061D000236C002BB2D020469847AFE702208840BE
:1061E00010EA0C0F60D012F0020F5DD0786012F44C
:1061F000004F0ED012F4803F05D1636C002B9DD070
:10620000204698479AE7E36B002B97D020469847A3
:1062100094E712F0200F40D123683549354A934264
:1062200018BF8B422FD0183293422CD01832934291
:1062300029D01832934226D01832934223D01832F4
:10624000934220D0183293421DD002F556729342E9
:1062500019D01832934216D01832934213D0183204
:10626000934210D0183293420DD0183293420AD084
:106270001832934207D01832934204D01A6822F0A1
:106280000A021A6003E01A6822F014021A6001235D
:1062900084F83530002384F83430E36B002B3FF46E
:1062A0004DAF2046984749E7082000FA01F111EA6E
:1062B0000C0F3FF443AF12F0080F3FF43FAF1A68E2
:1062C00022F00E021A60E36D03F01F03012202FAAE
:1062D00003F37B60626584F83520002384F8343052
:1062E000E36C002B3FF42AAF2046984726E700BF17
:1062F000100002402800024070B582B000236EE01A
:1063000085685E000324B44025EA0405CC68B440E7
:106310002C438460446824EA0C0C4C68C4F30014D9
:106320009C4044EA0C0444606CE0DD08083550F8F9
:10633000256003F007044FEA840C0F2404FA0CF4E0
:1063400026EA040E0C6904FA0CF444EA0E0440F840
:1063500025406FE0092400E0002404FA0EF42C43E9
:106360000CF1020C6B4D45F82C404FF0B044256801
:10637000D44325EA0206D1F804C01CF4801F01D0E2
:1063800042EA05064FF0B0452E606D6804EA050646
:10639000D1F804C01CF4001F01D042EA05064FF0FA
:1063A000B0456E60D5F8845004EA0506D1F804C003
:1063B0001CF4003F01D042EA05064FF0B045C5F895
:1063C0008460D5F880502C404E6816F4803F01D090
:1063D00042EA05044FF0B042C2F8804001330A6837
:1063E00032FA03F400F093804FF0010C0CFA03FC36
:1063F0001CEA0202F2D04C6804F00304013C012CB8
:106400007FF67EAF4C6804F00304032C0CD0C46804
:106410005D004FF0030C0CFA05FC24EA0C0C8C68B0
:10642000AC4044EA0C04C4604C6804F00304022C41
:106430003FF47BAF04684FEA430E4FF0030C0CFAB5
:106440000EFC24EA0C0C4C6804F0030404FA0EF46D
:1064500044EA0C0404604C6814F4403FBED02E4C57
:10646000D4F8F45045F00205C4F8F450D4F8F440E0
:1064700004F002040194019C4FEA930C0CF1020514
:10648000244C54F8255003F003044FEA840E0F24E3
:1064900004FA0EF425EA0405204CA0423FF45CAF58
:1064A00004F58064A04222D004F58064A04220D08C
:1064B00004F58064A0421ED004F58064A0421CD084
:1064C00004F58064A0421AD004F58064A04218D07C
:1064D00004F58064A04216D004F58064A04214D074
:1064E00004F58064A0423FF435AF0A2435E7012467
:1064F00033E7022431E703242FE704242DE70524A2
:106500002BE7062429E7072427E7082425E702B01C
:1065100070BD00BF0004005800440258000002583B
:106520000AB181617047090481617047134BDB68D0
:1065300013F0040F07D1114BDB6803F0070383420C
:106540001AD00120704710B50C4AD36823F0070316
:106550001843D060FDF75CFA0446084B5B6813F4FF
:10656000005F07D1FDF754FA001BB0F57A7FF4D92C
:10657000012000E0002010BD0020704700480258B4
:10658000002800F0398338B50446036813F0010F82
:1065900025D0944A136903F03803926A102B15D062
:1065A000182B0FD06368B3F5803F3FD0002B53D139
:1065B0008C4B1A6822F480321A601A6822F4802206
:1065C0001A6038E002F00302022AEBD1854B1B6807
:1065D00013F4003F03D06368002B00F00F8323689F
:1065E00013F0020F00F0A1807E4A1369926A13F043
:1065F00038035AD0182B55D0E368002B00F0DE800A
:1066000078490A6822F0190213430B60FDF700FA7B
:106610000546744B1B6813F0040F40F0AD80FDF786
:10662000F7F9401B0228F4D90320EEE26D4A136803
:1066300043F48033136063682BB3FDF7E9F9054633
:10664000684B1B6813F4003FC9D1FDF7E1F9401B0B
:106650006428F5D90320D8E2B3F5A02F09D0614B07
:106660001A6822F480321A601A6822F480221A60B2
:10667000E1E75C4B1A6842F480221A601A6842F41F
:1066800080321A60D7E7FDF7C3F90546554B1B6802
:1066900013F4003FA3D0FDF7BBF9401B6428F5D9E4
:1066A0000320B2E212F0030FA6D14E4B1B6813F089
:1066B000040F03D0E368002B00F0A282494A13685C
:1066C00023F01903E1680B431360FDF7A1F90546B8
:1066D000444B1B6813F0040F06D1FDF799F9401BDA
:1066E0000228F5D9032090E2FDF798F941F203035F
:1066F000984212D82269402A07D03A494B6823F4BD
:106700007C3343EA02334B600FE0364A536823F48C
:106710007C3343F40033536007E0324A536823F07C
:10672000FE43216943EA01635360236813F0100FAD
:1067300000F088802B4A136903F03803926A082B13
:1067400056D0182B50D0E369002B00F0B880254AB2
:10675000136843F080031360FDF75AF90546214B97
:106760001B6813F4807F40F08880FDF751F9401BCF
:106770000228F4D9032048E2FDF750F941F203035F
:10678000984212D82269402A07D016494B6823F450
:106790007C3343EA02334B60C7E7124A536823F461
:1067A0007C3343F400335360BFE70E4A536823F051
:1067B000FE43216943EA01635360B6E7094A13685F
:1067C00023F001031360FDF723F90546054B1B6811
:1067D00013F0040FA9D0FDF71BF9401B0228F5D9CF
:1067E000032012E20044025802F00302012AAAD157
:1067F000A14B1B6813F4807F03D0E369802B40F02A
:106800000182FDF70BF941F20303984212D8226A84
:10681000202A07D098494B6823F0F84343EA826363
:106820004B600FE0944A536823F0F84343F08043F1
:10683000536007E0904AD36823F07C53216A43EA0F
:106840000163D360236813F0080F60D06369002BE5
:1068500049D0894A536F43F001035367FDF7D8F8D5
:106860000546854B5B6F13F0020F50D1FDF7D0F852
:10687000401B0228F5D90320C7E1FDF7CFF841F20C
:106880000303984212D8226A202A07D07A494B681B
:1068900023F0F84343EA82634B60D3E7764A5368B8
:1068A00023F0F84343F080435360CBE7724AD36848
:1068B00023F07C53216A43EA0163D360C2E76E4A46
:1068C000136823F080031360FDF7A2F805466A4BB6
:1068D0001B6813F4807FB5D0FDF79AF8401B02289F
:1068E000F5D9032091E1644A536F23F00103536704
:1068F000FDF78EF80546604B5B6F13F0020F06D074
:10690000FDF786F8401B0228F5D903207DE12368B6
:1069100013F0200F29D0A3699BB1574A136843F4A1
:1069200080531360FDF774F80546534B1B6813F44E
:10693000005F1AD1FDF76CF8401B0228F5D903203F
:1069400063E14D4A136823F480531360FDF760F848
:106950000546494B1B6813F4005F06D0FDF758F855
:10696000401B0228F5D903204FE1236813F0040FE0
:1069700021D1636A002B00F047813F4A126902F07F
:106980003802182A00F0EE80022B79D03A4A1368B8
:1069900023F080731360FDF73BF80446364B1B6809
:1069A00013F0007F00F0DC80FDF732F8001B0228B6
:1069B000F4D9032029E1314A136843F4807313604A
:1069C000FDF726F805462D4B1B6813F4807F06D192
:1069D000FDF71EF8401B6428F5D9032015E1A368D4
:1069E000012B0AD00BBB244B1A6F22F001021A674D
:1069F0001A6F22F004021A6704E01F4A136F43F073
:106A000001031367A36833B3FDF702F805461A4B79
:106A10001B6F13F0020FACD1FCF7FAFF401B41F2E1
:106A200088339842F3D90320EFE0052B09D0124BAD
:106A30001A6F22F001021A671A6F22F004021A6715
:106A4000E0E70D4B1A6F42F004021A671A6F42F02A
:106A500001021A67D6E7FCF7DBFF0546064B1B6F02
:106A600013F0020F85D0FCF7D3FF401B41F28833AF
:106A70009842F3D90320C8E0004402580048025865
:106A8000694A136823F080731360FCF7C1FF054661
:106A9000654B1B6813F0007F06D0FCF7B9FF401B65
:106AA0000228F5D90320B0E05F4B996A5F4A0A409B
:106AB000A16AE06A41EA00110A439A62226B013A34
:106AC000C2F30802616B0139490289B20A43A16B22
:106AD0000139090401F4FE010A43E16B0139090699
:106AE00001F0FE410A431A63DA6A22F00102DA6217
:106AF000596B4F4A0A40A16C42EAC1025A63DA6AF2
:106B000022F00C02216C0A43DA62DA6A22F00202F5
:106B1000616C0A43DA62DA6A42F48032DA62DA6A73
:106B200042F40032DA62DA6A42F48022DA62DA6A25
:106B300042F00102DA621A6842F080721A60FCF7D1
:106B400067FF0446384B1B6813F0007F06D1FCF743
:106B50005FFF001B0228F5D9032056E0002054E017
:106B6000002052E0304A916A106B012B4ED001F0A8
:106B70000303A26A93424BD1C1F30511E36A994220
:106B800048D1C0F30802236B013B9A4244D1C0F3C1
:106B90004622636B013B9A4240D1C0F30642A36B8D
:106BA000013B9A423CD1C0F30660E36B013B984243
:106BB00038D11D4B5B6BC3F3CC03A26C9A4201D15D
:106BC000002022E0184AD36A23F00103D362FCF7C5
:106BD0001FFF0546FCF71CFFA842FBD0124A516B71
:106BE000134B0B40A16C43EAC1035363D36A43F0D8
:106BF0000103D362002008E001207047012004E077
:106C0000012002E0012000E0002038BD0120FCE767
:106C10000120FAE70120F8E70120F6E70120F4E778
:106C20000120F2E70120F0E7004402580CFCFFFFCE
:106C30000700FFFFF8B57E4B1B6903F03803102BEC
:106C400000F0F280182B10D013B17A4C2046F8BD1A
:106C5000774B1B6813F0200F00F0E880744B186826
:106C6000C0F3C100744CC440F0E7714B9D6A05F05D
:106C700003059C6AC4F30514D86A00F001005B6B3D
:106C8000C3F3CC0303FB00F0F9F772FE0646002CB9
:106C9000DCD0012D76D0022D00F0A4800DB320466B
:106CA000F9F766FE01466548F9F76EFF0446604B4A
:106CB000186BC0F30800F9F75BFE05464FF064510E
:106CC0003046F9F7ADFE01462846F9F7A1FD4FF031
:106CD0007E51F9F79DFD01462046F9F7A1FE0446D5
:106CE00071E0534B1B6813F0200F29D0504F3B68C5
:106CF000C3F3C1035048D840F9F73AFE0546204691
:106D0000F9F736FE01462846F9F73EFF0446386B90
:106D1000C0F30800F9F72CFE05464FF064513046E9
:106D2000F9F77EFE01462846F9F772FD4FF07E51D5
:106D3000F9F76EFD01462046F9F772FE044642E07F
:106D40002046F9F715FE01463D48F9F71DFF0446B8
:106D5000374B186BC0F30800F9F70AFE05464FF0F1
:106D600064513046F9F75CFE01462846F9F750FDBC
:106D70004FF07E51F9F74CFD01462046F9F750FEE1
:106D8000044620E02046F9F7F3FD01462B48F9F7C9
:106D9000FBFE0446264B186BC0F30800F9F7E8FD2C
:106DA00005464FF064513046F9F73AFE0146284651
:106DB000F9F72EFD4FF07E51F9F72AFD01462046E6
:106DC000F9F72EFE04461A4B1B6BC3F34623581CDF
:106DD000F9F7CEFD01462046F9F7D6FEF9F770FF28
:106DE000044633E72046F9F7C3FD01461548F9F795
:106DF000CBFE04460E4B186BC0F30800F9F7B8FD44
:106E000005464FF064513046F9F70AFE0146284620
:106E1000F9F7FEFC4FF07E51F9F7FAFC01462046E7
:106E2000F9F7FEFD0446CEE7074C0FE7024C0DE7ED
:106E30000044025800093D000090D0030024744A29
:106E40000024744C0024F44A00127A00002800F058
:106E5000328170B50D4604469B4B1B6803F00F034F
:106E60008B420BD2984A136823F00F030B43136035
:106E7000136803F00F038B4240F01F81236813F067
:106E8000040F0CD02269914B9B6903F070039A4266
:106E900005D98E498B6923F070031A438A612368F0
:106EA00013F0080F0CD06269884BDB6903F07003A4
:106EB0009A4205D98549CB6923F070031A43CA6108
:106EC000236813F0100F0CD0A269804BDB6903F428
:106ED000E0639A4205D97D49CB6923F4E0631A4304
:106EE000CA61236813F0200F0CD0E269774B1B6A4C
:106EF00003F070039A4205D974490B6A23F07003BA
:106F00001A430A62236813F0020F0CD0E2686F4B39
:106F10009B6903F00F039A4205D96C498B6923F0F2
:106F20000F031A438A61236813F0010F41D0674AA7
:106F3000936923F47063A1680B4393616368022B28
:106F40000AD0032B27D0012B2CD0604A126812F0F4
:106F5000040F06D10120ADE0126812F4003F00F0EA
:106F6000AE805A490A6922F0070213430B61FCF70D
:106F70004FFD0646554B1B6903F038036268B3EBBF
:106F8000C20F16D0FCF744FD801B41F288339842B3
:106F9000F0D903208EE04D4A126812F0007FE0D154
:106FA000012087E0494A126812F4807FD9D101207C
:106FB00080E0236813F0020F0CD0E268434B9B691A
:106FC00003F00F039A4205D240498B6923F00F0367
:106FD0001A438A613C4B1B6803F00F03AB420AD98A
:106FE000394A136823F00F032B431360136803F02F
:106FF0000F03AB4265D1236813F0040F0CD0226954
:10700000324B9B6903F070039A4205D22F498B697A
:1070100023F070031A438A61236813F0080F0CD021
:1070200062692A4BDB6903F070039A4205D2274953
:10703000CB6923F070031A43CA61236813F0100F61
:107040000CD0A269214BDB6903F4E0639A4205D2BC
:107050001E49CB6923F4E0631A43CA61236813F025
:10706000200F0CD0E269194B1B6A03F070039A429F
:1070700005D216490B6A23F070031A430A62FFF720
:10708000D9FD12498B69C3F30323114AD35C03F082
:107090001F03D8408B6903F00F03D35C03F01F0379
:1070A00020FA03F30B4A13600B4B18600B4B186864
:1070B000FCF74CFC70BD012070470120FAE701206D
:1070C000F8E70120F6E700BF002000520044025814
:1070D00084320108200000241C0000242800002421
:1070E00008B5FFF7A7FD0B4A9369C3F303230A49C9
:1070F000CB5C03F01F0320FA03F3926902F00F0246
:10710000885C00F01F0023FA00F0044A1060044A73
:10711000136008BD00440258843201082000002496
:107120001C00002408B5FFF7DBFF054BDB69C3F348
:107130000213044AD35C03F01F03D84008BD00BF0C
:10714000004402588432010808B5FFF7C9FF054B17
:10715000DB69C3F30223044AD35C03F01F03D84066
:1071600008BD00BF0044025884320108404B9B6AAE
:1071700003F00303032B79D070B505460E463C4A55
:10718000136823F080631360FCF742FC0446384B1D
:107190001B6813F0006F06D0FCF73AFC031B022BB0
:1071A000F5D9032070BD324B9A6A22F47C322968EB
:1071B00042EA01329A626A68013AC2F30802A96897
:1071C0000139490289B20A43E9680139090401F425
:1071D000FE010A4329690139090601F0FE410A430B
:1071E0009A63DA6A22F0C00269690A43DA62DA6AEB
:1071F00022F02002A9690A43DA62DA6A22F0100258
:10720000DA62D96B1B4A0A40E96942EAC102DA63D1
:10721000DA6A42F01002DA62C6B91A46DB6A43F44F
:107220000023D362124A136843F080631360FCF7B3
:10723000EFFB04460E4B1B6813F0006F14D1FCF7F4
:10724000E7FB001B0228F5D90320ABE7012E05D090
:10725000074AD36A43F40013D362E3E7044AD36ACC
:1072600043F48013D362DDE700209BE701207047E1
:10727000004402580700FFFF404B9B6A03F00303E2
:10728000032B79D070B505460E463C4A136823F0AF
:1072900080531360FCF7BCFB0446384B1B6813F0AB
:1072A000005F06D0FCF7B4FB031B022BF5D90320CB
:1072B00070BD324B9A6A22F07C72296842EA015210
:1072C0009A626A68013AC2F30802A9680139490260
:1072D00089B20A43E9680139090401F4FE010A434D
:1072E00029690139090601F0FE410A431A64DA6A84
:1072F00022F4406269690A43DA62DA6A22F40072AF
:10730000A9690A43DA62DA6A22F48072DA62596C95
:107310001B4A0A40E96942EAC1025A64DA6A42F445
:107320008072DA62C6B91A46DB6A43F48003D3621C
:10733000124A136843F080531360FCF769FB04465C
:107340000E4B1B6813F0005F14D1FCF761FB001BB0
:107350000228F5D90320ABE7012E05D0074AD36AEE
:1073600043F08073D362E3E7044AD36A43F4000333
:10737000D362DDE700209BE70120704700440258FC
:107380000700FFFFF8B50446036813F0006F30D024
:10739000836EB3F5001F26D00ED8EBB1B3F5801F76
:1073A00007D102210830FFF7E1FE054645B12E4620
:1073B00021E0012635461EE0B3F5401F09D1002526
:1073C000984A136D23F44013A16E0B4313650026F6
:1073D00011E0012635460EE0924AD36A43F40033A9
:1073E000D3620025ECE702212830FFF745FF054670
:1073F000DCE700263546236813F4807F14D0A36DA4
:10740000042B32D8DFE803F003232A080800854A5A
:10741000D36A43F40033D36255BB824A136D23F021
:107420000703A16D0B431365236813F4007F31D06C
:10743000E36D802B4CD020D8002B43D0402B19D1AA
:10744000002104F10800FFF791FE05461AE0002133
:1074500004F10800FFF78AFE0546DDE7002104F18C
:107460002800FFF709FF0546D6E701263546DBE78A
:107470002E46D9E7012635460CE0C02B02D0B3F5E5
:10748000807F1CD15DBB674A136D23F4E073E16D0F
:107490000B431365236813F4806F46D0D4F8A830EB
:1074A000B3F5800F39D01FD88BB3B3F5001F18D1B7
:1074B000002104F10800FFF759FE05461AE00126F5
:1074C0003546E7E7574AD36A43F40033D362D9E736
:1074D000002104F12800FFF7CFFE0546D2E72E4633
:1074E000D8E70126354620E0B3F5C00F02D0B3F54A
:1074F000000F09D1C5B94B4A936D23F46003D4F84A
:10750000A8100B43936510E0012635460DE0454A6F
:10751000D36A43F40033D362ECE7002104F128007E
:10752000FFF7AAFE0546E5E72E46236813F4006F31
:1075300024D0D4F8AC30B3F1007F42D00ED8002B69
:1075400039D0B3F1807F06D1002104F10800FFF7A4
:107550000DFE054608E0012635460FE0B3F1407FF9
:1075600002D0B3F1806F23D1002D31D12D4A936D1C
:1075700023F0E063D4F8AC100B439365236813F059
:10758000007F2ED0E36C202B40D026D833B1102BB7
:1075900020D1244AD36A43F40033D362002D3CD176
:1075A000204AD36C23F03003E16C0B43D36418E022
:1075B00001263546E2E71B4AD36A43F40033D3621F
:1075C000D2E7002104F12800FFF756FE0546CBE77D
:1075D0002E46D3E70126354603E0302BDED00126C8
:1075E0003546236813F4805F2DD0236EB3F5005F1A
:1075F0004FD019D8002B46D0B3F5805F0FD10021B2
:1076000004F10800FFF7B2FD054613E0022104F182
:107610000800FFF7ABFD0546C0E72E46E1E701266F
:10762000354610E000440258B3F5405F02D0B3F590
:10763000804F25D1002D33D1774A136D23F4E043D9
:10764000216E0B431365236813F4005F38D0636E1B
:10765000B3F5003F53D028D843B1B3F5803F21D1D3
:10766000012104F10800FFF781FD0546002D4DD1F1
:10767000694A136D23F4E023616E0B4313651FE029
:1076800001263546DFE7644AD36A43F40033D36208
:10769000D0E7002104F12800FFF7EEFD0546C9E719
:1076A0002E46D0E7012635460AE0B3F5802FDDD01F
:1076B000B3F5A02FDAD0B3F5403FD7D00126354639
:1076C000236813F4804F31D0D4F8B030B3F1005FA9
:1076D00045D020D843B1B3F1805F19D1012104F125
:1076E0000800FFF743FD0546002D3FD14A4A936D40
:1076F00023F0E043D4F8B0100B43936516E001216A
:1077000004F12800FFF7B8FD0546AFE72E46D7E79E
:10771000012635460AE0B3F1804FE5D0B3F1A04F22
:10772000E2D0B3F1405FDFD001263546236813F481
:10773000004F09D0236FB3F1805F19D0B3F1005F20
:1077400024D0D3B101263546236813F0807F33D08F
:10775000A36C032B5BD8DFE803F02722532701211A
:1077600004F12800FFF788FD0546BDE72E46DDE75A
:10777000294AD36A43F40033D36275B9264A136D9C
:1077800023F04053216F0B431365DDE7012104F122
:107790000800FFF7EBFC0546EFE72E46D4E71E4A4C
:1077A000D36A43F40033D362A5BB1B4AD36C23F0E6
:1077B0000303A16C0B43D364236813F4800F2DD112
:1077C000236813F0010F00F0A580E36F282B00F26F
:1077D0009F80DFE803F08D9D9D9D9D9D9D9D879DD4
:1077E0009D9D9D9D9D9D969D9D9D9D9D9D9D8D9DE0
:1077F0009D9D9D9D9D9D8D9D9D9D9D9D9D9D8D0076
:10780000022104F10800FFF7B1FC0546CCE7012690
:107810003546D1E72E46CFE700440258914A136817
:1078200043F480731360FCF7F3F807468D4B1B6835
:1078300013F4807F05D1FCF7EBF8C01B6428F5D961
:107840000325002D4AD1884B1B6FD4F8B420534038
:1078500013F4407F0CD0844B1A6F22F44072196FDE
:1078600041F480311967196F21F4803119671A6763
:10787000D4F8B430B3F5807F15D08DBBD4F8B430D4
:1078800003F44072B2F5407F1ED0774A136923F4A7
:107890007C53136174490B6FD4F8B420C2F30B020C
:1078A00013430B678CE7FCF7B3F807466E4B1B6F6F
:1078B00013F0020FE1D1FCF7ABF8C01B41F28833A3
:1078C0009842F3D90325D8E76748026922F47C522D
:1078D000664901EA131313430361DBE72E466FE7A2
:1078E0002E466DE7012104F10800FFF73FFC054635
:1078F000E5B95D4A536D23F03803E16F0B435365DF
:1079000008E0012104F12800FFF7B6FC0546EFE787
:1079100001263546236813F0020F17D0A36F052BFD
:1079200028D8DFE803F00B05200B0B0B2E46F1E700
:10793000012104F10800FFF719FC0546EDB94A4A98
:10794000536D23F00703A16F0B435365236813F0B6
:10795000040F23D0D4F89430052B45D8DFE803F08A
:10796000150F3D151515012104F12800FFF784FCC2
:107970000546E3E701263546E8E72E46E6E701211E
:1079800004F10800FFF7F2FB054685BB364A936D0C
:1079900023F00703D4F894100B439365236813F086
:1079A000200F34D0D4F89030B3F1005F4ED023D8FC
:1079B00043B1B3F1805F1CD1002104F10800FFF74F
:1079C000D5FB0546002D48D1274A536D23F0E043EF
:1079D000D4F890100B43536519E0012104F12800FD
:1079E000FFF74AFC0546D0E701263546D6E72E4686
:1079F000D4E7012635460AE0B3F1804FE2D0B3F177
:107A0000A04FDFD0B3F1405FDCD0012635462368BC
:107A100013F0400F37D0D4F89C30B3F5006F53D03B
:107A200026D843B1B3F5806F19D1002104F10800C5
:107A3000FFF79CFB0546002D4DD10B4A936D23F4B7
:107A4000E053D4F89C100B4393651CE0022104F131
:107A50002800FFF711FC0546B4E72E46D7E70126BC
:107A6000354610E00048025800440258CFFFFF009E
:107A7000B3F5805FDFD0B3F5A05FDCD0B3F5406F26
:107A8000D9D001263546236813F0800F33D0D4F8BF
:107A9000A030B3F5804F00F0A38021D843B1B3F5F7
:107AA000005F1AD1002104F10800FFF75FFB0546D3
:107AB000002D40F09C80814A936D23F46043D4F8FC
:107AC000A0100B43936516E0022104F12800FFF794
:107AD000D3FB0546AFE72E46D5E7012635460AE03B
:107AE000B3F5004FE4D0B3F5204FE1D0B3F5C04F6C
:107AF000DED001263546236813F0080F0CD0D4F8E9
:107B00008430B3F5805F74D06C4A536D23F44053D6
:107B1000D4F884100B435365236813F0100F0CD076
:107B2000D4F89830B3F5807F6CD0644A936D23F419
:107B30004073D4F898100B439365236813F4002F17
:107B40000BD0D4F8A430B3F5803F74D0B3F5003F28
:107B500067D0002B5FD001263546236813F4802FB1
:107B60000CD0D4F88830B3F5001F7CD0B3F5401F9B
:107B70006FD0B3F5801F67D001263546236813F414
:107B8000803F08D0236D002B76D0B3F5803F00F006
:107B9000818001263546236813F0005F40F0838022
:107BA000236813F4003F00F08E80D4F88030B3F5E2
:107BB000807F00F0EC8040F28380B3F5007F03D03B
:107BC000B3F5407F40F0E180002D40F0E6803B4A75
:107BD000536D23F44073D4F880100B43536572E067
:107BE000022104F12800FFF747FB054660E72E4617
:107BF00081E7022104F12800FFF73EFB002883D033
:107C0000012681E7022104F12800FFF735FB002857
:107C10008BD0012689E7002104F10800FFF7A6FABE
:107C200005467DB9254A936D23F44033D4F8A4105A
:107C30000B43936591E7022104F12800FFF71CFB39
:107C40000546EEE72E4688E71C4AD36A43F4003324
:107C5000D3627DB9194A536D23F44013D4F88810C8
:107C60000B4353658AE7012104F12800FFF704FB69
:107C70000546EEE72E4681E7104AD36A43F4003307
:107C8000D36275B90D4AD36C23F48033216D0B4355
:107C9000D36480E7022104F10800FFF767FA054684
:107CA000EFE72E4677E7022104F12800FFF7E4FA18
:107CB00000283FF475AF012672E700BF0044025868
:107CC000002B81D00126236813F4801F06D04F4A71
:107CD000136D23F00043616F0B431365236813F0AA
:107CE000805F07D0494A136923F48043D4F8B81061
:107CF0000B431361236813F4001F06D0434A136D2E
:107D000023F08073E16E0B431365236813F0804FFB
:107D100009D03E4B1A6922F400421A611A69D4F85C
:107D2000BC100A431A612368002B06DA374AD36C69
:107D300023F04053616D0B43D364236813F4000FA9
:107D400007D0324A536D23F44003D4F88C100B4310
:107D50005365636813F0010F21D1636813F0020FBC
:107D600026D1636813F0040F2BD1636813F0080F5A
:107D700030D1636813F0100F35D1636813F0200F12
:107D80003AD106B101263046F8BD01269BE71F4ACD
:107D9000D36A43F40033D36216E72E4693E70021FB
:107DA00004F10800FFF7E2F90028D6D00646D4E730
:107DB000012104F10800FFF7D9F90028D1D00646C7
:107DC000CFE7022104F10800FFF7D0F90028CCD05A
:107DD0000646CAE7002104F12800FFF74DFA002803
:107DE000C7D00646C5E7012104F12800FFF744FA91
:107DF0000028C2D00646C0E7022104F12800FFF7A0
:107E00003BFA0028BDD00646BBE700BF004402583D
:107E100008B5FFF765F9054B1B6AC3F30213044A63
:107E2000D35C03F01F03D84008BD00BF00440258D4
:107E3000843201082DE9F0410446864B9D6A9E6A12
:107E4000C6F30536D86AC0F30010DB6BC3F3CC036E
:107E500003FB00F0F8F78CFD002E00F0F58005F034
:107E600003050746012D79D0022D00F0CB800DB31C
:107E70003046F8F77DFD01467748F8F785FE054660
:107E8000744B986BC0F30800F8F772FD06464FF08C
:107E900064513846F8F7C4FD01463046F8F7B8FC9F
:107EA0004FF07E51F8F7B4FC01462846F8F7B8FDCC
:107EB000054674E0674B1B6813F0200F2CD0DFF8E9
:107EC0009481D8F80030C3F3C1036448D840F8F770
:107ED0004FFD05463046F8F74BFD01462846F8F7BA
:107EE00053FE0546D8F83800C0F30800F8F740FD07
:107EF00006464FF064513846F8F792FD0146304689
:107F0000F8F786FC4FF07E51F8F782FC01462846D0
:107F1000F8F786FD054642E03046F8F729FD0146B0
:107F20004F48F8F731FE05464A4B986BC0F30800FE
:107F3000F8F71EFD06464FF064513846F8F770FD1D
:107F400001463046F8F764FC4FF07E51F8F760FCCC
:107F500001462846F8F764FD054620E03046F8F76C
:107F600007FD01463C48F8F70FFE0546394B986B74
:107F7000C0F30800F8F7FCFC06464FF064513846A1
:107F8000F8F74EFD01463046F8F742FC4FF07E51BF
:107F9000F8F73EFC01462846F8F742FD05462D4E0F
:107FA000B06BC0F34620F8F7E3FC4FF07E51F8F7D2
:107FB0002FFC01462846F8F7E7FDF8F781FE206020
:107FC000B06BC0F30640F8F7D3FC4FF07E51F8F7E2
:107FD0001FFC01462846F8F7D7FDF8F771FE6060F0
:107FE000B06BC0F30660F8F7C3FC4FF07E51F8F7B2
:107FF0000FFC01462846F8F7C7FDF8F761FEA060C0
:10800000BDE8F0813046F8F7B3FC01461548F8F7B3
:10801000BBFD05460F4B986BC0F30800F8F7A8FCB2
:1080200006464FF064513846F8F7FAFC01463046F0
:10803000F8F7EEFB4FF07E51F8F7EAFB01462846D1
:10804000F8F7EEFC0546AAE7002323606360A3600F
:10805000D6E700BF004402580024744A0090D003C1
:108060000024744C0024F44A2DE9F0410446864B68
:108070009D6A9E6AC6F30556D86AC0F300205B6C01
:10808000C3F3CC0303FB00F0F8F772FC002E00F002
:10809000F58005F003050746012D79D0022D00F08B
:1080A000CB800DB33046F8F763FC01467748F8F70C
:1080B0006BFD0546744B186CC0F30800F8F758FCCC
:1080C00006464FF064513846F8F7AAFC01463046A0
:1080D000F8F79EFB4FF07E51F8F79AFB01462846D1
:1080E000F8F79EFC054674E0674B1B6813F0200F01
:1080F0002CD0DFF89481D8F80030C3F3C103644872
:10810000D840F8F735FC05463046F8F731FC014613
:108110002846F8F739FD0546D8F84000C0F30800B6
:10812000F8F726FC06464FF064513846F8F778FC1D
:1081300001463046F8F76CFB4FF07E51F8F768FBCC
:1081400001462846F8F76CFC054642E03046F8F751
:108150000FFC01464F48F8F717FD05464A4B186CCF
:10816000C0F30800F8F704FC06464FF064513846A7
:10817000F8F756FC01463046F8F74AFB4FF07E51BF
:10818000F8F746FB01462846F8F74AFC054620E08A
:108190003046F8F7EDFB01463C48F8F7F5FC05469C
:1081A000394B186CC0F30800F8F7E2FB06464FF0B5
:1081B00064513846F8F734FC01463046F8F728FB9E
:1081C0004FF07E51F8F724FB01462846F8F728FCCB
:1081D00005462D4E306CC0F34620F8F7C9FB4FF032
:1081E0007E51F8F715FB01462846F8F7CDFCF8F765
:1081F00067FD2060306CC0F30640F8F7B9FB4FF024
:108200007E51F8F705FB01462846F8F7BDFCF8F764
:1082100057FD6060306CC0F30660F8F7A9FB4FF0C3
:108220007E51F8F7F5FA01462846F8F7ADFCF8F765
:1082300047FDA060BDE8F0813046F8F799FB0146A4
:108240001548F8F7A1FC05460F4B186CC0F3080061
:10825000F8F78EFB06464FF064513846F8F7E0FB1E
:1082600001463046F8F7D4FA4FF07E51F8F7D0FACD
:1082700001462846F8F7D4FB0546AAE70023236009
:108280006360A360D6E700BF004402580024744A2C
:108290000090D0030024744C0024F44A2DE9F041EE
:1082A0000446864B9D6A9E6AC6F30516D86A00F09E
:1082B00001005B6BC3F3CC0303FB00F0F8F758FB42
:1082C000002E00F0F58005F003050746012D79D05A
:1082D000022D00F0CB800DB33046F8F749FB014684
:1082E0007748F8F751FC0546744B186BC0F308004B
:1082F000F8F73EFB06464FF064513846F8F790FB1E
:1083000001463046F8F784FA4FF07E51F8F780FACC
:1083100001462846F8F784FB054674E0674B1B6866
:1083200013F0200F2CD0DFF89481D8F80030C3F37D
:10833000C1036448D840F8F71BFB05463046F8F700
:1083400017FB01462846F8F71FFC0546D8F8300011
:10835000C0F30800F8F70CFB06464FF064513846AE
:10836000F8F75EFB01463046F8F752FA4FF07E51BF
:10837000F8F74EFA01462846F8F752FB054642E068
:108380003046F8F7F5FA01464D48F8F7FDFB05468B
:108390004A4B186BC0F30800F8F7EAFA06464FF0AC
:1083A00064513846F8F73CFB01463046F8F730FA9E
:1083B0004FF07E51F8F72CFA01462846F8F730FBCB
:1083C000054620E03046F8F7D3FA01463E48F8F774
:1083D000DBFB0546394B186BC0F30800F8F7C8FA09
:1083E00006464FF064513846F8F71AFB014630460E
:1083F000F8F70EFA4FF07E51F8F70AFA01462846D0
:10840000F8F70EFB05462D4E306BC0F34620F8F70B
:10841000AFFA4FF07E51F8F7FBF901462846F8F71E
:10842000B3FBF8F74DFC2060306BC0F30640F8F763
:108430009FFA4FF07E51F8F7EBF901462846F8F71E
:10844000A3FBF8F73DFC6060306BC0F30660F8F703
:108450008FFA4FF07E51F8F7DBF901462846F8F71E
:1084600093FBF8F72DFCA060BDE8F0813046F8F7EB
:108470007FFA01461548F8F787FB05460F4B186B46
:10848000C0F30800F8F774FA06464FF06451384616
:10849000F8F7C6FA01463046F8F7BAF94FF07E51C0
:1084A000F8F7B6F901462846F8F7BAFA0546AAE7FA
:1084B000002323606360A360D6E700BF0044025836
:1084C0000024744C0090D0030024744A0024F44A21
:1084D00000B58BB0A0F580730B432ED0A0F50073D0
:1084E0000B437ED0A0F580630B4300F0D480A0F551
:1084F00000630B4300F02C81A0F580530B4300F088
:108500008B81A0F500530B4300F0E381A0F500231D
:108510000B4300F02C82A0F580330B4300F06F82F8
:10852000A0F580430B4300F09082A0F5004050EA94
:10853000010300F0D382002001E3954B1B6D03F093
:108540000703042B00F2F282DFE803F005101B039F
:1085500026009048F3E28E4B186810F0007000F08F
:10856000EE8207A8FFF79AFE0898E8E2884B1868A1
:1085700010F0006000F0E38204A8FFF75BFC0498B1
:10858000DDE2834B186810F0005000F0D88201A89B
:10859000FFF76AFD0198D2E27D4AD36C03F04053A5
:1085A000126812F0040F07D033B9794B1B68C3F37C
:1085B000C1037948D840C2E2754A126812F4807F3C
:1085C00003D0B3F1805F00F0B382714A126812F4F5
:1085D000003F00F0AF82B3F1005F00F0AD820020F9
:1085E000ADE26B4B1B6D03F4E073802B33D015D9D8
:1085F000C02B00F0A382B3F5807F1FD1644AD36CF7
:1086000003F04053126812F0040F2FD073BB604B7D
:108610001B68C3F3C1036048D84090E283B1402B8C
:108620000AD15B4B186810F0006000F0888204A843
:10863000FFF700FC049882E2002080E200207EE246
:10864000534B186810F0007000F0798207A8FFF70C
:1086500025FE089873E24E4B186810F0005000F0A9
:108660006E8201A8FFF700FD019868E2484A12688F
:1086700012F4807F03D0B3F1805F00F06382444A3C
:10868000126812F4003F00F05F82B3F1005F00F067
:108690005D82002053E23E4B9B6D03F46003B3F513
:1086A000800F35D016D9B3F5C00F00F05182B3F565
:1086B000000F20D1364AD36C03F04053126812F0F9
:1086C000040F30D07BBB324B1B68C3F3C10332486D
:1086D000D84034E28BB1B3F5001F0AD12C4B186897
:1086E00010F0006000F02B8204A8FFF7A3FB0498B1
:1086F00025E2002023E2002021E2254B186810F03B
:10870000007000F01C8207A8FFF7C8FD089816E269
:108710001F4B186810F0005000F0118201A8FFF7FD
:10872000A3FC01980BE21A4A126812F4807F03D06E
:10873000B3F1805F00F00E82154A126812F4003F18
:1087400000F00A82B3F1005F00F008820020F6E139
:108750000F4B9B6D03F0E063B3F1007F3CD01DD95C
:10876000B3F1407F00F0FC81B3F1806F27D1084A5C
:10877000D36C03F04053126812F0040F37D0002B73
:1087800035D1034B1B68C3F3C1030348D840D6E17E
:10879000004402580080BB000090D0038BB1B3F1BD
:1087A000807F0AD19A4B186810F0006000F0C781F2
:1087B00004A8FFF73FFB0498C1E10020BFE10020BF
:1087C000BDE1934B186810F0007000F0B88107A865
:1087D000FFF764FD0898B2E18D4B186810F0005067
:1087E00000F0AD8101A8FFF73FFC0198A7E1884A9E
:1087F000126812F4807F03D0B3F1805F00F0B28181
:10880000834A126812F4003F00F0AE81B3F1005FBA
:1088100000F0AC81002092E17D4B1B6D03F4E0433E
:10882000B3F5005F35D016D9B3F5405F00F0A081F5
:10883000B3F5804F20D1764AD36C03F040531268D1
:1088400012F0040F30D07BBB714B1B68C3F3C10324
:108850007048D84073E18BB1B3F5805F0AD16C4B9F
:10886000186810F0006000F06A8104A8FFF7E2FACF
:10887000049864E1002062E1002060E1644B186824
:1088800010F0007000F05B8107A8FFF707FD089863
:1088900055E15F4B186810F0005000F0508101A8BE
:1088A000FFF7E2FB01984AE1594A126812F4807F0F
:1088B00003D0B3F1805F00F05D81554A126812F475
:1088C000003F00F05981B3F1005F00F057810020B4
:1088D00035E14F4B1B6D03F4E023B3F5403F32D03D
:1088E00016D8B3F5803F23D0B3F5003F0AD1484BEB
:1088F000186810F0005000F0228101A8FFF7B4FBC7
:1089000002981CE113B9FEF70DFC18E1002016E1F6
:10891000B3F5802F23D0B3F5A02F07D13C4B1868B7
:1089200010F4003000F00B813B4808E1002006E124
:10893000374B186810F0006000F0018104A8FFF7C1
:1089400079FA0598FBE0324B186810F0040000F04B
:10895000F6801B68C3F3C1032E48D840EFE02C4BD0
:10896000186810F4807000F0EA802C48E7E0284B8B
:108970009B6D03F44033B3F5803F10D0B3F5003F57
:1089800018D00BB10020DAE0214B186810F000601D
:1089900000F0D58004A8FFF74DFA0498CFE01C4BF7
:1089A000186810F0005000F0CA8001A8FFF75CFBC7
:1089B0000398C4E0164AD36C03F04053126812F0D7
:1089C000040F07D033B9124B1B68C3F3C10311481E
:1089D000D840B4E00E4A126812F4807F03D0B3F19D
:1089E000805F00F0CD800A4A126812F4003F00F068
:1089F000C980B3F1005F00F0C78000209FE0044B06
:108A0000DB6C13F480330BD0ABB9002097E000BFD0
:108A1000004402580090D00300127A0000093D0083
:108A20005A4B186810F0007000F0898007A8FFF713
:108A300035FC089883E0554B186810F000607ED034
:108A400004A8FFF7F7F9069879E0504B9B6D03F007
:108A5000E043B3F1405F2FD015D8B3F1805F21D050
:108A6000B3F1005F09D1494B186810F0005066D08F
:108A700001A8FFF7F9FA029861E013B9FFF7C8F906
:108A80005DE000205BE0B3F1804F20D0B3F1A04F58
:108A900006D13E4B186810F4003050D03C484EE0F0
:108AA00000204CE0394B186810F0006047D004A853
:108AB000FFF7C0F9059842E0344B186810F0040045
:108AC0003DD01B68C3F3C1033248D84037E02F4B79
:108AD000186810F4807032D02F4830E02B4B1B6D9B
:108AE00003F04053B3F1805F0CD0B3F1005F13D0BB
:108AF0000BB1002023E0254B186810F400301ED085
:108B000023481CE0214B186810F0007017D007A80C
:108B1000FFF7C4FB089812E01C4B186810F00060C7
:108B20000DD004A8FFF786F9059808E0002006E0BC
:108B3000194804E0002002E0154800E017480BB097
:108B40005DF804FB1448FAE70020F8E71048F6E760
:108B50001248F4E71048F2E70020F0E70C48EEE78F
:108B60000E48ECE70C48EAE70020E8E70848E6E7AB
:108B70000A48E4E70848E2E70020E0E70448DEE7C7
:108B80000548DCE70020DAE70148D8E7004402584E
:108B900000127A000090D00300093D000080BB0065
:108BA000F0B4036A23F001030362036A4668846930
:108BB0001F4A22400D68154323F002038C682343AB
:108BC0001C4A1D4CA04218BF90420CBF012200223B
:108BD0000CD004F58044A04214BF00240124174F98
:108BE000B84203D014B9164CA04205D123F00803B3
:108BF000CC68234323F004035AB9124A904214BFAD
:108C0000002201220D4CA04203D012B90C4A90421E
:108C100007D126F4407C4A6942EA0C0C8E6946EA88
:108C20000C06466085614A6842630362F0BC704787
:108C30008CFFFEFF000001400004014000400140A5
:108C4000004801400044014070B4036A23F480737B
:108C50000362036A4568C4691A4A22400E681643D3
:108C600023F400738A6843EA0223174A174CA04290
:108C700018BF90420CBF0122002206D123F40063EA
:108C8000CC6843EA042323F480635AB9104A904223
:108C900014BF002201220F4CA04203D012B90E4A89
:108CA000904207D125F4405C4A694CEA021C8D6968
:108CB0004CEA05154560C6614A68C263036270BC30
:108CC000704700BF8CFFFEFF000001400004014020
:108CD00000440140004001400048014070B4036A74
:108CE00023F480530362036A4468C569144A2A4026
:108CF0000D6842EA052223F400538D6843EA0533E8
:108D0000104E114DA84218BFB0420DD005F5804558
:108D1000A84214BF0025012506F58046B04203D0C5
:108D200015B90A4DA84204D124F480444D6944EA9F
:108D300085144460C2614A680264036270BC704773
:108D4000FF8CFFFE0000014000040140004801408C
:108D500070B4036A23F480330362036A4268456D8A
:108D6000144C2C400D682C4323F400338D6843EAE7
:108D70000543114E114DA84218BFB0420DD005F564
:108D80008045A84214BF0025012506F58046B04263
:108D900003D015B90A4DA84204D122F480324D699E
:108DA00042EA0522426044654A688265036270BCFB
:108DB000704700BF8FFFFEFF00000140000401402C
:108DC0000048014070B4036A23F480130362036A0D
:108DD0004468456D144A2A400D6842EA052223F48E
:108DE00000138D6843EA0553104E114DA84218BF79
:108DF000B0420DD005F58045A84214BF00250125DD
:108E000006F58046B04203D015B90A4DA84204D1F8
:108E100024F480244D6944EA8524446042654A680C
:108E2000C265036270BC7047FF8FFFFE0000014007
:108E3000000401400048014010B4036A046A24F0B1
:108E400001040462846924F0F00C4CEA021223F05D
:108E50000A030B438261036210BC704730B4046A9A
:108E600024F0100404628469056A24F4407C4CEA0E
:108E7000022C2CF4704C1B039BB243EA0C0325F02C
:108E8000A005090101F0A00129438361016230BC02
:108E9000704710B4046A24F0100404628469036A01
:108EA00024F4704C4CEA023223F0A00343EA01138D
:108EB0008261036210BC704730B4046A24F4807489
:108EC0000462C469056A24F0030C4CEA020C2CF01D
:108ED000F00C1B01DBB243EA0C0325F42065090208
:108EE00001F420612943C361016230BC704730B492
:108EF000046A24F480540462C469056A24F4407C42
:108F00004CEA022C2CF4704C1B039BB243EA0C037A
:108F100025F42045090301F420412943C36101627E
:108F200030BC70477047704770477047704710B546
:108F3000044603681A6912F0020F11D0DA6812F0C1
:108F4000020F0DD06FF002021A610123037703684C
:108F50009B6913F0030F79D0FAF736FB00232377D0
:108F600023681A6912F0040F12D0DA6812F0040FA5
:108F70000ED06FF004021A610223237723689B69E5
:108F800013F4407F68D02046FAF71EFB00232377B6
:108F900023681A6912F0080F12D0DA6812F0080F6D
:108FA0000ED06FF008021A61042323772368DB696F
:108FB00013F0030F57D02046FAF706FB0023237760
:108FC00023681A6912F0100F12D0DA6812F0100F2D
:108FD0000ED06FF010021A61082323772368DB6933
:108FE00013F4407F46D02046FAF7EEFA00232377A9
:108FF00023681A6912F0010F03D0DA6812F0010F2A
:109000003FD123681A6912F0800F03D0DA6812F09A
:10901000800F3DD123681A6912F4807F03D0DA688B
:1090200012F0800F3BD123681A6912F0400F03D071
:10903000DA6812F0400F39D123681A6912F0200F54
:1090400003D0DA6812F0200F37D110BDFFF76CFFA4
:109050002046FFF76AFF81E72046FFF765FF2046BD
:10906000FFF763FF92E72046FFF75EFF2046FFF71A
:109070005CFFA3E72046FFF757FF2046FFF755FFA9
:10908000B4E76FF001021A612046FFF74CFFB8E722
:109090006FF080021A61204600F085FDBAE76FF498
:1090A00080721A61204600F07FFDBCE76FF040023D
:1090B0001A612046FFF73AFFBEE76FF020021A61FF
:1090C000204600F06FFDC0E730B50368394A904292
:1090D00014BF4FF0000E4FF0010EB0F1804F14BFDF
:1090E00072464EF00102AAB9334CA04214BF0024CC
:1090F0000124324DA8420DD064B904F1804404F536
:109100008234A04214BF0024012405F50065A84262
:1091100000D01CB123F070034C68234312BB264AD5
:10912000904214BF00220122244CA0421AD0CAB996
:1091300002F1804202F58232904214BF00220122E5
:1091400004F50064A0420DD062B91D4A904214BFDC
:109150000022012204F59A34A04203D012B9194A20
:10916000904204D123F4407CCB6843EA0C0323F003
:1091700080034A69134303608A68C2620A68826294
:10918000114A904214BF73464EF0010363B90C4B71
:10919000984214BF0023012302F57052904203D07D
:1091A00013B9084B984201D10B6903630123436152
:1091B00030BD00BF00000140000800400004004036
:1091C00000440140004801400004014060B310B574
:1091D000044690F83D3013B3022384F83D30214615
:1091E00051F8040BFFF770FF012384F8483084F82E
:1091F0003E3084F83F3084F8403084F8413084F8C1
:10920000423084F8433084F8443084F8453084F8A0
:10921000463084F8473084F83D30002010BD80F897
:109220003C30FAF79FF8D7E70120704760B310B5DC
:10923000044690F83D3013B3022384F83D302146B4
:1092400051F8040BFFF740FF012384F8483084F8FD
:109250003E3084F83F3084F8403084F8413084F860
:10926000423084F8433084F8443084F8453084F840
:10927000463084F8473084F83D30002010BD80F837
:109280003C30FAF71FF9D7E70120704760B310B5FB
:10929000044690F83D3013B3022384F83D30214654
:1092A00051F8040BFFF710FF012384F8483084F8CD
:1092B0003E3084F83F3084F8403084F8413084F800
:1092C000423084F8433084F8443084F8453084F8E0
:1092D000463084F8473084F83D30002010BD80F8D7
:1092E0003C30FFF71FFED7E70120704770B4036AD8
:1092F00023F010030362036A456884691A4A224016
:109300000E6842EA062623F020038A6843EA021325
:10931000164A174CA04218BF90420CBF01220022EF
:1093200006D123F08003CC6843EA041323F0400302
:109330005AB9104A904214BF002201220E4CA0429A
:1093400003D012B90D4A904207D125F4406C4A6906
:109350004CEA820C8D694CEA8505456086614A6855
:109360008263036270BC7047FF8CFFFE0000014007
:109370000004014000440140004001400048014019
:1093800038B590F83C30012B00F0958004460D462E
:10939000012380F83C30142A00F28880DFE802F0D4
:1093A0000B8686861F8686863486868648868686CF
:1093B0005D86868671000068FFF7F2FB226893697C
:1093C00043F0080393612268936923F004039361D7
:1093D0002268936929690B439361002067E0006864
:1093E000FFF784FF2268936943F400639361226866
:1093F000936923F48063936122689369296943EA3E
:1094000001239361002052E00068FFF71DFC2268F1
:10941000D36943F00803D3612268D36923F00403BE
:10942000D3612268D36929690B43D36100203EE0F0
:109430000068FFF753FC2268D36943F40063D361EB
:109440002268D36923F48063D3612268D3692969D0
:1094500043EA0123D361002029E00068FFF778FC8C
:109460002268536D43F0080353652268536D23F05F
:10947000040353652268536D29690B43536500202B
:1094800015E00068FFF79EFC2268536D43F400630B
:1094900053652268536D23F4806353652268536DCE
:1094A000296943EA01235365002000E001200023DD
:1094B00084F83C3038BD0220FCE7000070B49446CC
:1094C000046A24F0010404628469066A1D4DB0F147
:1094D000804F18BFA84223D01B4A904214BF0022DD
:1094E0000122A5F57C45A8421AD0CAB902F18042F2
:1094F00002F58232904214BF0022012205F5006578
:10950000A8420DD062B9114A904214BF0022012234
:1095100005F54065A84203D012B944F0010203E00A
:1095200024F0030242EA0C0222F0F0021B01DBB23B
:10953000134326F00A0201F00A011143836101621C
:1095400070BC70470000014000080040004001402E
:1095500038B590F83C30012B5AD004460D46012313
:1095600080F83C3052B1042A1AD0082A2BD00C2A99
:109570003BD00120002384F83C3038BDCB684A68DA
:1095800009680068FFF79AFF2268936923F00C03CB
:10959000936122689369A9680B4393610020E9E70E
:1095A000CB684A6809680068FFF758FC226893692D
:1095B00023F44063936122689369A96843EA012315
:1095C00093610020D6E7CB684A6809680068FFF716
:1095D00073FC2268D36923F00C03D3612268D3693A
:1095E000A9680B43D3610020C4E7CB684A680968C7
:1095F0000068FFF77CFC2268D36923F44063D361E1
:109600002268D369A96843EA0123D3610020B1E746
:109610000220B2E710B4846824F47F4C42EA0322AB
:109620000A4342EA0C02826010BC704710B504681D
:10963000A3684C4A1A404B6813434B4A1A400B68C4
:109640001343A3604B68602B68D01CD8402B50D0CC
:1096500008D9502B15D10A6989680068FFF7ECFB1F
:10966000002035E0202B60D003D9302B07D001201B
:109670002EE0002B5BD0102B5BD1002028E00020D7
:1096800026E0012024E0702B2BD001D201201FE026
:10969000364A93424FD008D9B3F5001F57D018D996
:1096A000334A934259D1002012E0303A934244D0D9
:1096B00007D9304A934246D01032934245D1002018
:1096C00006E0B3F5801F3AD0B3F1101F39D1002066
:1096D00010BD294A93423CD0103293423BD1002026
:1096E000F6E70B698A68C9680068FFF793FF0020F6
:1096F000EEE70B68052B32D003681C6A1A6A22F069
:1097000001021A620268936923F0F003096943EACF
:109710000113936103681C620020D9E70A69896814
:109720000068FFF7B6FB0020D2E70020D0E700205A
:10973000CEE70120CCE70020CAE70020C8E70020E0
:10974000C6E70120C4E70020C2E70120C0E70020EF
:10975000BEE70020BCE70120BAE70120B8E70120FE
:10976000B6E700BF8FFFCFFFF8FFFEFF50001000ED
:1097700010002000300010006000100090F83C3015
:10978000012B22D010B50446012380F83C3002237F
:1097900080F83D30FFF74AFF80B92268D36823F094
:1097A0004003D3602268D36823F48043D36001234D
:1097B00084F83D30002384F83C3010BD012084F84B
:1097C0003D00002384F83C30F7E70220704701F0A9
:1097D0001F01012303FA01FC036A23EA0C0303625D
:1097E000036A02FA01F10B430362704710B50446A5
:1097F000084600294ED194F83E30DBB2013B18BF39
:109800000123002B40F09B8000286ED1022384F8B6
:109810003E30012201462068FFF7D9FF23684A49FC
:109820004A4A934218BF8B420BD002F570529342C2
:1098300007D002F58062934203D002F58062934222
:1098400003D15A6C42F400425A6423683E4AB3F191
:10985000804F18BF934264D0A2F57C42934260D0FF
:1098600002F5806293425CD002F58062934258D048
:1098700002F57842934254D0A2F56C42934250D004
:1098800002F5943293424CD01A6842F001021A60F9
:10989000002055E004290CD0082911D00C2916D03D
:1098A00010291BD094F84330DBB2013B18BF0123D1
:1098B000A7E794F83F30DBB2013B18BF0123A0E7D4
:1098C00094F84030DBB2013B18BF012399E794F8CC
:1098D0004130DBB2013B18BF012392E794F84230DC
:1098E000DBB2013B18BF01238BE7042809D008280D
:1098F0000BD00C280DD010280FD0022384F8433051
:1099000087E7022384F83F3083E7022384F840305E
:109910007FE7022384F841307BE7022384F842305A
:1099200077E799680A4A0A40062A18BFB2F5803FCD
:1099300007D01A6842F001021A60002000E00120FE
:1099400010BD0020FCE700BF000001400004014002
:109950000700010010B504460B4611BB90F83E10FD
:10996000C9B2002B39D194F84420D2B2012A08BFE1
:10997000012940F0BD80002B3FD1022284F83E2017
:10998000002B56D1022284F844200C2B00F2B28026
:10999000DFE803F05FB0B0B08EB0B0B094B0B0B05C
:1099A0009A00042909D008290BD00C290DD01029C0
:1099B0000FD090F84310C9B2D3E790F83F10C9B266
:1099C000CFE790F84010C9B2CBE790F84110C9B288
:1099D000C7E790F84210C9B2C3E7042B05D0082BA3
:1099E00007D094F84720D2B2C0E794F84520D2B20D
:1099F000BCE794F84620D2B2B8E7042B09D0082B74
:109A00000BD00C2B0DD0102B0FD0022284F843204A
:109A1000B6E7022284F83F20B2E7022284F8402011
:109A2000AEE7022284F84120AAE7022284F842200D
:109A3000A6E7042B05D0082B07D0022284F8472084
:109A4000A3E7022284F845209FE7022284F84620FB
:109A50009BE72168CA6842F00202CA6001221946E7
:109A60002068FFF7B4FE2368244AB3F1804F18BF83
:109A700093422FD0A2F57C4293422BD002F5806214
:109A8000934227D002F58062934223D002F57842B8
:109A900093421FD0A2F56C4293421BD002F5943240
:109AA000934217D01A6842F001021A60002022E0A7
:109AB0002168CA6842F00402CA60CFE72168CA6818
:109AC00042F00802CA60C9E72168CA6842F0100281
:109AD000CA60C3E799680A4A0A40062A18BFB2F565
:109AE000803F09D01A6842F001021A60002002E0AB
:109AF000012000E0012010BD0020FCE70000014033
:109B00000700010090F83C30012B45D070B40123D0
:109B100080F83C30022380F83D3003685A689C6826
:109B20001E4E1F4DAB4218BFB34203D122F4700248
:109B30004D682A4322F070020D682A435A60036878
:109B4000164AB3F1804F18BF934217D0A2F57C425A
:109B5000934213D002F5806293420FD002F58062E7
:109B600093420BD002F57842934207D0A2F56C42A3
:109B7000934203D002F59432934204D124F080043E
:109B80008A6814439C60012380F83D30002380F8EC
:109B90003C30184670BC70470220704700000140FE
:109BA00000040140704770477047026852E8003F68
:109BB00023F0C00342E800310029F6D1026802F127
:109BC000080353E8003F23F40003083242E8003161
:109BD0000029F3D12023C0F888307047026852E88A
:109BE000003F23F4907342E800310029F6D1026867
:109BF00002F1080353E8001F0D4B0B40083242E806
:109C000000310029F3D1C36E012B06D02023C0F808
:109C10008C300023C36643677047026852E8003FF8
:109C200023F0100342E800310029F6D1EEE700BF2F
:109C3000FEFFFFEF1346D0F88820202A3DD110B553
:109C40000446002B18BF002939D00165A0F8543014
:109C5000A0F856300022C0F890202122C0F88820B9
:109C6000C26FCAB11749D163C26F17491164C26F7D
:109C70001649D164C26F0021116502682832016D56
:109C8000C06FFBF779FB38B11023C4F89030202364
:109C9000C4F8883001200FE0236840221A6222684D
:109CA00002F1080353E8003F43F08003083242E822
:109CB00000310029F3D1002010BD0220704701209F
:109CC000FAE700BFD39C00083F9D00084B9D0008A9
:109CD000704708B50346806BDB69B3F5807F18D009
:109CE0000023A0F85630026802F1080353E8003F51
:109CF00023F08003083242E800310029F3D10268E2
:109D000052E8003F43F0400342E800310029F6D119
:109D100008BDFFF7DDFFFBE708B5026852E8003F2A
:109D200023F0400342E800310029F6D12023C0F897
:109D3000883000238367FFF7CBFF08BD704708B565
:109D4000806BFFF7FBFF08BD704738B5846BD4F814
:109D50008820D4F88C5023689B6813F0800F01D0C2
:109D6000212A10D023689B6813F0400F01D0222DC8
:109D700010D0D4F8903043F01003C4F8903020464F
:109D8000FFF7E2FF38BD0023A4F856302046FFF766
:109D90000CFFE7E70023A4F85E302046FFF71EFF24
:109DA000E7E708B5806B0023A0F85E30A0F85630D6
:109DB000FFF7CAFF08BD704770B504460168CB695C
:109DC00008688D6840F60F021A4008D113F0200F82
:109DD00005D010F0200F34D115F0805F31D12AB1B9
:109DE0008B4A2A4033D18B4E304230D1E26E012A69
:109DF00000F0C68013F4801F03D015F4800F40F0EC
:109E00009B8113F0800F07D010F0800F40F09B81F2
:109E100015F4000F40F0978113F0400F03D010F0BD
:109E2000400F40F0978113F4000F03D010F0804FE3
:109E300040F0948113F0807F02D00028C0F292811C
:109E400070BD636F002BFBD020469847F8E713F0F6
:109E5000010F09D010F4807F06D001260E62D4F8DD
:109E600090103143C4F8901013F0020F0BD015F08E
:109E7000010F08D0216802260E62D4F8901041F03C
:109E80000401C4F8901013F0040F0BD015F0010F6B
:109E900008D0216804260E62D4F8901041F0020127
:109EA000C4F8901013F0080F0BD010F0200F00D161
:109EB0003AB1226808211162D4F890200A43C4F80C
:109EC000902013F4006F0CD010F0806F09D022683E
:109ED0004FF400611162D4F8902042F02002C4F8DF
:109EE0009020D4F89020002AAAD013F0200F09D097
:109EF00010F0200F02D115F0805F03D0636F0BB11B
:109F000020469847D4F8902023689B6813F0400FB0
:109F100002D112F0280F2CD02046FFF75FFE2368F5
:109F20009B6813F0400F20D0226802F1080353E829
:109F3000003F23F04003083242E800310029F3D10A
:109F4000D4F880306BB1344A1A65D4F88000FBF73E
:109F5000FFFC00283FF474AFD4F88000036D9847ED
:109F60006EE72046FFF7F0FE6AE72046FFF7ECFEBB
:109F700066E72046FFF7E8FE0023C4F890305FE76D
:109F800013F0100F3FF436AF10F0100F3FF432AF64
:109F900010230B6223689B6813F0400F00F092803F
:109FA000D4F8802013681D481D498B4218BF834296
:109FB00038D018318B4235D018318B4232D018311D
:109FC0008B422FD018318B422CD018318B4229D0A4
:109FD00018318B4226D001F556718B4222D01831B0
:109FE0008B421FD018318B421CD018318B4219D0B4
:109FF00018318B4216D018318B4213D018318B4256
:10A0000010D018318B420DD05B689BB20CE000BFC2
:10A010000100001020010004A39D00081000024070
:10A02000280002405B689BB2002B3FF409AFB4F8F4
:10A030005C1099427FF604AFA4F85E30D369B3F5A3
:10A04000807F32D0226852E8003F23F4807342E8D8
:10A0500000310029F6D1226802F1080353E8003FDD
:10A0600023F00103083242E800310029F3D12268CD
:10A0700002F1080353E8003F23F04003083242E8AE
:10A0800000310029F3D12023C4F88C300023E3668B
:10A09000226852E8003F23F0100342E80031002913
:10A0A000F6D1D4F88000FBF7B3FA02232367B4F8A3
:10A0B0005C10B4F85E309BB2C91A89B22046FFF733
:10A0C0007AFEBDE6B4F85C10B4F85E309BB2C91AF3
:10A0D00089B2B4F85E309BB2002B3FF4B1AE0029D8
:10A0E0003FF4AEAE226852E8003F23F4907342E89A
:10A0F00000300028F6D1226802F1080353E8000F6F
:10A100001A4B0340083242E800300028F3D12023E4
:10A11000C4F88C300023E3666367226852E8003F8E
:10A1200023F0100342E800300028F6D10223236711
:10A130002046FFF740FE83E64FF480130B62204673
:10A1400001F0DCF87CE6A36F002B3FF479AE2046EB
:10A15000984775E62046FFF7DFFD71E6204601F0DF
:10A16000CFF86DE6204601F0CAF869E6FEFFFFEF82
:10A1700008B5B0F86030D0F88C20222A05D00268EB
:10A18000936943F00803936108BD0268516ADBB22A
:10A19000826D0B401370836D01338365B0F85E30C0
:10A1A0009BB2013B9BB2A0F85E30B0F85E309BB230
:10A1B000002BE9D1026852E8003F23F4907342E893
:10A1C00000310029F6D1026802F1080353E8003F8C
:10A1D00023F00103083242E800310029F3D12023A3
:10A1E000C0F88C300023436703670368164A934224
:10A1F0000CD05B6813F4000F08D0026852E8003FEF
:10A2000023F0806342E800310029F6D1C36E012BB0
:10A2100016D10023C366026852E8003F23F0100302
:10A2200042E800310029F6D10368DA6912F0100F14
:10A2300001D010221A62B0F85C10FFF7BCFDA3E752
:10A24000F9F716FBA0E700BF000C005808B5B0F8FE
:10A250006020D0F88C30222B05D00268936943F03F
:10A260000803936108BD03685B6A816D13400B802E
:10A27000836D02338365B0F85E309BB2013B9BB2C5
:10A28000A0F85E30B0F85E309BB2002BEAD10268D5
:10A2900052E8003F23F4907342E800310029F6D1E0
:10A2A000026802F1080353E8003F23F0010308327B
:10A2B00042E800310029F3D12023C0F88C3000237C
:10A2C000436703670368164A93420CD05B6813F434
:10A2D000000F08D0026852E8003F23F0806342E894
:10A2E00000310029F6D1C36E012B16D10023C366BD
:10A2F000026852E8003F23F0100342E800310029D1
:10A30000F6D10368DA6912F0100F01D010221A6238
:10A31000B0F85C10FFF74FFDA4E7F9F7A9FAA1E741
:10A32000000C00582DE9F843B0F860600368DD695F
:10A33000D3F80090D3F80880D0F88C20222A05D0DA
:10A340009A6942F008029A61BDE8F8830446B0F8C1
:10A35000687008E0D4F89030002B4CD1B4F85E302F
:10A360009BB2002B4ED0002F00F0988015F0200FEC
:10A3700000F094802368596AF3B2A26D0B40137009
:10A38000A36D0133A365B4F85E309BB2013B9BB271
:10A39000A4F85E302368DD6915F0070FDED015F0F4
:10A3A000010F09D019F4807F06D001221A62D4F877
:10A3B00090301343C4F8903015F0020F0BD018F012
:10A3C000010F08D0236802221A62D4F8903043F0BB
:10A3D0000403C4F8903015F0040FBBD018F0010F3F
:10A3E000B8D0236804221A62D4F8903043F00203F4
:10A3F000C4F89030AEE72046FFF7A6FC0023C4F86F
:10A400009030ABE7226852E8003F23F4807342E8C3
:10A4100000310029F6D1226802F1080353E8001F39
:10A42000304B0B40083242E800310029F3D12023A1
:10A43000C4F88C3000236367236723682A4A934259
:10A4400003D05B6813F4000F06D1E36E012B0DD02F
:10A450002046F9F70DFA86E7226852E8003F23F01C
:10A46000806342E800310029F6D1EEE70023E3667D
:10A47000226852E8003F23F0100342E8003100292F
:10A48000F6D12368DA6912F0100F01D010221A6297
:10A49000B4F85C102046FFF78EFC64E7B4F85E3039
:10A4A0009BB2002B3FF450AFB4F868209A427FF67D
:10A4B0004BAF226802F1080353E8003F23F08053BA
:10A4C000083242E800310029F3D1084B6367226863
:10A4D00052E8003F43F0200342E800310029F6D162
:10A4E00032E700BFFEFFFFEF000C005871A100082B
:10A4F0002DE9F843B0F860600368DD69D3F8009097
:10A50000D3F80880D0F88C20222A05D09A6942F02E
:10A5100008029A61BDE8F8830446B0F8687008E064
:10A52000D4F89030002B4BD1B4F85E309BB2002BA6
:10A530004DD0002F00F0978015F0200F00F0938091
:10A5400023685B6AA26D33401380A36D0233A36559
:10A55000B4F85E309BB2013B9BB2A4F85E30236836
:10A56000DD6915F0070FDFD015F0010F09D019F4E0
:10A57000807F06D001221A62D4F890301343C4F8C9
:10A58000903015F0020F0BD018F0010F08D023689F
:10A5900002221A62D4F8903043F00403C4F89030D9
:10A5A00015F0040FBCD018F0010FB9D023680422B5
:10A5B0001A62D4F8903043F00203C4F89030AFE749
:10A5C0002046FFF7C1FB0023C4F89030ACE72268B7
:10A5D00052E8003F23F4807342E800310029F6D1AD
:10A5E000226802F1080353E8001F304B0B40083289
:10A5F00042E800310029F3D12023C4F88C30002335
:10A600006367236723682A4A934203D05B6813F485
:10A61000000F06D1E36E012B0DD02046F9F728F983
:10A6200087E7226852E8003F23F0806342E8003168
:10A630000029F6D1EEE70023E366226852E8003FE6
:10A6400023F0100342E800310029F6D12368DA69CB
:10A6500012F0100F01D010221A62B4F85C102046DC
:10A66000FFF7A9FB65E7B4F85E309BB2002B3FF41F
:10A6700051AFB4F868209A427FF64CAF226802F1DD
:10A68000080353E8003F23F08053083242E80031CA
:10A690000029F3D1074B6367226852E8003F43F07B
:10A6A000200342E800310029F6D133E7FEFFFFEF37
:10A6B000000C00584DA2000870B586B00446016831
:10A6C00083680269134342691343C26913430868EC
:10A6D000884A024013430B602268536823F44053B6
:10A6E000E1680B435360A1692268834B9A4201D011
:10A6F000236A19439068814B03400B43936022689F
:10A70000D36A23F00F03616A0B43D36222687C4B48
:10A710009A4221D07B4B9A4200F08C807A4B9A422D
:10A7200000F0A280794B9A4200F0B580784B9A42B3
:10A7300000F0C880774B9A4200F0F480764B9A4242
:10A7400000F01981754B9A4200F02C816A4B9A42B5
:10A7500000F03F81802333E0714B5B6D03F03803E1
:10A76000282B65D8DFE813F029006400640064003A
:10A7700064006400640064004D01640064006400CF
:10A7800064006400640064002B00640064006400E2
:10A7900064006400640064005E006400640064009F
:10A7A000640064006400640060006400640064008D
:10A7B00064006400640064006200012300E0082378
:10A7C0004D498A4200F02F81E069B0F5004F00F05A
:10A7D000AF81202B00F20782202B00F25182DFE8AC
:10A7E00013F01E0224024F024F0227024F024F02B3
:10A7F0004F022C024F024F024F024F024F024F02F4
:10A800004F0231024F024F024F024F024F024F02DE
:10A810004F024F024F024F024F024F024F024F02B0
:10A820004F023D021023CBE72023C9E74023C7E7AF
:10A830008023C5E73A4B5B6D03F00703052B11D866
:10A84000DFE813F00600E10008000A000C000E002B
:10A850000023B5E70823B3E71023B1E72023AFE7D0
:10A860004023ADE78023ABE72D4B5B6D03F007037F
:10A87000052B0ED8DFE803F003C90507090B0023F9
:10A880009EE708239CE710239AE7202398E74023BC
:10A8900096E7802394E7224B5B6D03F00703052BBB
:10A8A0000ED8DFE803F003B40507090B002387E7A0
:10A8B000082385E7102383E7202381E740237FE7F0
:10A8C00080237DE7164B5B6D03F00703052B0ED845
:10A8D000DFE803F0039F0507090B002370E7082357
:10A8E0006EE710236CE720236AE7402368E78023A4
:10A8F00066E700BFF369FFCF000C0058FFF4FF11BB
:10A90000001001400044004000480040004C00405E
:10A91000005000400014014000780040007C0040DE
:10A92000004402587D4B5B6D03F03803282B20D880
:10A93000DFE803F0151F1F1F1F1F1F1F711F1F1FA1
:10A940001F1F1F1F171F1F1F1F1F1F1F191F1F1F25
:10A950001F1F1F1F1B1F1F1F1F1F1F1F1D00012346
:10A960002EE708232CE710232AE7202328E740239B
:10A9700026E7802324E7694B5B6D03F00703052B73
:10A980000ED8DFE803F0034A0507090B002317E799
:10A99000082315E7102313E7202311E740230FE7CF
:10A9A00080230DE75D4B5B6D03F00703052B0ED88D
:10A9B000DFE803F003350507090B002300E7082350
:10A9C000FEE61023FCE62023FAE64023F8E6802387
:10A9D000F6E603F50E339B6D03F00703052B0ED847
:10A9E000DFE803F0031F0507090B0223E8E608234D
:10A9F000E6E61023E4E62023E2E64023E0E68023B7
:10AA0000DEE60423DCE60423DAE60423D8E60423A6
:10AA1000D6E60423D4E60423D2E60423D0E60423B6
:10AA2000CEE60423CCE6202B27D8022BC0F01A81D7
:10AA3000023B1E2B00F21881DFE813F050001601D4
:10AA400056001601160116015B00160116011601CB
:10AA500016011601160116016000160116011601F5
:10AA6000160116011601160116011601160116012E
:10AA700016011601160116016C00402B2CD14FF463
:10AA80000040626A264B33F81220B0FBF2F365688F
:10AA900005EB4501994200F2E980B3EB053F00F276
:10AAA000E780002633463146F6F72AF9090241EAE3
:10AAB000106100026B08C0182A46334641F10001BC
:10AAC000F6F71EF9A0F54072164B9A4200F2D280BA
:10AAD0002368D8603046D4E00120D2E0FDF798F931
:10AAE0000028CED10020CCE003A8FDF7A3F90498FC
:10AAF000F6E76846FDF7B8FA0198F1E7074B1B68DF
:10AB000013F0200F08D0054B1B68C3F3C1030648A0
:10AB1000D840E5E70548B4E70348B2E700440258E7
:10AB20009C320108FFFC0F000090D00300093D009B
:10AB3000202B15D8202B00F29F80DFE803F031375F
:10AB40009D9D3A9D9D9D3F9D9D9D9D9D9D9D449D4F
:10AB50009D9D9D9D9D9D9D9D9D9D9D9D9D9D50000F
:10AB6000402B1BD1626A4D4B33F81230B0FBF3F02F
:10AB70006268530803EB4000B0FBF2F0A0F1100252
:10AB80004FF6EF739A4279D883B223F00F03C0F3E4
:10AB9000420018432368D860002072E0012070E072
:10ABA000FCF7C0FA0028DDD100206AE0FCF7CCFAFF
:10ABB000F8E703A8FDF73EF90498F3E76846FDF7C8
:10ABC00053FA0198EEE7364B1B6813F0200F08D0BC
:10ABD000334B1B68C3F3C1033248D840E2E7324825
:10ABE000C0E73048BEE7402B17D14FF40040626AFF
:10ABF0002A4B33F81230B0FBF3F0636800EB5300DC
:10AC0000B0FBF3F0A0F110024FF6EF739A4242D876
:10AC1000236880B2D860002033E0012031E0FCF7E7
:10AC200081FA0028E3D100202BE0FCF78DFAF8E749
:10AC300003A8FDF7FFF80498F3E76846FDF714FA58
:10AC40000198EEE7164B1B6813F0200F08D0144B49
:10AC50001B68C3F3C1031348D840E2E71248C6E7B4
:10AC60001048C4E701200CE001200AE0012008E0C0
:10AC7000012006E0012004E0012002E0012000E0C4
:10AC800001200123A4F86A30A4F868300023636728
:10AC9000A36706B070BD0120F3E700BF9C32010836
:10ACA000004402580090D00300093D00836A13F06D
:10ACB000010F06D00268536823F40033C16A0B43C6
:10ACC0005360836A13F0020F06D00268536823F4BE
:10ACD0008033016B0B435360836A13F0040F06D07B
:10ACE0000268536823F48023416B0B435360836AEB
:10ACF00013F0080F06D00268536823F40043816BF9
:10AD00000B435360836A13F0100F06D002689368F8
:10AD100023F48053C16B0B439360836A13F0200FBD
:10AD200006D00268936823F40053016C0B439360D0
:10AD3000836A13F0400F0AD00268536823F480132B
:10AD4000416C0B435360436CB3F5801F0BD0836A97
:10AD500013F0800F06D00268536823F40023C16CFF
:10AD60000B43536070470268536823F4C003816C3F
:10AD70000B435360EBE72DE9F84305460F461646B3
:10AD80009946DDF820802C68E46937EA04030CBF9B
:10AD90004FF0010C4FF0000CB44532D1B8F1FF3F39
:10ADA000F1D0F8F735FEA0EB090040452CD8B8F1FA
:10ADB000000F2BD02B681A6812F0040FE3D0DA6969
:10ADC00012F0080F11D1DA6912F4006FDBD04FF4E2
:10ADD00000621A622846FEF701FF2023C5F8903072
:10ADE000002385F8843003200CE008241C622846E8
:10ADF000FEF7F4FEC5F89040002385F8843001206A
:10AE000000E00020BDE8F8830320FBE70320F9E71A
:10AE10002DE9F04182B01E46D0F88830202B5BD15E
:10AE200004460D469046002A18BF002901D1012092
:10AE300053E00023C0F890302123C0F88830F8F7A1
:10AE4000E7FD0746A4F85480A4F85680A368B3F53C
:10AE5000805F02D04FF0000816E0236943B34FF043
:10AE6000000811E02023C4F88830032035E038F8CA
:10AE7000023B2268C3F308039362B4F8562092B2EF
:10AE8000013A92B2A4F85620B4F856309BB293B16E
:10AE900000963B46002280212046FFF76CFF0028E9
:10AEA000E0D1002DE3D015F8012B23689A62E4E786
:10AEB000A8460025E8E700963B46002240212046B0
:10AEC000FFF759FF18B92023C4F8883005E0202384
:10AED000C4F88830032000E0022002B0BDE8F08111
:10AEE0002DE9F04383B01E46D0F88C30202B7ED164
:10AEF00004460D469046002A18BF002901D10120C2
:10AF000076E00023C0F890302222C0F88C20C3667F
:10AF1000F8F77EFD0746A4F85C80A4F85E80A3687D
:10AF2000B3F5805F06D0A3B9226972B9FF22A4F8F5
:10AF3000602014E0226922B940F2FF12A4F86020D8
:10AF40000DE0FF22A4F8602009E07F22A4F8602031
:10AF500005E0B3F1805F0AD00022A4F86020B4F8C5
:10AF60006080B3F5805F0CD04FF0000924E02269C7
:10AF70001AB97F22A4F86020F1E73F22A4F86020EC
:10AF8000EDE7236913B14FF0000915E0A94600254C
:10AF900012E02023C4F88C30032029E023685A6A89
:10AFA0005FFA88F3134005F8013BB4F85E2092B2D3
:10AFB000013A92B2A4F85E20B4F85E309BB28BB135
:10AFC00000963B46002220212046FFF7D4FE0028B1
:10AFD000DFD1002DE2D123685B6A08EA030329F878
:10AFE000023BE2E72023C4F88C30002000E002207E
:10AFF00003B0BDE8F08330B583B004460023C0F849
:10B000009030F8F705FD05462268126812F0080F27
:10B0100010D123681B6813F0040F28D12023C4F833
:10B020008830C4F88C300020E066206784F8840003
:10B0300003B030BD6FF07E430093034600224FF40F
:10B0400000112046FFF797FE0028E2D0226852E860
:10B05000003F23F0800342E800310029F6D120238D
:10B06000C4F88830002384F884300320E0E76FF0D0
:10B070007E4300932B4600224FF480012046FFF7C9
:10B080007AFE0028CAD0226852E8003F23F4907369
:10B0900042E800310029F6D1226802F1080353E8A2
:10B0A000003F23F00103083242E800310029F3D1C8
:10B0B0002023C4F88C30002384F884300320B7E7C1
:10B0C00078B310B50446D0F888300BB32423C4F805
:10B0D00088302268136823F0010313602046FFF7CD
:10B0E000EBFA012813D0A36ABBB92268536823F492
:10B0F000904353602268936823F02A039360226888
:10B10000136843F0010313602046FFF774FF10BD7E
:10B1100080F88430F8F734FBD8E72046FFF7C6FD07
:10B12000E3E701207047000010B48165A0F85C20BF
:10B13000A0F85E20002343678368B3F5805F06D0E4
:10B14000A3B9036973B9FF23A0F8603014E0036961
:10B1500023B940F2FF13A0F860300DE0FF23A0F800
:10B16000603009E07F23A0F8603005E0B3F1805F34
:10B170002DD00023A0F860300023C0F890302223A7
:10B18000C0F88C30016801F1080353E8003F43F038
:10B190000103083141E80034002CF3D1436EB3F1D0
:10B1A000005F1ED08368B3F5805F42D0294B4367B0
:10B1B0000369002B43D0026852E8003F43F49073C8
:10B1C00042E800310029F6D1002010BC7047036925
:10B1D0001BB97F23A0F86030CEE73F23A0F8603092
:10B1E000CAE7B0F868309342DCD88368B3F5805F73
:10B1F00019D0194B4367036943B1026852E8003F15
:10B2000043F4807342E800310029F6D1026802F16C
:10B21000080353E8003F43F08053083242E800310E
:10B220000029F3D1D0E70369002BE2D10B4B436730
:10B23000E1E70369002BB9D1094B4367B8E702681E
:10B2400052E8003F43F0200342E800310029F6D1E4
:10B25000BAE700BF71A1000825A30008F1A4000807
:10B260004DA2000838B5D0F88C30202B19D1002A17
:10B2700018BF002917D00023C36603680B4CA342F4
:10B280000CD05B6813F4000F08D0046854E8003F4A
:10B2900043F0806344E80035002DF6D1FFF744FF0A
:10B2A00000E0022038BD0120FCE700BF000C005880
:10B2B000436E2BB90123A0F86A30A0F868307047BC
:10B2C00030B403689A68C2F342629968490F094D25
:10B2D0006B5C1B01084C615C93FBF1F3A0F86A30D6
:10B2E000AB5C1B01A25C93FBF2F3A0F8683030BCAE
:10B2F000704700BFBC320108B43201087047704784
:10B30000704790F88430012B18D0012380F88430E6
:10B310002423C0F8883003681A68196821F00101F5
:10B32000196022F000520023436601680A6020225F
:10B33000C0F8882080F88430184670470220704793
:10B3400038B590F88430012B1DD00446012380F8D5
:10B3500084302423C0F8883003681D681A6822F0FE
:10B3600001021A600268936823F0604319439160F8
:10B37000FFF79EFF23681D602023C4F8883000205B
:10B3800084F8840038BD0220FCE738B590F884309A
:10B39000012B1DD00446012380F884302423C0F8FB
:10B3A000883003681D681A6822F001021A6002687A
:10B3B000936823F0606319439160FFF779FF236876
:10B3C0001D602023C4F88830002084F8840038BD34
:10B3D0000220FCE7014B1868704700BF2C000024D6
:10B3E00070B50D4E0D4D761BB61006D0002455F8E5
:10B3F000043B01349847A642F9D1094E094D761B0A
:10B4000007F050FEB61006D0002455F8043B013476
:10B410009847A642F9D170BDC4380108C438010864
:10B42000CC380108C4380108024B0146186800F006
:10B430000BB800BF2C000024024B0146186804F032
:10B4400085BE00BF2C0000242DE9F04F01F10B0652
:10B45000162E83B0044624D8102900F2BA8000F0DA
:10B46000F5FA102618220220B54F3A44A2F108013D
:10B4700053688B4200F0BA805A68D96822F0030200
:10B480001A449D68E9608D60516841F001012046D1
:10B49000516003F1080500F0DFFA284603B0BDE86B
:10B4A000F08F36F0070600F19480B14200F29180EF
:10B4B00000F0CCFAB6F5FC7FC0F09A81730A00F078
:10B4C0008F80042B00F26F81B30903F1390003F17F
:10B4D000380CC3009A4F3B44A3F108055B689D42BA
:10B4E00006D10CE0002980F22781DB689D4206D05E
:10B4F0005A6822F00302911B0F29F3DD60463D6973
:10B50000DFF840C265457CD06A6822F00302931BD5
:10B510000F2B00F37B81002BC7E904CC80F26C81F8
:10B52000B2F5007F80F01A81D308796801334FEAC1
:10B53000521E012202FA0EF20A4357F833E0C5F810
:10B5400008E007EBC3010839E9607A6047F8335037
:10B55000CEF80C50831001219940914257D81142E6
:10B5600006D120F003004900114200F10400FAD096
:10B5700007EBC0094D468646D5F80C80454508D1F5
:10B580001DE1002B80F22481D8F80C80454500F0A5
:10B590001681D8F8042022F00302931B0F2BF0DD54
:10B5A0002046D8E9025408EB060146F00106C8F827
:10B5B0000460EC60A56043F00104C7E90411C1E92F
:10B5C00002CC4C6048F8023000F046FA08F1080559
:10B5D00002E00C2323600025284603B0BDE8F08F6D
:10B5E0004FF4007340204FF03F0C73E7D3689A424A
:10B5F00008BF02307FF440AF3D69DFF848C16545C0
:10B6000082D17A688310012199409142A7D9BD68FF
:10B610006B6823F003094E4503D8A9EB06030F2BF3
:10B620007ADCDFF824B1494BDBF800201B680132DB
:10B63000334405EB090A00F0338103F580530F33DF
:10B6400023F47F6828F00F084146204600F06CFC88
:10B65000411C024600F0F380824500F2EE803C4B34
:10B66000196841441960084600F04E81DBF800106B
:10B67000019301311BBFA2EB0A0A5044CBF8002012
:10B68000186012F0070B00F01781CBF108010A4493
:10B69000CBF5805190440831A1EB0801C1F30B0AAE
:10B6A00051462046009200F03FFC421CDDE9002399
:10B6B00000F04F81801A00EB0A081968BA6048F060
:10B6C00001005144BD425060196000F02981B9F178
:10B6D0000F0F40F227816868A9F10C0C2CF0070CC1
:10B6E00000F0010040EA0C0068604FF0050E05EB29
:10B6F0000C00BCF10F0FC0E901EE00F2328150687E
:10B700001546144B1A688A4238BF1960124B1A68E2
:10B710008A4238BF196094E0AA1943F0010346F049
:10B7200001066E602046BA60536000F095F9083556
:10B73000284603B0BDE8F08FD9681A44A1E600BFDF
:10B74000580400246004002460080024442B0024D2
:10B75000142B00243C2B0024402B0024B2F5206F36
:10B760004FEA522363D3142B00F2B78003F15C013C
:10B77000C9005B3307EB010E7958AEF1080E8E4518
:10B7800000F091804B6823F00303934202D989684B
:10B790008E45F7D1D1F80CE07A68C5E9021ECEF8E3
:10B7A0000850CD60D6E6142B59D9542B00F29D8059
:10B7B000330B03F16F0003F16E0CC3008AE60EF148
:10B7C000010E1EF0030F05F108057FF4D5AE51E020
:10B7D000424445465368D8F80C1043F001035360C7
:10B7E00055F8083F2046D9608B6000F035F9F3E644
:10B7F000F00806F1080237E62A442046536843F071
:10B8000001035360083500F027F9E5E6A919204641
:10B8100046F0010643F001046E60C7E90411C1E976
:10B8200002CC4C60AB5000F017F90835D4E6930910
:10B8300003F13901C90038339CE7BD425FD0BD68D0
:10B84000686820F003084645A8EB060302D80F2BD2
:10B850003FF762AF204600F0FFF80025BCE603F199
:10B860005C0003F15B0CC30034E659F808394B4522
:10B8700040F0968010F0030F00F1FF30F5D17B68A7
:10B8800023EA01037B60490099423FF6C0AE19B933
:10B89000BDE649000EF1040E1942FAD0704667E683
:10B8A00003F11008D0E69A104FF001087B6808FAFF
:10B8B00002F21A437A6070E702EB08014942C1F3D1
:10B8C0000B0A51462046009200F02EFB431CDDE996
:10B8D00000237FF4EFAEDA46EFE6542B25D8130BA6
:10B8E00003F16F01C9006E3344E7B3F5AA7F25D891
:10B8F000F30B03F1780003F1770CC300EAE5294B61
:10B90000186840441860B1E6CAF30B0CBCF1000F94
:10B910007FF4ACAEBD68C84448F001006860F0E652
:10B920001546EEE60123536094E7B3F5AA7F23D8CA
:10B93000D30B03F17801C90077331BE740F254526F
:10B94000934223D8B30C03F17D0003F17C0CC300B8
:10B95000C0E5ABF1080BD844A8EB02084FF0000A91
:10B96000ABE605F108012046009304F0EFFBBD684B
:10B97000009B68681968C4E640F254518B420BD8AA
:10B98000930C03F17D01C9007C33F3E64FF47E7321
:10B990007F204FF07E0C9DE54FF47E717E23E9E61B
:10B9A0007B6870E7142B0024830730B548D0541E01
:10B9B000002A3FD0CAB2034601E0013C3AD303F863
:10B9C000012B9D07F9D1032C2DD9CDB245EA0525D0
:10B9D0000F2C45EA054536D9A4F1100222F00F0CD0
:10B9E00003F1200EE6444FEA121C03F1100242E973
:10B9F000045542E9025510327245F8D10CF10102AA
:10BA000014F00C0F03EB021204F00F0C13D0ACF186
:10BA1000040323F003030433134442F8045B93420A
:10BA2000FBD10CF003042CB1CAB21C4403F8012B67
:10BA30009C42FBD130BD64461346002CF4D1F9E79B
:10BA400003461446BFE71A46A446E0E7014805F05E
:10BA500049BA00BF4C2B0024014805F045BA00BF8D
:10BA60004C2B00240FB400B5074983B004AB086821
:10BA700053F8042B8168019301F06CFB03B05DF86F
:10BA800004EB04B0704700BF2C00002470B50546DD
:10BA900088B008460C46F5F7D3FC224EAA6B0590F9
:10BAA00001214318CDE9066104A8022104940393FF
:10BAB000AC680190029122B3636E13F0010FB4F9E8
:10BAC0000C309AB201D1980525D5910406D4626E46
:10BAD00043F4005322F40052A3816266284601AA6F
:10BAE000214604F039FC636E002814BF4FF0FF3587
:10BAF0000A25DA0702D4A3899B0506D5284608B093
:10BB000070BD284604F02AFAD6E7A06D05F0ECF9DE
:10BB1000284608B070BDA06D05F0E4F9B4F90C300A
:10BB20009AB2D2E750310108024B01461868FFF77C
:10BB3000ADBF00BF2C00002410B4044C03460A46DD
:10BB4000206810BC194600F003B800BF2C00002488
:10BB50002DE9F84F1746002900F0988007F10B05F2
:10BB600080460C46FFF772FF162D5DD810252A4639
:10BB7000AF425ED854F8041C21F003069642A4F1AB
:10BB8000080962DABC4BD3F808C009EB060084450B
:10BB900000F09780D0F804C02CF0010303445B68E8
:10BBA000DB0768D42CF0030C06EB0C03934247DA56
:10BBB000CB0710D454F8083CA9EB030ADAF8043098
:10BBC00023F003018C44B444944580F2118173182E
:10BBD000934280F2E88039464046FFF735FC07463D
:10BBE000E0B154F8043C23F001034B44A0F10802F7
:10BBF000934200F0D280321F242A00F2F580132AEB
:10BC000000F2AC8003462246116819605168596001
:10BC100092689A602146404604F098FA4046FFF741
:10BC20001BFF3846BDE8F88F25F00705002D2A4692
:10BC30009EDA0C23C8F8003000273846BDE8F88F9C
:10BC40001E46D0E90223D3609A60731B0F2B22D8C3
:10BC5000D9F8043003F0010333434E44C9F80430EB
:10BC6000736843F00103736040462746FFF7F4FE14
:10BC70003846BDE8F88FC907ADD454F8083CA9EBA5
:10BC8000030ADAF8041021F00301A0E7BDE8F84F39
:10BC90001146FFF7D9BBD9F8041001F0010129437F
:10BCA000C9F8041009EB05014E4443F001034B6051
:10BCB000736843F0010308317360404604F046FAAC
:10BCC000D2E7DCF8040020F0030B06EB0B0C05F1C7
:10BCD000100084454DDAC9073FF57DAF54F8081CC4
:10BCE000A9EB010ADAF8041021F003018B44B344F4
:10BCF00058453FF76CAF5746DAF80C1057F8080F65
:10BD0000321F242AC160886000F2DB80132A40F2CF
:10BD1000D6802168CAF808106168CAF80C101B2A7E
:10BD200000F2DF8008340AF11002216811606168B6
:10BD30005160A16891600AEB0501ABEB050242F08E
:10BD4000010299604A60DAF8043003F001031D43F0
:10BD50004046CAF80450FFF77FFE6EE72368036091
:10BD6000636843601B2A68D804F1080200F10803E5
:10BD70004AE709EB05029A60ACEB050343F00103C7
:10BD8000536054F8043C03F001031D43404644F85B
:10BD9000045CFFF761FE27464FE750F8043C23F0B0
:10BDA00003031E4451E75746DAF80C1057F8080F02
:10BDB000321F242AC16088604CD8132A48D92168D0
:10BDC000CAF808106168CAF80C101B2A56D8083443
:10BDD0000AF110021E462368136063685360A3686B
:10BDE0009360D1463C4630E7214605F04BF911E718
:10BDF000D0E902135746CB60996057F8081FDAF86C
:10BE00000C30CB60321F242A99602DD8132A29D9EF
:10BE10002368CAF808306368CAF80C301B2A42D875
:10BE200008340AF1100322681A6062685A60A26836
:10BE30009A606646D1463C4607E7A3688360E3689C
:10BE4000C360242A26D004F1100200F11003DBE6BF
:10BE50003A46BFE7214638461E46D14605F012F95C
:10BE60003C46F2E63B46DEE7214638466646D1468A
:10BE700005F008F93C46E8E658040024A168CAF831
:10BE80001010E168CAF81410242A20D010340AF1E6
:10BE900018029FE7236903616169416104F1180297
:10BEA00000F11803B0E6A368CAF81030E368CAF8D6
:10BEB0001430242A21D010340AF11803B3E73A468B
:10BEC00033E72146384605F0DDF8164B33E72269A3
:10BED000CAF818206269CAF81C2018340AF1200236
:10BEE00078E7A168CAF81010E168CAF81410242A8B
:10BEF0000DD010340AF1180217E72369CAF8183078
:10BF00006369CAF81C3018340AF120038BE72269F0
:10BF1000CAF818206269CAF81C2018340AF12002F5
:10BF200003E700BF5804002438B5074D002204463B
:10BF300008462A60F7F782F8431C00D038BD2B680A
:10BF4000002BFBD0236038BD582B00242DE9F04393
:10BF5000694CD4F8008083B004460E4617461D464F
:10BF6000B8F1000F03D0D8F83830002B77D0022F6B
:10BF700005D0012F00F2AC80002DC0F2A980636EC5
:10BF8000DA0752D52146404603F0B4FF216B41B198
:10BF900004F14003994202D0404604F0D7F8002350
:10BFA0002363B4F90CC000231CF0800FA36163600D
:10BFB00064D12CF44A6C2CF0030C022FA4F80CC0B2
:10BFC0006AD001AB6A462146404605F015F8A389C0
:10BFD0001843A081002D2FD0002E2ED0D8F8383055
:10BFE000002B38D0009B2660AB42B4F90C301CBF4C
:10BFF00043F40063A381012F04BF43F00103A38135
:10C000009AB213F00803C4E904652CD0D1075DD5BA
:10C010006D42A561656E002315F00105A36027D070
:10C020000025284603B0BDE8F083A3899B05A9D469
:10C03000A06D04F057FFA5E7009D2846FFF7F4F92F
:10C040000646002847D0A38943F08003A381D8F88F
:10C050003830002BC6D1404603F080FFC2E740468F
:10C0600003F07CFF83E7A360656E15F00105D7D16F
:10C07000930524D5284603B0BDE8F08321694046E6
:10C0800004F064F8B4F90CC02CF44A6C2CF0030CE6
:10C09000022FA4F80CC094D10025002204F1430320
:10C0A000A2600122C4E904322360636E4CF0020CEA
:10C0B000D807A4F80CC0DDD41CF4007FDAD1A06D41
:10C0C00004F012FF284603B0BDE8F083A560CBE77B
:10C0D0004FF0FF35CEE7DDF80090A94504D0484683
:10C0E000FFF7A2F9064620B9B4F90CC04FF0FF35AE
:10C0F000D3E74D46A7E700BF2C00002410B50C463F
:10C10000B1F90E1005F054FD002803DB236D034444
:10C11000236510BDA38923F48053A38110BD00BF04
:10C120002DE9F0410C46B1F90C101F46CB05054630
:10C1300016460BD421F48051A1813B46B4F90E1070
:10C1400032462846BDE8F04102F0AEBDB4F90E100B
:10C150000223002204F0CAFEB4F90C10EAE700BF83
:10C1600010B50C46B1F90E1004F0C0FEA389421CB4
:10C170000EBF23F4805343F480532065A38110BD88
:10C18000B1F90E1002F020BEA2B330B540EA0104AE
:10C19000A40784460B462AD09CF800000C78844201
:10C1A0002FD1012A0DD0E64660B11EF8010F11F81B
:10C1B000014F6FEA0E03A042134422D11CEB03038C
:10C1C000F2D1002030BD0468194653F8045BA4F195
:10C1D000013EAC4284462EEA040E00F104000BD16D
:10C1E000043A84461946ECD01EF0803FE9D1032A78
:10C1F000E9D8D1E7104670479CF800000C78A042BF
:10C20000D1D0001B30BD00BF2DE9F04F1C46984B2C
:10C210001B68A1B0002581461846884608921C95E7
:10C220000493F5F70DF9002183460020CDE90601BE
:10C23000CDF86C804246174612F8013B2D2B2FD8C3
:10C24000DFE813F0A1002E002E002E002E002E009D
:10C250002E002E002E00AF00AF00AF00AF00AF00E9
:10C260002E002E002E002E002E002E002E002E005E
:10C270002E002E002E002E002E002E002E002E004E
:10C280002E002E00AF002E002E002E002E002E00BD
:10C290002E002E002E002E002E0006042E00FC0381
:10C2A00000220A92302B7ED0002209922F2B1C46AE
:10C2B00040F233854FF0000A38465646554612E0A4
:10C2C0000130082D1B90C8BF0AEB8A0A0478C6BF4C
:10C2D00003EB4A03A3F1300AA2F130062F2C05F13B
:10C2E0000105234670DD06EB8602392C03EB420282
:10C2F000E6DD04995A46FFF747FF0346002835D18B
:10C300001B9A11465A441B9211F80B40002D40F025
:10C31000AC85302C40F06485C2F101015318013224
:10C320001B921478302CF9D0A4F13102082A00F2C3
:10C330003883A4F1300E1B9C03F1010B002301256F
:10C340002746049306EB86060EEB46060023621C86
:10C350001B926478A4F13001092900F2ED820133C7
:10C360008E46002940F0B8841B9CF0E70023652C22
:10C3700004959B469E4601D0452C32D1002D7CD1A0
:10C38000099A1A4378D1089B13B1089BC3F800801F
:10C390004FF0000BCDF810B00499584621B0BDE81D
:10C3A000F08F1B9247E77B7803F0DF03582B00F0F8
:10C3B000748401371B973B78302BFAD0002B00F0A8
:10C3C000CC800122099271E704995A46FFF7DCFEFE
:10C3D0000346002800F0D68004954FF0000B5B4622
:10C3E000DE4600220B92002D00F09380049A134643
:10C3F000002A08BF2B4630460493F4F7C3F80B46D7
:10C400000246CDE906230B9B102DA3EB0B032C4614
:10C41000A8BF1024092D0E9313DD164B03EBC403A4
:10C4200053E91223F5F7CCF8CDE906015046F4F7AD
:10C43000A9F802460B46DDE90601F3F767FFCDE9EF
:10C4400006010F2D00F3A7800E9B002B00F018842F
:10C450000E9B40F39283162B40F3F9840E9AC5F19C
:10C460002503934280F20C850E9B2C1B1C4498E004
:10C47000C4360108883701080025DDF86C8008F112
:10C4800001021B9298F801402B2C00F087822D2C82
:10C4900000F0218200220E92A4F13002092A00F25B
:10C4A0001582302C05D11B9A01321B921478302C46
:10C4B000FAD0A4F13102082A93D81B990B914A1C97
:10C4C0001B92A4F130004C782F2C09DC00F034BC16
:10C4D00001321B929CF801402F2CA1F1300006DDA7
:10C4E00000EB8001392C944604EB4101F0DD0B99FF
:10C4F000521A082A40F3208444F61F620B920E9AC7
:10C50000002A3FF470AF0B9A52420B92002D7FF439
:10C510006DAF099A134320D1BEF1000F7FF433AF02
:10C52000692C00F03B8400F34183492C00F03684F1
:10C530004E2C7FF428AFAC491BA804F0D5FB002893
:10C540003FF421AF1B9B1B78282B00F06D85A7487B
:10C5500005F07CFB8346049103E04FF0000BCDF81F
:10C5600010B0089A0AB11B9B13600A9B002B3FF482
:10C5700013AF049901F1004304930499584621B084
:10C58000BDE8F08F1B9A049502EB0B011B9112F88A
:10C590000B409B46DEE60E9B2C1B1C44002C40F3FC
:10C5A0000A8314F00F000AD0914901EBC001DDE9C4
:10C5B0000623D1E90001F5F703F8CDE9060134F0CF
:10C5C0000F0340F08B8200230993049A00962B46B8
:10C5D0003946484604F052FE1390002800F0558377
:10C5E0000B9BABEB03000E9B002BB4BF024600225B
:10C5F0000F9223EAE3730022934612939046139C12
:10C600004846616804F0BAFD0746002800F0418101
:10C6100022690232920004F10C010C30F4F7F2FCB2
:10C62000DDE9060104910B461EA901911DA90B909D
:10C6300002460091484605F0CDF91C90002800F014
:10C6400018810121484604F0C1FE8046002800F010
:10C6500020811D9B002BC0F20F810F9A129D9E1806
:10C66000099A1E9C9B1A2344624A013B9342C4F1DF
:10C67000360480F2AE80D21A1F2AA4EB020400F323
:10C680001D814FF0010A00230AFA02FA0C93099B5C
:10C6900025443444A6421D443346A8BF2346AB423A
:10C6A000A8BF2B46002B02DDE41AED1AF61A0F9BE9
:10C6B000002B00F3BE80002C00F3D2800E9B002BD9
:10C6C00000F3DE80002D00F3EF80002E08DD4146F0
:10C6D0003246484604F0B6FF8046002800F0D98074
:10C6E0001C993A46484605F045F88346002800F074
:10C6F000D0800026C368C6604146109305F01AF842
:10C70000B042C0F2638400F0D2834146584605F03F
:10C71000C3F900224FF0804304460D46F4F716F8A3
:10C7200000286FD0109B002B00F0E180079B119335
:10C73000314B314C0022CDE90C2335462F4E119A56
:10C740002F4B02EA060A9A4500F0FC80099B93B140
:10C75000BAF1D46F0FD822A3D3E90023284621468B
:10C76000F3F7F4FF002840F087810D9B03F1D663B7
:10C77000A3EB0A030D93049E0B98DDE90C233146CD
:10C78000CDE9042305F09CF802460B46DDE90401DF
:10C79000F4F716FF33460B9AF3F7B8FDCDE906011F
:10C7A0000E46099B23B9154B33409A4500F0028190
:10C7B0001C99484604F008FD3946484604F004FD3B
:10C7C0004146484604F000FD5946484604F0FCFC4A
:10C7D00015E700230C934FF0010A58E7AFF30080F0
:10C7E0000000C0FFFFFFDF41D8330108C43101085A
:10C7F0008837010802FCFFFF0000F03F0000F07FD7
:10C800000000E07FAE4B204629460022F4F7D8FE18
:10C81000109B024605460C46002B64D101F10043F3
:10C8200014901593079B1193DDE91423CDE90C2394
:10C8300084E741461A46484604F0A4FE804640B3C9
:10C8400001461C9A484604F0EFFD10B310901C9965
:10C85000484604F0B9FC109B1C93002C7FF72EAFC8
:10C860001C992246484604F0EDFE1C9000287FF4F7
:10C8700025AFBA465E460FE0129A0F9ED51AEFE634
:10C880003946129A484604F07DFE074600287FF498
:10C8900019AFBA465E461C982223C9F80030894B6E
:10C8A00004934FF0000BB4E039462A46484604F0A2
:10C8B000C9FE074600287FF408AFEAE7824A4FF036
:10C8C000010AD31A0AFA03F30C93E0E60022CDF82A
:10C8D0006C800B9287E501220E9208F102021B92F6
:10C8E00098F80240D8E50B46CDE914239AE7DDE934
:10C8F0000612002940F0AF80C2F313031192002BFF
:10C9000040F0AF80714B002220462946F3F714FF18
:10C91000002840F0AE826A4B204629460022F4F7F8
:10C920004FFE01F1004305460C4618901993DDE9CE
:10C930001823CDE90C2301E7652C4FF0010E3FF4DD
:10C940009CAD19E5A2F154730793DDE90623DDE9F7
:10C950000C01CDE9060110461946CDE90C2304F07F
:10C96000AFFF02460B46DDE90601F4F729FEDDE9DB
:10C970000C23F3F7CBFC564A0E409642CDE9060154
:10C9800076D9049A534B9A4202D10B9B013380D043
:10C99000504A4FF0FF33CDE9063209E700220E92EC
:10C9A0009BE7652C00F0FB80452C00F0F8804FF0F1
:10C9B000010EAEE528462146F5F734F8F3F72EFED2
:10C9C0000B46024621462846F3F79EFC109C069D26
:10C9D000C6F3130644EA050C5CEA060304460D465A
:10C9E00000F0C28032A3D3E90023F3F7A5FE48B9D3
:10C9F00031A3D3E9002320462946F3F7BBFE0028E4
:10CA00003FF4D6AEDDE906341C9804945E46BA467F
:10CA10009B460146484604F0D7FB5146484604F081
:10CA2000D3FB4146484604F0CFFB1399484604F037
:10CA3000CBFB3146484604F0C7FB92E501230A933D
:10CA40007A1C1B927B78002B3FF49DAC174629E49F
:10CA500000230A93F4E7DDE90612012900F074814E
:10CA600011921D4B194C0022CDE90C23002565E6DF
:10CA700001F15476079694E621462846F4F7B2FF72
:10CA8000012838BF0120F3F77DFD109B02460546C3
:10CA90000C46002B40F0698101F10043169017937A
:10CAA000DDE91623CDE90C235FE600BFAFF300807C
:10CAB0009535A094FFFFDF3F35E5AF350000E03F3F
:10CAC0000000E03F0000F07FE2FBFFFF0000F03FCE
:10CAD000FFFF9F7CFFFFEF7F0000F0BFB3F59A7F61
:10CAE00000F3D380102B4FEA2314A54B40F3C682EA
:10CAF000DDE906019846099300239A4614F0010FD8
:10CB00000AF1010A4FEA640404D0D8E90023F4F7DB
:10CB100057FD0123012C08F10808EFD10BB1CDE935
:10CB20000601099B03EBCA01079BA3F1547307930A
:10CB3000DDE90623D1E90001F4F742FD914BCDE98F
:10CB400006010B400A4690498B4200F29E80A1F5F7
:10CB500080118B4240F21C828C494FF0FF33CDE9AB
:10CB600006310023099330E583A3D3E90023F3F7CB
:10CB7000E3FD00283FF41CAE44E71633FFF60BAD8F
:10CB80000B9BABEB0302824B03EBC203DDE9060117
:10CB9000D3E90023F4F73EFE83460491E1E400224A
:10CBA000049293464FF0010EFFF7EABB6E2C3FF460
:10CBB000C2ACFFF7E8BB3FF406AD644214F00F02CD
:10CBC0000AD0734B03EBC203DDE90601D3E900236E
:10CBD000F4F720FECDE9060124113FF4F4AC1F2C3C
:10CBE00035DC14F01003DDE9060118BF6A23DFF815
:10CBF000A48109930023E20704D5D8E90023F4F7C0
:10CC0000DFFC0123641008F10808F4D10BB1CDE971
:10CC10000601099B93B1DDE90601C1F30A52C2F195
:10CC20006B03002B0ADD1F2B40F350820020342BB6
:10CC3000069040F356824FF05C730793DDE90601DE
:10CC400000220023F3F76EFD00283FF4BEAC222340
:10CC50004FF0000BC9F80030CDF810B081E41E9BF6
:10CC600006931D9B03F233421F9B23F4801343EA78
:10CC700002530793200742BF079B43F000430793EB
:10CC8000DDE906349B4604946BE43E4A0492222379
:10CC9000C9F800304FF0000B63E40A9B01931CAB12
:10CCA000029400933C4A1DAB1BA9484603F03EFD8D
:10CCB00010F0070504463FF450AC062D40F0938079
:10CCC000089B0137002B3FF463AB4FF0000B1F6054
:10CCD000CDF810B0FFF760BB6A1C012B1B9C9B4476
:10CCE000104615D02B4403F1FF3C03E04600944569
:10CCF0000DD001322B46082B154606EB8600F5D9E0
:10CD0000102ADCBF0AEB8A0A4FEA4A0AEFE7981CAE
:10CD1000082D5BDC0546FFF715BB04995A463846DB
:10CD2000FFF732FA002800F0888000231D460493A4
:10CD30009A461E46FFF751BB44F61F629042A8BFB9
:10CD400010460B90FFF7DBBBDDE906341194002C95
:10CD50007FF487AEBA465E4622234FF0000B1C9844
:10CD6000C9F80030CDF810B053E60B46CDE91623D4
:10CD700096E600BFAFF300809535A094FFFFCF3F4C
:10CD8000603701080000F07F0000A07CFFFFEF7F0C
:10CD90008837010808340108DC330108AD491BA8B5
:10CDA00003F0A2FF00283FF4EEAA1B9BAA49013B17
:10CDB0001BA81B9303F098FF10B91B9B01331B9317
:10CDC000A64B04934FF0000BFFF7CBBB1028DCBF42
:10CDD0000AEB8A0A01EB4A0A05460023FFF7B7BAB5
:10CDE0000023FFF7A1BA1C9A3AB135211EA804F01E
:10CDF00081FE1C99484604F0E7F9013D042D3FF6F9
:10CE000039AF01A353F825F05FCC000831CE0008FC
:10CE10002BCE00081DCE00085FCC00084FF0FF337A
:10CE20006FF00045CDE9063524E78C4B079321E7E9
:10CE30001E9B06931F9B07931CE71B9A13465A449D
:10CE40001B9213F80B4006468246FFF762BA0E9813
:10CE5000834901EBC001DDE90623D1E90001F4F7C4
:10CE6000AFFB83460491FFF77CBB04958346FFF735
:10CE700071BA7C4B7C4C109D0022CDE9182356E5FD
:10CE8000774CC5F10F0504EBC501DDE90623D1E9B7
:10CE90000001F4F795FB0E9B5D1B04EBC504D4E980
:10CEA0000023F4F78DFB83460491FFF75ABB109BD8
:10CEB0005E46D446BA46DDE90BB7002B6FD0DDE9FC
:10CEC00006456A4BC5F3130199422A463CD0002F10
:10CED00000F0A380DDE906231F421C4621D0109BF1
:10CEE00004995846002B00F0CD8004F0E9FC099D20
:10CEF00002460B467DB1C4F30A54C4F16B04002C06
:10CF000009DD240504F17F53002203F54013F4F7F3
:10CF100057FB02460B4604995846F3F7F7F9834648
:10CF20000491099B73B10499514B58460022F4F7C0
:10CF300047FB03460B4308BF22238346049108BFE7
:10CF4000C9F800301C9864E5099B0699002B00F095
:10CF5000C580424B2B40B3F1D46F00F2BF801B0D54
:10CF6000C3F16B034FF0FF3000FA03F39942AED1E7
:10CF7000404B9A4200F0D880384B134003F58013A1
:10CF8000079300230693DDE906349B460494C8E723
:10CF900002F15473079300230993FFF716BBDDE9F1
:10CFA0000612C2F313030B43144690D1099B002BC6
:10CFB00040F0AF80294B2340A3F580136FEA135351
:10CFC0006FEA035307934FF0FF33DBE7DDE9061207
:10CFD000109B0B4358465E46BA46DDF82CB0A0D1F4
:10CFE000C2F313031446002B9BD122F000431B0D08
:10CFF0001B05B3F1D66F94D9436913B90369012BAB
:10D000008FDD31460122484604F01CFB41460646AE
:10D0100004F090FB002884DDC8E7DDE906341CEA53
:10D02000030F3FF47EAF5AE713491BA81EAA03F073
:10D0300075FE05287FF48BAA1F9B43F0FF4343F442
:10D04000E00307931E9B0693DDE906349B46049498
:10D05000FFF787BACC330108D03301080000F07F16
:10D06000883701080000E0BF0000E03FFFFF0F002D
:10D0700000005039FFFFEF7FF033010809934FF0B4
:10D08000000A4EE504F01CFC099D02460B4695B3D0
:10D09000C4F30A54C4F16B04002C09DD240504F127
:10D0A0007F53109A03F54013F4F78AFA02460B46B1
:10D0B00004995846F3F728F9002200238346049187
:10D0C000F3F730FB00283FF42EAF45E64FF0FF3278
:10D0D00002FA03F3069A1A400692AFE54FF0FF33C7
:10D0E00044E74FF0FF33C2F14B0203FA02F202EAC7
:10D0F00001030793A2E504995846F3F705F90022C6
:10D10000002383460491F3F70DFB00283FF41AAF88
:10D1100022E6084B2340B3F1D66F3FF74DAFB3F192
:10D120005C7F3FF700AF17E601317FF425AFFFF7D3
:10D13000B2BB00BF0000F07F10B4044C044B844627
:10D140000A46206810BC6146FFF75EB82C00002438
:10D15000700800242DE9F04FD5B01C460791914688
:10D160000546099003F0B6FE0268179210460E9429
:10D17000F4F766F916901DB1AB6B002B00F02A8214
:10D18000079A536EDD0740F13881B2F90C2091B255
:10D190008F0409D4079B42F400529A8191B21A4637
:10D1A0005B6E23F4005353660E0740F1CB80079B60
:10D1B0001B69002B00F0C68001F01A030A2B00F057
:10D1C000CF8000242BAB4D46CDE92944CDE919444D
:10D1D000CDE91B44129428939846189400230B948D
:10D1E0000024CDE914342B78002B00F09D81AA4651
:10D1F00004E01AF8013F002B00F0C780252BF8D17E
:10D20000BAEB050640F0C5809AF80030002B00F01C
:10D210008B8100234FF0FF329AF801608DF8833044
:10D220000A930AF1010A08921F462B244FF02009A5
:10D230000AF1010AA6F120035A2B00F2ED80DFE883
:10D2400013F0EB02EB00EB00E602EB00EB00EB006F
:10D250006A00EB00EB005C028002EB0067028A02CE
:10D26000EB0085025B005B005B005B005B005B002A
:10D270005B005B005B00EB00EB00EB00EB00EB0006
:10D28000EB00EB007A01EB00F801D2017A017A01A0
:10D290007A01EB00EB00EB00EB00E102EB00EB00AE
:10D2A0002D02EB00EB00EB000202EB00A402EB000E
:10D2B000EB008307EB00EB00EB00EB00EB00EB0077
:10D2C000EB00EB007A01EB00F801D4017A017A015E
:10D2D0007A01C702D401CD01EB00D402EB006C024D
:10D2E0002F02B502CD01EB0002027E008007EB00A9
:10D2F000EB006107EB007E00A6F1300300221AF874
:10D30000016B02EB820203EB4202A6F13003092B10
:10D31000F5D90A928EE7DDF824B0584603F0DAFD1D
:10D3200043681B931846F4F78BF81C900646584642
:10D3300003F0D0FD83681993002E40F0CD869AF853
:10D34000006075E7079D0998294601F0C3FC002895
:10D3500041F01C83A98901F01A030A2B7FF431AF35
:10D36000079AB2F90E30002BFFF62BAF536ED80799
:10D3700002D4890541F13B810799099823464A4621
:10D3800055B0BDE8F04F01F04FBCBAEB050600F018
:10D39000CB802A9B33442A93299B0133072BC8E96E
:10D3A0000056299305DC08F108080B9B33440B93C6
:10D3B0002AE70799099828AA04F0BCFC80B90DF166
:10D3C000AC08F2E70799099828AA04F0B3FC0028F2
:10D3D00000F09B800D9B1BB10998194602F0B6FE28
:10D3E000079A536ED90740F1EA8093895B0601F1F1
:10D3F000D9820B9855B0BDE8F08F079BB3F90C208C
:10D40000900591B23FF5C4AE1D46986D03F06AFDDC
:10D41000B5F90C2091B2BBE6002E00F08580002209
:10D420008DF8EC608DF883200123CDE90C32069352
:10D4300008920F92139210923BAD17F0020302D0A4
:10D4400006990231069117F0840B07D10A990698C4
:10D45000A1EB0009B9F1000F00F370832A9C8AB197
:10D46000299A0DF1830101320134C8F80010072A0E
:10D470004FF001012A942992C8F8041000F3B683F2
:10D4800008F1080883B1299B21AA01330234C8F8A6
:10D490000020072B4FF002022A942993C8F8042099
:10D4A00000F3B28308F10808BBF1800F00F0698235
:10D4B000089B0C9AA3EB020BBBF1000F00F3AA82AE
:10D4C000FB0500F100820C9BC8F804301C44299B2A
:10D4D000C8F800500133072B2A94299300F32283C4
:10D4E00008F10808780705D50A9B069A9D1A002DB1
:10D4F00000F39683DDE90A2306998A42ACBF9B18A4
:10D500005B180B93002C7FF45DAF002329930D9BD8
:10D510001BB10D99099802F019FE0DF1AC085546A2
:10D520002B78002B7FF463AE2A9B002B41F0D38134
:10D530000023299354E70E9B073323F00702F2E8F8
:10D540000234CDE91434DDE9143424F000440E92A1
:10D55000994618462146B54B4FF0FF32F3F714F9C0
:10D56000002840F0EF84B14B484621464FF0FF328F
:10D57000F3F7ECF8002840F0E584DDE9140100221F
:10D580000023F3F7D9F8002840F067879DF883203F
:10D59000A74DA84B27F080070321472EC8BF1D4683
:10D5A00000230D9306910C9108930F9313931093FE
:10D5B000002A3FF442AF069B013306933DE7079BE9
:10D5C0009B899A053FF512AF079CA06D03F08CFC78
:10D5D000A3890BE7099802F0C1FCD1E59AF8006035
:10D5E00047F0200724E647F01007BA060E9B40F1EB
:10D5F0003B84073323F007031A465B6852F8084B55
:10D600000E929946002BC0F24C84089B013300F027
:10D61000D88254EA090327F0800B40F0D382089B9C
:10D62000002B40F0D4825F46002308930C9354AD46
:10D630001DE10E9B002253F8041B8DF883208DF80A
:10D64000EC100E93F0E60E9C089B54F8045B4FF030
:10D6500000098DF88390002D00F093855A1C00F08E
:10D6600051861A4649462846F3F75AFF0D9000287E
:10D6700001F00E810D9BCDF820905B1B0C930E9456
:10D6800023EAE3739DF883200693CDF83490CDF818
:10D690003C90CDF84C90CDF8409089E747F01007CA
:10D6A00017F0200900F0D2830E9B073323F0070305
:10D6B000D3F8049053F8084B0E9327F4806B0023A3
:10D6C00000228DF88320089A511C00F0B88054EA9B
:10D6D00009012BF0800740F0B180002A40F0F68568
:10D6E000002BA1D11BF001030C9300F01484302314
:10D6F0008DF84F310DF24F15B9E00E9B53F8042B06
:10D700000A92002A80F2DA830A9A0E9352420A920F
:10D710009AF8006047F004078AE5BD0600F1D1845D
:10D72000FC0600F1D885780600F1A586B90540F120
:10D73000D2850E9B0B9953F8042B0E93117055460E
:10D74000EEE69AF800608DF8834071E59AF8006083
:10D7500047F080076CE5524612F8016B2A2E01F063
:10D760003F82A6F13003092B924698BF002201F2B6
:10D77000BC801AF8016B02EB820203EB4202A6F1B5
:10D780003003092BF5D9089254E547F0100B1BF034
:10D79000200900F076830E9B073323F00703D3F8AC
:10D7A000049053F8084B0E93012389E70E9B53F81E
:10D7B000044B0E93302378268DF884301E4B18933B
:10D7C00047F0020B8DF885604FF00009022377E7E0
:10D7D0009AF80060682E03BF9AF8016047F400775A
:10D7E0000AF1010A47F0400722E59AF800606C2E22
:10D7F00003BF9AF8016047F020070AF1010A47F0D9
:10D80000100715E59AF8006047F0080710E59AF848
:10D81000006047F001070BE59DF88330002B7FF493
:10D820008EAD9AF800608DF8839001E5FFFFEF7FE1
:10D83000303401083434010840340108BB46012B60
:10D8400000F0C081022B54AD20D1189A04F00F03D0
:10D850002409D35C05F8013D44EA09744FEA19191B
:10D8600054EA0903F2D154AB5B1B5F460C93089951
:10D870000C989DF8832081424FF00003B8BF014609
:10D880000D9306910F931393109391E604F0070301
:10D89000E40844EA49744FEAD909303354EA0901EB
:10D8A0002A4605F8013DF1D11BF0010FDBD0302BEA
:10D8B000D9D03023023A05F8013C54AB9B1A5F469D
:10D8C0000C931546D3E7652E40F3E680DDE914019D
:10D8D00000220023F2F726FF002800F0DC81299BBC
:10D8E000BF4AC8F80020013301340122072B2A94D3
:10D8F0002993C8F8042000F3CC8408F10808229B7F
:10D90000129A934280F2D682169B179A1C44C8E959
:10D910000023299B2A940133072B299300F32484A5
:10D9200008F10808129B5D1E002D7FF7DBAD102D5E
:10D93000299BDFF8B09240F3BD8449462246B946A0
:10D94000DDF824B0079C10260F4605E008F1080812
:10D95000103D102D40F3AA8401331032072BC8E983
:10D960000076CDE92932F1DD28AA2146584604F097
:10D97000E1F900287FF42EADDDE929320DF1AC0884
:10D98000E6E70A9B069AA3EB020BBBF1000F7FF7B9
:10D990008FADBBF1100F299ADFF848922CDD1D9650
:10D9A00021464E46079CDDF82490102306E0ABF19B
:10D9B000100BBBF1100F08F108081ADD013210310D
:10D9C000072AC8E90063CDE92921F0DD28AA21460C
:10D9D00048460DF1AC0804F0ADF900287FF4FAAC2C
:10D9E000ABF1100BBBF1100FDDE929214FF0100353
:10D9F000E4DCB1461D9E0C4601325C44072ACDE9A9
:10DA00002924C8F80090C8F804B000F3A08308F1F6
:10DA100008084DE5BBF1100F299ADFF8C8912DDDFC
:10DA200041462046A8464C46079DDDF82490102329
:10DA300006E0ABF1100BBBF1100F01F1080119DD8D
:10DA400001321030072AC1E90043CDE92920F0DD79
:10DA500028AA2946484604F06DF900287FF4BAAC9C
:10DA6000ABF1100BBBF1100FDDE929202BA94FF012
:10DA70001003E5DC4546A1468846044601325C4475
:10DA8000072ACDE92924C8F80090C8F804B000F3AB
:10DA9000D08108F1080813E5129B012B40F3808127
:10DAA000299EC8F80050013601340123072E2A941C
:10DAB0002996C8F8043000F37C8308F10808169B07
:10DAC000179A01361C44072EC8E90023CDE92964C2
:10DAD00000F37C8308F10808DDE91401002200232B
:10DAE000F2F720FE002840F07881129B0136013BBE
:10DAF00001351C44072EC8F800502996C8F8043098
:10DB00002A9400F35D8108F108081A9BC8F80430D4
:10DB100001361C44072E24ABCDE92964C8F8003037
:10DB20007FF7DEAC0799099828AA04F003F90028CA
:10DB30007FF450AC2A9C0DF1AC08D3E4B9F1100F7E
:10DB4000DDE929212BDDCDE91D3B1F96DDF824B051
:10DB50004E461024A946079D04E0103E102E08F101
:10DB6000080817DD0132204B1031072AC8E90034BC
:10DB7000CDE92921F1DD28AA294658460DF1AC0846
:10DB800004F0D8F800287FF425AC103E102EDDE913
:10DB90002921E7DCDDE91D3B4D46B1461F9EC8F853
:10DBA0000490013209EB0104072A0F49C8F800105C
:10DBB000CDE9292400F351839DF8832008F108085A
:10DBC0004DE4BB460A2C79F1000380F00C8330341D
:10DBD00001238DF84F415F460C930DF24F1546E639
:10DBE00070340108843401087434010807990998D5
:10DBF0001D9328AA04F09EF800287FF4EBAB2A9C22
:10DC00001D9B0DF1AC083DE40799099828AA04F082
:10DC100091F800287FF4DEAB2A9C0DF1AC0843E4B8
:10DC2000102D299B21DD099FDDF81C90102604E0B2
:10DC3000103D102D08F1080817DD0133BB4A1034E0
:10DC4000072BC8E90026CDE92934F1DD28AA494689
:10DC500038460DF1AC0804F06DF800287FF4BAAB3B
:10DC6000103D102DDDE92934E7DC0133AF4AC8F857
:10DC700004502C44072BCDE92934C8F800207FF745
:10DC800039AC0799099828AA04F054F800287FF4C1
:10DC9000A1AB2A9C2EE42299002940F31481DDF8DF
:10DCA0004090129B9945A8BF9946B9F1000F0BDD32
:10DCB000299B01334C44072BC8E900592A94299326
:10DCC00000F39A8508F10808109EB9F1000FA8BF6B
:10DCD000A6EB0906002E00F34683DDF840B0790577
:10DCE000AB4400F1CE84229B129A934202DBFA07E6
:10DCF00040F1B883169A17991444C8E90012299A7A
:10DD00002A940132072A299200F3838508F1080832
:10DD1000129AAE18A6EB0B06D51AAE42A8BF2E4635
:10DD2000002E0DDD299BC8F800B001333444072BC9
:10DD3000C8F804602A94299300F3F18508F10808D3
:10DD4000002EA8BFAD1B002D7FF7CCAB102D299B5B
:10DD5000DFF8DC9140F3AE8249462246B946DDF851
:10DD600024B0079C10260F4605E008F10808103D76
:10DD7000102D40F39B8201331032072BC8E9007647
:10DD8000CDE92932F1DD28AA2146584603F0D2FF19
:10DD900000287FF41FABDDE929320DF1AC08E6E77E
:10DDA000FE073FF57DAE299EC8F8005001360134CC
:10DDB0000123072E2A942996C8F804307FF7A3AED2
:10DDC0000799099828AA03F0B5FF00287FF402AB51
:10DDD000DDE929640DF1AC0897E6129B5D1E002D6C
:10DDE0007FF793AE102DDFF8489140F37F822246F3
:10DDF0000897099C079F4FF0100B05E008F10808F1
:10DE0000103D102D40F3708201361032072EC8E904
:10DE1000009BCDE92962F1DD28AA3946204603F0AE
:10DE200089FF00287FF4D6AADDE929620DF1AC084C
:10DE3000E6E70799099828AA03F07CFF00287FF4F9
:10DE4000C9AA2A9C0DF1AC08FFF73ABB17F01003E2
:10DE500072D117F0400200F0BD820E9A52F8044BC6
:10DE60000E929946A4B228E453F8044B0E93FB0695
:10DE700056D47D0651D544F3C0394B4624B2FFF742
:10DE8000C1BB1BF0100340F036811BF0400200F0D4
:10DE900092820E9A52F8044B0E929946A4B2012334
:10DEA0000EE42D2364428DF8833069EB4909BB46AB
:10DEB000012308E4F8077FF515AB25E59AF8006023
:10DEC0000E93FFF7B5B9299B1A4AC8F80020013311
:10DED00001340122072B2A942993C8F8042000F367
:10DEE000708408F10808002940F01E82129A07F099
:10DEF000010313433FF4F6AA169B1799E218C8E9E9
:10DF00000013299B2A920133072B299300F3618385
:10DF100008F1080819E254ADA9E4B80500F1B4828B
:10DF20004FEAE4794B46FFF76DBB00BF743401083C
:10DF300084340108703401080E9B53F8044B0E938F
:10DF4000FFF7BBBBDDE9140102460B46F2F71CFCF0
:10DF5000002840F0A085612E00F05085412E00F091
:10DF60009982089B013326F02003069300F08F85E9
:10DF7000472B00F07985DDE9141247F480730F9385
:10DF80001346002BC0F2ED850C9300231D938B46A6
:10DF90000D93069B462B00F04A84452B00F04F85DD
:10DFA0000899019126A9049123A9039122A902911C
:10DFB00002210C9B099800915A4600F0A9FF069B8C
:10DFC000472B054640F01C8617F0010FB9460F9FFE
:10DFD00040F0D984269B5B1B1293069B472B00F0D5
:10DFE0001883069B462B00F05F84229B1093109BA6
:10DFF000069A013B412A229300F0AA85F2B2002141
:10E00000002BB8BF109B8DF89020BABFC3F101035D
:10E010002D222B22092B8DF8912040F363850DF1E1
:10E020009F04BD4F2246104687FB0321DA17C2EB3F
:10E03000A10202EB8201A3EB4101303100F8011C87
:10E0400019466329134600F1FF32ECDC3033D9B2B4
:10E05000831E9C4202F8011C40F2CE8513460DF14E
:10E06000920201E013F8011B02F8011B9C42F9D156
:10E070000DF1A1030DF192021B1A134424AA9B1A5D
:10E080001A93129B1A9A012B1A440C9240F3728530
:10E090000C9B169A13440C930C9A002329F4806766
:10E0A00022EAE27247F480770F930692139310935B
:10E0B0001D9B002B40F0DE829DF883200893FFF724
:10E0C00077BA0E9B0B9853F8041B0E93C217C1E945
:10E0D00000025546FFF724BA199B002B3FF42FA9E5
:10E0E000199B1B78002B3FF42AA99AF8006047F48B
:10E0F0008067FFF79DB80E9B53F8044B0E930123E6
:10E10000FFF7DEBA854B189317F0200949D00E9B14
:10E11000073323F00703D3F8049053F8084B0E930A
:10E12000F80709D554EA090306D030238DF8856035
:10E1300047F002078DF8843027F4806B0223FFF745
:10E14000BFBABB46FFF723BB754B1893DCE70799B3
:10E15000099828AA03F0EEFD00287FF43BA92A9C29
:10E160000DF1AC08FFF7A4B90799099828AA03F0A4
:10E17000E1FD00287FF42EA92A9C0DF1AC08FFF7E1
:10E18000D1BB062B294628BF062308950D952A46A4
:10E190000693644D0E940C930F9113911091FFF719
:10E1A00007BA17F0100369D00E9B53F8044B0E9377
:10E1B000B6E70799099828AA03F0BCFD00287FF468
:10E1C00009A9DDE929640DF1AC0878E407990998FB
:10E1D00028AA03F0AFFD00287FF4FCA8DDE929643C
:10E1E0000DF1AC0878E40BF480630022CDE90CA8B3
:10E1F0000696DDF8648054AF16469A460CE000237C
:10E20000204649460A22F2F77BFD0A2C79F10003E9
:10E210001BD3044689462F4620460A22002349463E
:10E22000F2F76EFD30327D1E013607F8012CBAF18F
:10E23000000FE4D098F800309E42E0D1FF2EDED0EF
:10E240000A2C79F1000380F0F480CDF864801296F6
:10E25000DDE90CA8069EFFF706BB079909981D93F8
:10E2600028AA03F067FD00287FF4B4A89DF8832056
:10E270002A9C1D9B0DF1AC08FFF7F1B817F0400286
:10E2800000F0B6800E9A52F8044B0E929946A4B252
:10E2900046E70799099828AA03F04CFD00287FF467
:10E2A00099A82A9C0DF1AC08FFF729BB14463A4601
:10E2B0004F46914601332C44072BC8F80090C8F80C
:10E2C0000450CDE929347FF70BA92BE4012BBB4681
:10E2D0007FF4B8AA7BE40E9B0B9953F8042B5546A8
:10E2E00011600E93FFF71CB9089F144601362C44A9
:10E2F000072ECDE92964C8F80090C8F804507FF7CC
:10E3000002AC5DE52846CDF820900E94F3F798F81E
:10E3100003460C90FFF7B4B967666666403401089F
:10E320005434010868340108169B1798E218C8E9AC
:10E330000003299B2A920133072B299300F349817B
:10E3400008F108080029C0F2FA821299C8F80050B2
:10E3500001338C18072BCDE92934C8F804107FF756
:10E36000BFA8FFF7DFBB102E299BDFF8C09252DD5C
:10E37000484642462146A846B946099C079D4FF0AB
:10E38000100B074603E00832103E102E3DDD01332E
:10E390001031072BC2E9007BCDE92931F3DD28AA32
:10E3A0002946204603F0C6FC00287FF413A8DDE9C7
:10E3B00029312BAAE8E70E9B1BF4007914BF53F810
:10E3C000044B53F8044B0E931CBF9146E4B2012357
:10E3D000FFF776B90E9B17F4007914BF53F8044B7E
:10E3E00053F8044B0E931CBF9146E4B2FFF765B996
:10E3F0000E9B17F4007914BF53F8044B53F8044BE9
:10E400000E931CBF9146E4B28AE6454690463A46D2
:10E410000C464F46914601333444072BCDE929344D
:10E42000C8F80090C8F8046000F3E68008F1080816
:10E4300053E41C9B1B99ED1A1A46284603F00CFC6A
:10E4400098F801300BB108F10108204649460A222C
:10E4500000230026F2F754FCDBE62D228DF8832002
:10E46000FFF796B8129AAE18A6EB0B06D51AAE4275
:10E47000A8BF2E4664E40E9B0B9953F8042B0E9311
:10E4800011805546FFF74CB844F3C0194B4664B2AF
:10E49000FFF7B8B830238DF8843058238DF88530D5
:10E4A000089B632B47F0020400F39B8200230D932B
:10E4B0003BADDDE9141247F481730F931346002B33
:10E4C0002746C0F220820C9326F0200306930023F7
:10E4D0008B461D93612E00F0ED82412E7FF459ADE5
:10E4E00022AA0C99584603F079FB00224FF07F5383
:10E4F000F3F766F802460B46CDE91023002200230D
:10E50000F2F710F908B101232293494B0C93089BB1
:10E51000CDE912A6CDE91E78DDF830A0DDE910675F
:10E5200003F1FF39AB46109506E00022002309F104
:10E53000FF39F2F7F7F8E8B93E4B0022304639468A
:10E54000F3F73EF80F460646F2F734F90446F2F7C1
:10E5500029F80B46024639463046F1F7D5FE1AF83F
:10E560000430B9F1FF3FD8464D460BF8013B064653
:10E570000F46DAD1304639462F4BDDF848A0139EBE
:10E58000CDF848800022A946DDF87C80109D1E9FB2
:10E59000CDE91001F2F7EEF8002840F03482DDE911
:10E5A0001001254B0022F2F7BDF810B1E10700F190
:10E5B0002A824B46002B06DB01335B4430220BF8EA
:10E5C000012B5B45FBD1ABEB0503B94612930F9FC3
:10E5D00003E50799099828AA03F0ACFB00287EF40C
:10E5E000F9AEDDE9293222990DF1AC08AAE6906D69
:10E5F00002F07AFCFEF7C0BE0799099828AA03F03A
:10E6000099FB00287EF4E6AE2A9C0DF1AC08FFF7DA
:10E6100064BB229B1093DA1C02DB089A93420DDD47
:10E62000023E26F020030693E1E400BF8434010893
:10E6300054340108000030400000E03F109B129A63
:10E640009342C0F2568119F0010F00F08782169AAA
:10E6500013440C9319F4806F03D0109B002B00F32C
:10E6600050820C9B23EAE3730693672600230F93E3
:10E6700013931DE52D2200238DF883200893FEF7C8
:10E680009ABF129BCDF830A04246DDF84C8010971F
:10E69000EB1808935E46199FDDF87090DDF824A012
:10E6A000DDF81CB00F9B13952146B8F1000F2ED05A
:10E6B000002B6BD1013F08F1FF381B9BC2E90039E9
:10E6C000299B01334944072B2A91299362DC0832A4
:10E6D000089B38789B1B8342A8BF0346002B1C462F
:10E6E0000ADD2998013019440728C2E900632A91FC
:10E6F00029905ADC38780832002CACBF051B05463F
:10E70000002D15DC06440F9BB8F1000FD0D1002B73
:10E710003CD1DDE91235EB189E421997B346DDF87E
:10E7200030A0109F90460C4628BF9B46FFF7DBBAEF
:10E73000102D29981DDD102404E0103D102D02F14C
:10E74000080216DD0130AC4B10310728C2E9003455
:10E75000CDE92901F1DD28AA5946504603F0EAFA2D
:10E7600000287EF437AE103D102DDDE929012BAADB
:10E77000E8DC0130A04B556029440728CDE9290188
:10E7800013602CDC387808320644BCE70F9B013B51
:10E790000F9392E728AA5946504603F0CBFA002877
:10E7A0007EF418AE2A992BAA92E728AA5946504619
:10E7B00003F0C0FA00287EF40DAE38782A992BAA0F
:10E7C0009AE70799099828AA03F0B4FA00287EF47A
:10E7D00001AE22992A9C0DF1AC08FFF784BB28AA50
:10E7E0005946504603F0A6FA00287EF4F3AD387877
:10E7F0002A992BAA064486E70799099828AA03F0C4
:10E8000099FA00287EF4E6AD2A9C0DF1AC08FFF7DA
:10E810005BBA0799099828AA03F08CFA00287EF4BD
:10E82000D9AD229B2A9C0DF1AC08FFF771BA08996B
:10E83000019126A9049123A9039122A90291032100
:10E840000C9B099800915A4600F062FB0378302B2C
:10E85000054600F09581229B089AB94613440F9F04
:10E86000EC180C99584600220023F1F75BFF10B119
:10E870002346FFF7B0BB269BA342BFF4ACAB3021CD
:10E880005A1C26921970269B9C42F9D8FFF7A3BB0D
:10E89000089B9DF883200E9406930C9308900F908C
:10E8A00013901090FEF784BE229A1092002A40F333
:10E8B0008181089909F001030B4340F05581109BB9
:10E8C0000C93662619F4806F40F01C810C9B23EAA0
:10E8D000E3730693CAE60799099828AA03F02AFA6F
:10E8E00000283EF425AEFEF77BBD00230893FEF71B
:10E8F000A1BC129B169A9A18109B0C92002B40F305
:10E900004D816726DEE726F020030693DDE9143407
:10E910009B4604F100430C932D231D93DAE50799E0
:10E92000099828AA03F006FA00287EF453AD229D28
:10E93000129B2A9C5D1B0DF1AC08FFF701BA4E42F9
:10E940001031DFF8B49034DA4146DDF824B0A8463F
:10E950001024079D03E00831103E102E27DD0133FF
:10E960001032072BC1E90094CDE92932F3DD28AA42
:10E970002946584603F0DEF900287EF42BADDDE988
:10E9800029322BA9E8E7089BEC186AE7079B5B6E26
:10E99000DD0707D4079B9B899C0503D4079B986DD3
:10E9A00002F0A2FA4FF0FF330B93FEF722BD45466B
:10E9B000884601333244072BCDE92932C8F800904C
:10E9C000C8F804607FF7A4AA0799099828AA03F059
:10E9D000B1F900287EF4FEACDDE929320DF1AC0876
:10E9E000B3E40998591CFCF72FFD0546002800F0F8
:10E9F0000D810D905DE500BF8434010830238DF852
:10EA0000843078234AE5129B26930C9B1BF8012C3B
:10EA1000D97B8A425B4609D1302003F8010C269B42
:10EA20005A1E269213F8012C9142F6D0392A0BBFB8
:10EA30000C9A0132927AD2B203F8012CC3E50899FC
:10EA40000C9B09984C1C26A9049123A9039122A987
:10EA5000029102215A460194009100F059FA0546AC
:10EA6000B9462C440F9FFCE6089B002B08BF0123EE
:10EA7000089347F480730F93159B002BC0F2AE8070
:10EA8000DDF850B01D900C930D90FFF789BA062366
:10EA90000893FFF770BA159B604D002BB4BF2D2271
:10EAA0009DF883205E4BB8BF8DF8832027F0800748
:10EAB000FEF772BD22AA0C99584603F08FF8002287
:10EAC0004FF07F53F2F77CFD02460B46CDE9102351
:10EAD00000220023F1F726FE08B101232293514BB7
:10EAE0000C9314E5002962D130228DF892200DF1AB
:10EAF0009302303302F8013B24ABD31A1A93FFF789
:10EB0000C0BA672619990B78FF2B7BD00024109A86
:10EB1000204603E001300131FF2B08D0934206DA92
:10EB2000D21A4B78002BF5D10B780134F4E7199108
:10EB3000109213900F940F9A139B1C9913440C9AE4
:10EB400001FB03230C9323EAE3730693FFF7B0BAA8
:10EB500006F10F02D2B20121FFF752BA109B0C93BB
:10EB600078E500230D93D1E6169BD31819440C9138
:10EB70006626A7E619F0010F3FF48EAAFFF788BAC0
:10EB80000C99584600220023F1F7CCFD00287FF4B1
:10EB900062AE089BC3F1010322935DE6C3F101035A
:10EBA0001A4422EAE2730C92069367265EE50DF1A1
:10EBB00092029EE7089A09F0010959EA020304D17A
:10EBC0000123069366260C9350E5169B01331A44E5
:10EBD00022EAE2730C920693662647E50D9095E6CD
:10EBE0000E9B9AF80160924653F8042B0E9342EA6A
:10EBF000E2720892FEF71CBB02231A93FFF741BA98
:10EC0000089C2DE700230F93139394E7079A9389A9
:10EC100043F040039381FEF7E3BB00BF38340108A3
:10EC20003C34010840340108F0B51F468B89ADF231
:10EC30006C4D23F00203ADF80C304B6E1993CB8969
:10EC4000ADF80E30CB6907934B6A09931AAB00936A
:10EC500004934FF48063154606460293059316A865
:10EC600000230C46069302F039F92A463B466946D2
:10EC70003046FEF76FFA051E07DB6946304601F0A5
:10EC800039F9002818BF4FF0FF35BDF80C305B068E
:10EC900003D5A38943F04003A381169802F020F91D
:10ECA00028460DF26C4DF0BD38B50C46084D844633
:10ECB000114620461A4600232B606446F4F704F9F7
:10ECC000431C00D038BD2B68002BFBD0236038BD1F
:10ECD000582B002438B5334B1B6805460C460BB146
:10ECE0009A6B12B3B4F90C3018079AB225D5216982
:10ECF00000292DD012F0010007D00020A06060692B
:10ED00004042A06139B1002038BD950758BF606905
:10ED1000A0600029F7D1120658BF0846F4D543F089
:10ED20004003A3814FF0FF3038BD184601F016F9BB
:10ED3000B4F90C3018079AB2D9D4D1062AD55207A3
:10ED400014D4216943F00803A3819AB20029D1D1D8
:10ED500002F42070B0F5007FCCD02146284602F0A6
:10ED6000DBF8B4F90C3021699AB2C3E7216B51B1D9
:10ED700004F14002914204D0284601F0E7F9B4F9C9
:10ED80000C300022226321690022C4E9001223F022
:10ED90002403D7E7092243F040032A604FF0FF30F5
:10EDA000A38138BD2C000024024B13B1024800F0AF
:10EDB00005B87047000000008100010800230146EB
:10EDC0001A46184603F0DEBE38B5074D0022044649
:10EDD00008462A60F4F792F8431C00D038BD2B682F
:10EDE000002BFBD0236038BD582B00242DE9F04FB9
:10EDF00003690C69A34283B0C0F28680013C01F133
:10EE00001405A30000F11408009355F8243058F8B5
:10EE1000242001338A469A4208EB8401814605EB9F
:10EE200084070191B2FBF3F638D30023AE46404687
:10EE30009B465EF8041B02681FFA81FC06FB0C333C
:10EE4000090C4FEA134C06FB01CC99B2ABEB010164
:10EE50001FFA8CF311FA82F1C3EB124202EB21424A
:10EE600089B241EA0241774540F8041B4FEA1C434E
:10EE70004FEA224BDDD2009B58F8033073B9019B57
:10EE8000043B984504D307E0984504F1FF3403D2CE
:10EE900053F80429002AF7D0C9F8104051464846D3
:10EEA00002F048FC00282BDB01364046002355F8D1
:10EEB000041BD0F800C08AB29A1A0B0C12FA8CF21A
:10EEC000C3EB1C4303EB224392B242EA0342AF423C
:10EED00040F8042B4FEA2343E9D258F8242008EBEA
:10EEE00084036AB9043B984504D307E0984504F1CC
:10EEF000FF3403D253F80429002AF7D0C9F8104090
:10EF0000304603B0BDE8F08F002003B0BDE8F08FBD
:10EF10002DE9F04F016C99B090469946CDE90489EE
:10EF2000259D044641B1426C4A60012393408B60A9
:10EF300002F04AF900232364B9F1000AB4BF0123A7
:10EF400000232B60764BBCBF2AF0004ACDF814A0FA
:10EF500033EA0A0300F0AA80DDE9042310461946CB
:10EF600000220023CDE90A01F1F7DCFB074670B16E
:10EF7000249A01231360269B002B00F0E482694849
:10EF80001860431E0393039819B0BDE8F08F16ABC9
:10EF9000019317AB00932046DDE90A2302F01AFD26
:10EFA0005FEA1A56054640F09780DDE916763E4442
:10EFB00006F23240202840F3B583C0F140000AFA3F
:10EFC00000FA06F2124028FA00F04AEA0000F1F7CF
:10EFD000D9FA0123013EA1F1F8710F93524B00229F
:10EFE000F1F792F948A3D3E90023F2F7E9FA48A32D
:10EFF000D3E90023F1F78AF9804630468946F1F7D4
:10F00000D1FA45A3D3E90023F2F7DAFA02460B4618
:10F0100040464946F1F77AF980468946F1F7CAFB3E
:10F0200000228346002340464946F1F785FB00282D
:10F0300040F07C82BBF1160F00F26B823B4B03EB7E
:10F04000CB03D3E90023DDE90A01F1F775FB0028C2
:10F0500072D00023BE1B0E93731E0BF1FF3B069371
:10F0600000F15E8200230993BBF1000F6BDA099B6C
:10F07000CDF81CB0A3EB0B030993CBF100030D9368
:10F08000229B092B4FF0000B66D8052B40F34883D9
:10F09000043B22930026229B023B032B00F268864E
:10F0A000DFE813F05C04590450043304249A42F25C
:10F0B0000F73CAF3130A13605AEA08031AD1269B86
:10F0C000002B00F064861A4B03930833269A0398AA
:10F0D000136019B0BDE8F08FDDE90A12C2F3130323
:10F0E000084643F07F510F97A6F2FF36169F41F472
:10F0F000401173E7269B002B40F0EA830D4B0393EE
:10F1000041E700BFAFF3008061436F63A787D23F41
:10F11000B3C8608B288AC63FFB799F501344D33F06
:10F120000000F07F713401080000F83F88370108C3
:10F130009834010894340108BE1B731E069300F135
:10F1400085840E900990069B5B44CDE9063B002325
:10F150000D93229B092B98D90023CDE92233012658
:10F160004FF0FF330C960893089B129300216164C3
:10F17000204602F003F80390002800F00186039B6C
:10F180002364089B0E2B00F21381002E00F01081E7
:10F190000799002940F35C84AE4B01F00F0203EBAA
:10F1A000C2034FEA2118C905D3E9006740F114846E
:10F1B000A94BDDE90A01D3E90823F2F72BFBCDE9DE
:10F1C000100108F00F084FF0030AB8F1000F13D038
:10F1D000DFF8849218F0010F09D030463946D9E99A
:10F1E0000023F2F7EDF90AF1010A06460F465FEA3D
:10F1F000680809F10809EDD1DDE9100132463B4606
:10F20000F2F708FB804689460E9B43B1934B0022E0
:10F2100040464946F1F790FA002840F030855046C4
:10F22000F1F7C0F942464B46F2F7CAF98C4B00227F
:10F23000F1F76CF8A1F15073CDE910011193089B1F
:10F24000002B00F09780079B1493089B13930C9B53
:10F25000002B00F0A584139A7E4B8249039E03EB9A
:10F26000C20353E902230020F2F7D4FADDE91023A8
:10F27000F1F74AF8CDE9100149464046F1F79AFA0C
:10F280000746F1F78FF902460B4640464946F1F72B
:10F290003BF83037DDE9102306F8017B80468946CC
:10F2A000F1F74AFA002840F02985CDF854B000273C
:10F2B000DDE910AB1095139D13942AE00137AF429E
:10F2C00080F22C85684B504659460022F2F778F9B7
:10F2D000654B002282468B4640464946F2F770F95C
:10F2E00089468046F1F766FA0446F1F75BF9024673
:10F2F0000B4640464946F1F707F8303406F8014B13
:10F3000052465B4680468946F1F716FA002840F0DF
:10F31000F38442464B4651490020F0F7F5FF524630
:10F320005B46F1F709FA0028C8D0DDE91343109DC8
:10F33000039A079302E0964200F0C884B24616F89A
:10F34000013D392BF7D00133DBB23370079B01331A
:10F350000793C8E15046F1F725F942464B46F2F7CC
:10F360002FF93F4B0022F0F7D1FFA1F15073CDE907
:10F37000100111933D4B404649460022F0F7C4FF6F
:10F38000DDE910894B46424606460F46F1F7F2F991
:10F390008146002840F0AA84DDE91001024601F10F
:10F3A000004330463946F1F7C7F9002840F045835D
:10F3B000179B002BC0F28C80079A0E2A00F38880DE
:10F3C000244B03EBC203D3E900AB239B002B1BDAD6
:10F3D000089B002B18DC40F02E83244B0022504663
:10F3E0005946F2F7EDF802460B46DDE90A01F1F75E
:10F3F000ADF9DDF820904E46002800F0C782239B2F
:10F40000DDF80C80DF43C9E2DDE90A7852465B464D
:10F4100038464146F2F7FEF9F1F7CCF981460990FA
:10F42000F1F7C0F852465B46F2F7CAF8039E0B4666
:10F43000024641463846F0F767FF09F1300306F807
:10F44000013B089B012B00F05C8306940127049587
:10F450001C462AE088370108603701080000F03FA9
:10F4600000001C400000E03F000024400000144069
:10F4700052465B4640464946F2F7CCF9F1F79AF915
:10F480000546F1F78FF852465B46F2F799F80137D7
:10F490000B46024649464046F0F736FF05F1300379
:10F4A000A74206F8013B00F02983AC4B0022F2F79B
:10F4B00087F80022002380468946F1F733F90028B7
:10F4C000D6D0049D069C079B01330793B2460AE100
:10F4D0000C9A002A3DD0229A012A40F39C82089B74
:10F4E00003F1FF380D9B4345C0F26D82A3EB080882
:10F4F000089B002BC0F23C83069A1A440692099A94
:10F5000017461A4409920121204601F05FFF064682
:10F5100023E00123BE1B0E93731E06937FF5A2AD5D
:10F52000C6F101030993002306939DE55846F1F7C0
:10F5300039F842464B46F1F7F5F800287FF47AADEA
:10F540000BF1FF3B76E5864B0393039819B0BDE8BA
:10F55000F08FDDF83480099F0C9E002F0CDD06999A
:10F5600000290B4608DD099AB942A8BF3B46D21ACA
:10F57000FF1ACB1A099206930D9BDBB10C9B002B53
:10F5800000F05D82B8F1000F0FDD314642462046A3
:10F5900001F0F8FF2A4601460646204601F044FFE6
:10F5A00029460546204601F00FFE0D9BB3EB0802ED
:10F5B00040F0D8820121204601F008FFBBF1000F86
:10F5C000814600F3B480229B012B40F386814FF0EB
:10F5D000000A0120BBF1000F40F0B580069A1044EC
:10F5E00010F01F0000F09380C0F12003042B40F3C3
:10F5F000D283099BC0F11C000344024409930744D1
:10F600000692099B002B05DD29461A46204602F08A
:10F6100019F80546069B002B05DD49461A4620468B
:10F6200002F010F881460E9B002B40F03681089BBB
:10F63000002B40F31D810C9B002B40F0A080079B0A
:10F6400001330793DDF80C80DDF820A0012707E0E7
:10F65000294600230A22204601F0C0FD0137054655
:10F6600049462846FFF7C2FB574500F1300308F82A
:10F67000013BEDDB089A002AC8BF9346039AD8BF26
:10F680004FF0010B934400272946012220460493A2
:10F6900001F0D8FF4946054602F04CF8002840F337
:10F6A000A8811BF8013C039A0BF1FF3B04E05A458B
:10F6B00000F0AA811BF8013D392B0BF1010AF6D0AD
:10F6C00001338BF800304946204601F07DFD56B1EC
:10F6D0002FB1B74203D03946204601F075FD3146BF
:10F6E000204601F071FD2946204601F06DFD002302
:10F6F0008AF80030249B079A1A60269B002B3FF45F
:10F7000042AC0398C3F800A019B0BDE8F08F1C20EC
:10F71000099B03440993069B03440744069370E73F
:10F720000126B8E4C0F1200008FA00F04FE40146D9
:10F730005A46204601F026FF229B012B814640F3CA
:10F74000B3814FF0000AD9F8103009EB8303186930
:10F7500001F0EEFDC0F1200040E700BF00002440B2
:10F7600070340108314600230A22204601F036FD9C
:10F77000129B002B064640F3E782CDE90783002F5A
:10F7800000F31A81BAF1000F40F0D581B046049B16
:10F79000039F089903F001027B1E1944229B0C92DF
:10F7A000134309910A9349462846FFF71FFB314648
:10F7B0008346284601F0BEFF42464946824620461F
:10F7C00001F0D8FFC26801460BF13003002A42D194
:10F7D00006902846089301F0ADFF06990490204654
:10F7E00001F0F2FC049A089B1AB90A99002900F06A
:10F7F0009B82BAF1000FC0F2638122994AEA010AA2
:10F800000C9951EA0A0100F05B81002A00F3B481EF
:10F81000099A3B7007F1010A9742D34600F0B28182
:10F82000294600230A22204601F0D8FC4645054619
:10F8300031464FF000034FF00A02204612D001F08B
:10F84000CDFC4146064600230A22204601F0C6FCB4
:10F8500057468046A7E72046049301F0B5FC049B79
:10F860000122C6E701F0BAFC5746064680469AE7F1
:10F87000229B022B79DC0C9B002B80D1079B4946F5
:10F88000013328460793FFF7B1FADDF80CB000F119
:10F8900030030BF8013B0027F6E64946284601F005
:10F8A00049FF0028BFF6C3AE294600230A2220469E
:10F8B00001F094FC079B03F1FF380C9B0546002BDD
:10F8C0007FF450AF129B002B40F335820893B9E6CA
:10F8D000AF4B03930333FFF7F9BBDDE904120029B3
:10F8E0007FF475AEC2F31303002B7FF470AEA94B07
:10F8F0001340002B00F0FE81099B01330993069B06
:10F90000013306934FF0010A63E601230C93239B16
:10F91000079A134412930133012B1F460893B8BF73
:10F9200001270021172F61647FF722AC01220423F5
:10F930005B0003F11400B842114602F10102F7D94D
:10F94000616415E401230C93239B002B4CDD12937F
:10F9500008931F46E5E700230C93D8E700230C9398
:10F96000F2E7129BCDF81C800893089B002B7FF4D4
:10F9700046AD49460522204601F030FC014681464D
:10F98000284601F0D7FE00287FF739AD0398079F7E
:10F990003123804600F8013B013703904946204659
:10F9A00001F012FC7B1CDDF80CA00793CDF80C8055
:10F9B000002E7FF494AE96E631463A46204601F09A
:10F9C00041FE0646DEE60D9BCDF83480A8EB03032E
:10F9D0009B444FF000088BE5DDE90A234FF0020A53
:10F9E000CDE91023FFF7F1BB012323930893FFF721
:10F9F000BBBB03D1049BDB073FF553AEDA461BF8D4
:10FA0000013D302BFAD05EE6079B039A0133079342
:10FA10003123137057E60F9A002A00F0268103F273
:10FA20003343069ADDF834801A440692099A174641
:10FA30001A44099267E54FF000094E46DFE4294673
:10FA40000D9A204601F09EFD0546B3E50E9067E550
:10FA500000F00F81079A504B564206F00F0203EB5D
:10FA6000C203D3E90023DDE90A01F1F7A9FD36114C
:10FA70008046894600F07181484F00234FF0020A0A
:10FA8000F20706D5D7E90023F1F79AFD0AF1010A3A
:10FA90000123761007F10807F2D1002B3FF4B4AB35
:10FAA00080468946FFF7B0BB049B002B7FF449AE2C
:10FAB000DDE90412C2F31303002B3FF418AF40E654
:10FAC000002A12DD294601222046049301F0BAFDE6
:10FAD0004946054601F02EFE0028049B40F318819C
:10FAE000392B00F0F9800BF13103BA460AF8013BDB
:10FAF000079B0133374607934646E4E50995069C84
:10FB0000049D02460B46F0F701FC52465B468046D8
:10FB10008946F0F72FFE60B952465B46404649469B
:10FB2000F0F700FE00283FF4CEAC099BD9077FF523
:10FB3000CAAC039A02E47168204601F01FFB074635
:10FB4000002800F00E81336902339A0006F10C019F
:10FB50000C30F1F757FA39460122204601F072FDC8
:10FB6000804614E62946204601F00CFD054621E5B5
:10FB7000DDE908239F1AC6E4392B00F0AD80BA46B0
:10FB80000133B3E7079A01323746079246467BE5D1
:10FB9000943401080000F07F8837010860370108BD
:10FBA000DDF84CA0844901EBCA01DDE9102351E9DD
:10FBB0000201F1F705FDCDE9100149464046F0F795
:10FBC000F9FD0646F0F7EEFC0B4602464946404674
:10FBD000F0F79AFB039F53463036012B07F8016B71
:10FBE0008046894600F0AE80139E039B1E44734BF3
:10FBF000002240464946F1F7E3FC89468046F0F78B
:10FC0000D9FD8246F0F7CEFC0AF1300A02460B46D7
:10FC100040464946F0F778FB07F801ABB74280460B
:10FC20008946E4D1664B0022DDE91001F0F76EFB56
:10FC300042464B46F0F780FD002864D1DDE91023F1
:10FC40005F490020F0F760FB42464B46F0F792FD1B
:10FC500000283FF4ADABB246013E1AF8013C302B10
:10FC6000F9D0149B013307933DE5169BC3F136038E
:10FC7000D7E6DDE90A894FF0020AFFF7C5BA089B0B
:10FC8000002B3FF467AB129B002B7FF791AB079AD9
:10FC9000013ACDE913324046484B00224946F1F77C
:10FCA0008FFC804689460AF10100F0F77BFC424652
:10FCB0004B46F1F785FC434B0022F0F727FBA1F1FF
:10FCC0005073CDE910011193FFF7C1BA079B0133BF
:10FCD00007933123FFF739BB079BBB4601330793DB
:10FCE000392337460BF8013B4646DCE44FF0000968
:10FCF0004E464BE69A466CE4109D139C149B0133D0
:10FD00000793B246EFE4149B039A0793FFF716BBE1
:10FD10007FF4EBAEDA077FF5E8AEE1E6DDF854B04C
:10FD2000109D139CFFF744BB392BD5D0BAF1000FBF
:10FD30003FF7D9AED9E6229B022B3FF712AECDF8A2
:10FD40001C809BE53E466DE7229B022B3FF709AEE8
:10FD5000129BCDF81C80089311E54FF0020AFFF7C3
:10FD600053BA194B19483A4640F2EA2102F050FFC3
:10FD7000002666643146204601F000FA039078B907
:10FD8000114B124800224FF4D57102F041FF104B85
:10FD90000393FFF7F8B83FF434ACC0F13C00B7E48C
:10FDA000039B236401224FF0FF33239612930C929E
:10FDB0000893FFF7FDBA00BF883701080000244010
:10FDC0000000E03F00001C40A4340108B8340108E2
:10FDD00098340108B1F90C20F8B50C461107074614
:10FDE00042D4636842F40062002BA28159DDA56A07
:10FDF000002D54D000233E683B6093B212F4805231
:10FE000053D1E16901233846A847421C63D0A38936
:10FE1000A56A5B0705D56368C01A236B0BB1E36B5A
:10FE2000C01AE169024600233846A847411C3ED16A
:10FE30003B68002B3BD01D2B01D0162B52D1A38940
:10FE40002269226023F4006300216160A381216B99
:10FE50003E6021B304F14003994202D0384600F0DD
:10FE600075F900202063F8BD2669C6B193B22568F4
:10FE700026609A070CBF63690023AD1BA3600CE0EA
:10FE8000D4F824C0E1692B4632463846E047B0F149
:10FE9000000CA5EB0C05664416DD002DF0DC0020FF
:10FEA000F8BDE36B002BA2DCF9E7206DB1E7B4F9F4
:10FEB0000C302269226023F40063A3810022DB045A
:10FEC0006260C4D52065C2E7A38943F040034FF0C8
:10FED000FF30A381F8BD3B68002B98D01D2B06D0C6
:10FEE000162B04D0A38943F04003A381F8BD3E60E4
:10FEF000D5E700BF38B50C46054608B1836BA3B102
:10FF0000B4F90C00B8B1636EDB0701D4810515D5D7
:10FF100028462146FFF75EFF636EDA07054602D4E6
:10FF2000A3899B050ED5284638BD00F017F8B4F913
:10FF30000C000028E7D10546284638BDA06D00F02A
:10FF4000D1FFE5E7A06D00F0CFFF284638BD00BF28
:10FF5000014900F075BB00BFC92C01082DE9F0472D
:10FF60008246394800F0BEFFDAF83840002C66D1EE
:10FF7000DAF80450354ACAF83C200323CAE9B843EA
:10FF8000DFF8CC90DFF8CC80334F344E04230AF5F1
:10FF90003B72CAF8E8222146C5E90243C5E900449C
:10FFA000C5E904446C660822AC6105F15C00FBF70E
:10FFB000FBFCC5E90759C5E90987EE6205F1580060
:10FFC00000F08CFFDAF80850254BEB602146C5E9BC
:10FFD0000044C5E904446C66AC60AC61082205F1DC
:10FFE0005C00FBF7E1FCC5E90759C5E90987EE624A
:10FFF00005F1580000F072FFDAF80C50194BEB6075
:020000040801F1
:100000002146C5E90044C5E904446C66AC60AC61B6
:10001000082205F15C00FBF7C7FC05F15800C5E9B3
:100020000759C5E90A76C5F8248000F057FF012377
:10003000CAF838300448BDE8F04700F055BFBDE8C5
:10004000F047014800F050BF542B002451FF000836
:10005000FDC0000821C1000861C1000881C100087D
:100060000900010012000200014800F03BBF00BF80
:10007000502B0024014800F037BF00BF502B002454
:1000800038B5084B084D5B1B9C1007D0043B1D4442
:10009000013C55F804399847002CF9D1BDE83840A7
:1000A00003F006B8D0380108CC380108F8B5244F61
:1000B0000C460646FBF7CAFCBA685568C4F57E6371
:1000C0000F3325F003052B4423F47F6323F00F0344
:1000D000A3F58054B4F5805F07DB00213046FBF7C1
:1000E00023FFBB682B44984204D03046FBF7B4FC96
:1000F0000020F8BD61423046FBF716FF01300DD0FD
:10010000104ABB682D1B45F001055D601368304641
:100110001B1B1360FBF7A0FC0120F8BD002130463B
:10012000FBF702FFBA68831A0F2BDEDD43F00103F1
:100130005360054B03491B68C01A0860D5E700BF30
:1001400058040024142B002460080024002961D0E6
:10015000F8B50C460646FBF779FC54F8042C7B4FA7
:10016000A4F1080522F0010105EB010CB868DCF8E8
:100170000430604523F0030300F08B80D207CCF8F5
:10018000043032D454F8082CAD1A1144AA6807F18F
:10019000080082426AD00CEB0304D4F804E0EC6857
:1001A000D4601EF0010FA26000F0978041F00103BF
:1001B0006B60CCF80010B1F5007F35D27A68CB08BF
:1001C00048090121013381401143796007EBC302E3
:1001D00057F83310083AC5E9021247F83350CD609A
:1001E0003046BDE8F840FBF737BC0CEB0302526821
:1001F000D00710D4194407F10800DCF80830834216
:1002000073D0DCF80C20DA60936041F001036B607E
:100210006950D0E7704741F00103B1F5007F44F821
:10022000043CCCF80010C9D3B1F5206F4FEA51233C
:1002300048D28B0903F1390003F13802C300F818E2
:10024000FB580838984259D05A6822F003028A4273
:1002500002D99B689842F7D1D868C5E90230856019
:10026000DD603046BDE8F840FBF7F6BB0CEB03025F
:100270005268D20763D40B44DCE90212CA60916071
:1002800043F001026A603046EB50BDE8F840FBF7EE
:10029000E3BB0B44D10707D454F8082CAD1A134420
:1002A000D5E90212CA60916043F001026A60284AEF
:1002B000BD6012689A4293D8264B30461968FFF702
:1002C000F5FE8DE7142B0AD9542B1FD80B0B03F125
:1002D0006F0003F16E02C300B1E719448DE703F12B
:1002E0005C0003F15B02C300A9E741F00103C7E929
:1002F0000455C5E902006B60695071E77968921096
:10030000012404FA02F20A437A60A6E7B3F5AA7F51
:1003100006D8CB0B03F1780003F17702C3008EE718
:1003200040F25452934206D88B0C03F17D0003F146
:100330007C02C30083E74FF47E737E227FE741F0A7
:1003400001036B60CCF800104AE700BF580400249A
:1003500064080024442B00249368002B00F0818063
:100360002DE9F04FB1F90C300C461907804683B0E7
:10037000174698B223D523690BB310F002033D68EA
:100380002BD04FF0000ADFF8B4B256465E45334634
:10039000524628BF5B464046002E4FD0E169D4F854
:1003A00024C0E047002852DDBB681B1A8244361A7D
:1003B000BB60002BEAD1002003B0BDE8F08F2146DE
:1003C0004046FEF787FC002840F03481B4F90C3039
:1003D0003D6898B210F00203D3D110F0010942D168
:1003E0004E463EB38205D4F808B040F18180B34553
:1003F0005A4600F2B18010F4906F40F0BE80206841
:100400000192494600F03EFEA3682168019AA3EBE1
:100410000B030A44B246A36022600026B868A0EB32
:100420000A00D144B8600028C5D0B4F90C0080B2ED
:10043000002ED7D1D5E900960835D2E7D5E900A638
:100440000835A3E721464046FFF754FD80B3B4F9D1
:100450000C3043F040034FF0FF30A38103B0BDE800
:10046000F08F002070471E46AA46994618461D4642
:1004700056B388B34A46D4E904132068B24228BF71
:100480003246884205D9A16803EB010B5A4500F3B7
:10049000A780934264DCE169D4F824C02A46404630
:1004A000E047B0F1000BD2DDB9EB0B09CAD0012057
:1004B000BB68A3EB0B035D44A6EB0B06BB60002BF4
:1004C0003FF479AF002ED4D10AF1080353E9025664
:1004D0009A460833002EF9D032460A212846F1F711
:1004E0001FF8002800F09D800130A0EB0509C1E74E
:1004F00020682369984217D86369B34214D86FF013
:100500000042B24228BF3246E16992FBF3F2D4F8CE
:1005100024C002FB03F340464A46E047B0F1000A1C
:1005200095DDA6EB0A0679E7B345DA4628BFB24661
:100530005246494600F0A6FDA3682268A3EB0A03D1
:100540005244A3602260002BEBD121464046FFF7C6
:10055000D1FC0028E5D07AE72068B34632464FE761
:100560002946019200F08EFD019AA3689B1AA360B0
:10057000236813442360934696E723682169A3EB1D
:10058000010B636903EB430A0AEBDA7A0BF101030F
:100590004FEA6A0A33445345524684BF9A4652464C
:1005A00043052CD511464046FAF74EFF00283BD0B4
:1005B0005A4621690190F0F725FDA289019B22F49A
:1005C000906242F08002A28103EB0B002361AAEB50
:1005D0000B03C4F814A0A3602060B34632460FE7B3
:1005E00029465A4600F04EFD23685B4423602146AD
:1005F0004046FFF77FFC00283FF456AF27E7404610
:10060000FBF7A6FA03460028DED121694046FFF732
:100610009DFDB4F90C300C2223F08003C8F80020B3
:1006200017E7721C914626E70C22B4F90C30C8F883
:1006300000200EE74FF0FF30BEE600BF00FCFF7F5A
:100640002DE9F8430746884600F538764FF0000953
:10065000D6E90154013D11D4A389012B05F1FF35E1
:1006600008D9B4F90E300133214603D03846C047CB
:1006700049EA00096B1C04F16804EDD13668002ECC
:10068000E6D14846BDE8F8832DE9F0410469B4EBB2
:10069000611F2FDD00F1140E4E1111F01F0C0EEB37
:1006A00084050EEB86032BD05EF8262004339D4292
:1006B00022FA0CF1CCF1200818D977461A6802FA10
:1006C00008F20A4347F8042B53F8041B9D4221FA11
:1006D0000CF1F3D8A41BA300053B9B0801330EEBE0
:1006E00083044EF82310C9B1043417E04161744605
:1006F0000029F9D10023036100234361BDE8F081A3
:100700009D4288BF00F11002F4D953F8041B42F84F
:10071000041F9D42F9D8A41B0EEB8404A4EB0E0326
:100720009B1074450361E7D0BDE8F0812DE9F04FDF
:10073000A84C8BB024680590204689460292079306
:100740000394F0F77DFE21460144D9F8003011F8FA
:1007500001BC99783029024640F0DA816FF001003F
:10076000C01A033300EB030A1C4613F8011B30299F
:10077000F8D0DFF8648218F80130002B00F0F08028
:100780002378002718F803303D4626462BB116F88B
:10079000013F18F80330002BF9D10399019230463C
:1007A000FBF7F2FC019A0090002800F09180002DE8
:1007B00040F091803378009503F0DF03502B3546ED
:1007C00000F09380C9F80060002F40F0AB802B1B35
:1007D000013B072B394604DD5B10072B01F10101BA
:1007E000FADC0598049200F0C9FC049A01900028F4
:1007F00000F06782019BAC4203F11406069680F07C
:10080000DC810027C2F10103B946049310E0202FD8
:1008100000F091803946043715F8013C18F8033090
:10082000554603F00F038B40A54249EA030916D948
:1008300015F8013C5B4505F1FF3AE8D1049B5344B0
:10084000A342E4D31846039909920893FBF79CFC52
:10085000DDE908320028DAD11D46A542E8D846F87D
:10086000049B069BF61A019BB6101E61484600F0D9
:100870005FFD029B76011C68301AA04200F3AE8037
:10088000C0F226810027029B009A9B689342C0F227
:1008900089810299009A4B6893427EDD9D1AAC4291
:1008A00000F3BC80CA68022A00F0BC81032A00F071
:1008B000B481012A00F098810598019900F084FC28
:1008C0005025149A0023284613600BB0BDE8F08F22
:1008D000002D00F00B81AD1BAB000093337803F0CB
:1008E000DF03502B35467FF46DAF6B782B2B00F078
:1008F000ED802D2B6AD06E1C002018F803104B1EC3
:10090000182B61D8737818F803301039013623BBDF
:1009100000B14942009BC9F800600B440093002FCE
:100920003FF455AFBAF1000F14BF00250625284645
:100930000BB0BDE8F08F002146F8049B04278946E0
:100940006AE701EB810103EB4103A3F1100116F803
:10095000013F18F80330002BDAD0192BF1DDD7E76F
:10096000039900922046FBF70FFC009A002873D1F0
:10097000A15C18F80130A518002B6FD030292C4647
:1009800005D114F8013F302BFBD018F80330B3FA2F
:1009900083F77F094FF0010AF7E6012557B1029B63
:1009A000DB68022B62D0032B64D0012B00F0858022
:1009B00045F01005149B019A1A60079B009A1A6073
:1009C00028460BB0BDE8F08F2E46FBE60120AB7841
:1009D000AE1C92E7C4360108C0350108019D061B14
:1009E0003146284601F0B4F8074678B1721E53111B
:1009F0000699012751F8231002F01F0307FA03F3A9
:100A00000B4203D0BA4200F3E2800227009B019818
:100A1000334431460093FFF737FE34E76E1E002F54
:100A200040F0C980002E40F0CC807311069A0198E6
:100A300052F8232006F01F06012303FA06F6164299
:100A4000294618BF47F00207FFF71EFE029B5B68AE
:100A50000093641B0225A1E72178254601F0DF0100
:100A6000502900F0BD80C9F800505BE7159BC3F129
:100A700001031593159B002B9AD0019BDDF818906C
:100A80001E6900214B464FEA860809EB860003E009
:100A9000984243F8041C3FD91F4653F8042BB2F187
:100AA000FF3FF5D00132022D3A6000F0C08014F013
:100AB0001F0440F0E08021257CE7BA077FF578AF7E
:100AC000069B1B681F43FB07D7D471E700207EE716
:100AD000DDE90031221A9B1A0598009300F0B2FD5F
:100AE00003461433019006930027CCE6B35C18F854
:100AF0000310B018064600293FF45EAE16F8013F19
:100B000018F803100029F9D1801B8100009153E6E9
:100B10009C1C4FF0000A2CE6019B9B689E4280F2D1
:100B20008D803346019901EB830201330B61022D65
:100B30004FF0010151617AD09E42B8DA002B40F3A8
:100B4000A780019A09EB8303516902F118008342DF
:100B50004FEA510140F2AF804C46026841EAC2714F
:100B600044F8041B50F8041B83424FEA5101F4D8A7
:100B7000019A9B1A193B9B08013349F8231009EB92
:100B80008303002940F09B800199A3EB0902921096
:100B90004B450A617FD0029B009A9B6801329342C9
:100BA000009288DA0199059800F00EFB149A002350
:100BB0001360A325BBE6012737E7069E4FF0000927
:100BC0004DE60198314600F0C3FF07462DE7B11E00
:100BD000284600F0BDFF00283FF417AF032715E7B4
:100BE00000230093012780E6AC427FF465AE012C20
:100BF00008D00198611E00F0ABFF00283FF45CAE06
:100C0000029B5B6807990B60019B069901221A61A0
:100C10000A60149A6225136089E6159A002A3FF447
:100C20004BAEEFE7159A002A7FF446AEEAE7029B47
:100C30001B68013BA34232D02225BBE6019B0598ED
:100C40005968013100F09AFA074600283FD0DDF8D4
:100C50000490D9F81030494602339A000C310C3018
:100C6000F0F7D0F94946059800F0AEFA07F11409FB
:100C70003B69019756E7C844C4F1200458F8040CB6
:100C800000F056FBA042BFF616AF019B1B6955E76B
:100C9000019A00231361019A002353617BE76311DA
:100CA00004F01F0459F823200123A34013420CBF72
:100CB000222521257EE6C9F800104B4669B1043390
:100CC00062E7074B0748019ADE2101F0A1FF044BC0
:100CD00004483A46842101F09BFF019B1961DAE741
:100CE000A43401083835010810B4046809E014F888
:100CF000013FA3F1410CBCF1190F98BF203393427F
:100D000008D111F8012B002AF1D10134046001202F
:100D100010BC7047002010BC704700BF2DE9F04F99
:100D2000096885B04B1111F01F01029002EB83039B
:100D3000039140F08E801D1F0193029B01991C6856
:100D4000002341F8043C61780134002900F09780C9
:100D5000DFF87091A846AC469A461E460EE0202960
:100D600000F28B80B24506DAC44501D2072B5BDD69
:100D7000624551D3082314F8011FA1B119F80100ED
:100D80000028ECD00133082B06F101063ADCDCF830
:100D90000010090100F00F000843CCF8000014F81F
:100DA000011F0029EAD1002E69D0E04501D9072BA7
:100DB00073DD624551D2111F634653F8040B41F8AD
:100DC000040F9D42F9D2A5EB0C0323F00303691C29
:100DD00004330CF1010C614538BF04231344002196
:100DE00043F8041B9D42FBD2019B53F8043C2BB9F2
:100DF000AA4248D055F8043D002BF9D0052005B093
:100E0000BDE8F08F6245B6D200234CF8043C194689
:100E1000ACF1040C0123BDE70023ACF104084CF84D
:100E2000043CB246C446A6E7C3F108018900DCF8D9
:100E30000030C1F1200E60468B46416801FA0EF782
:100E40003B43036021FA0BF340F8043F4045F4D3E1
:100E50008EE7191D01911D466FE7039B002BC3D040
:100E6000039B0198C3F120014FF0FF33CB4050F8B2
:100E7000041C0B4040F8043CB9E7292909D00420A0
:100E800005B0BDE8F08F012305202B6005B0BDE85B
:100E9000F08F029901340C6085E7C3F108039B00D1
:100EA000DCF80010C3F120076446666806FA07F014
:100EB0000143216026FA03F144F8041FA045F4D849
:100EC00077E700BFC0350108014B93F82801704750
:100ED000700800240048704760090024704700BF74
:100EE000704700BF704700BF704700BF38B50C4661
:100EF000084D8446114620461A4600232B6064465E
:100F0000F2F708F8431C00D038BD2B68002BFBD04B
:100F1000236038BD582B00242DE9F0418B890C4605
:100F2000990796B008D504F143030122C4E90432BD
:100F3000236016B0BDE8F081B4F90E100029064612
:100F400027DB6A4601F0C2FF002821DB019D05F482
:100F50007045A5F50055B5FA85F54FF480686D0923
:100F60004FF4006741463046FAF76EFAB4F90C3098
:100F7000F0B1204AF26343F08003C4F81480A381E7
:100F80002060206135BB3B43A38116B0BDE8F081F2
:100F9000A38913F0800519D04FF040084146304630
:100FA000FAF752FA0025B4F90C302F460028E0D1A8
:100FB0009A05BED423F0030304F1430243F0020375
:100FC0000121C4E90421A3812260B2E74FF48068C3
:100FD0002F46C7E7B4F90E10304601F08DFF10B967
:100FE000B4F90C30CFE7A38923F0030343F00103E6
:100FF0001BB2C8E751FF000870B50C46B1F90E10DE
:10100000002996B015461E4614DB6A4601F05EFFC5
:1010100000280FDB019A02F47042A2F50052B2FAE6
:1010200082F24FF4806352094FF4006032602B600B
:1010300016B070BDB4F90C10002311F080003360BD
:1010400004D0402218462A6016B070BD4FF4806369
:101050002B6016B070BD00BF82B049B15AB16BB100
:1010600013780B601278101E18BF012002B0704771
:1010700001A9002AF3D1104602B070476FF00100B9
:10108000F4E700BF88420DD98B1883420AD900EBE0
:10109000020CBAB1624613F801CD02F801CD9942B3
:1010A000F9D170470F2A0ED8034602F1FF3C4AB12E
:1010B0000CF1010C013B8C4411F8012B03F8012FBA
:1010C0006145F9D1704740EA01039B0750D1A2F175
:1010D000100370B501F1200C23F00F0501F1100E83
:1010E00000F11004AC441B095EF8105C44F8105C7D
:1010F0005EF80C5C44F80C5C5EF8085C44F8085C34
:101100005EF8045C44F8045C0EF1100EE64504F150
:101110001004E9D1013312F00C0F01EB031102F0BE
:101120000F0400EB031327D0043C24F003064FEA1E
:10113000940C1E441C1F8E465EF8045B44F8045F4A
:10114000B442F9D10CF1010402F0030203EB840371
:1011500001EB840102F1FF3C4AB10CF1010C013BAF
:101160008C4411F8012B03F8012F6145F9D170BDB2
:1011700002F1FF3C03469BE72246EBE7C36C70B5E8
:1011800005460C464BB153F8240080B1026843F881
:1011900024200023C0E9033370BD2122042101F083
:1011A00057FD0346E8640028EDD1002070BD012101
:1011B00001FA04F6721D9200284601F049FD00284C
:1011C000F3D0C0E90146E4E731B1C36C4A6853F893
:1011D0002200086043F82210704700BF2DE9F0415B
:1011E0000D6907460E461C4601F1140E0020DEF87C
:1011F00000108BB202FB03434FEA134C090C02FBB5
:1012000001CC01309BB203EB0C4385424EF8043B0A
:101210004FEA1C44EBDC3CB1B368AB4207DD06EBA4
:10122000850301355C6135613046BDE8F081716848
:1012300038460131FFF7A2FF8046A8B13269023279
:1012400006F10C0192000C30EFF7DCFEFB6C7268CB
:1012500053F82210316043F82260464606EB8503BE
:1012600001355C613561DFE7024B03484246B52139
:1012700001F0CEFCA4340108DC3601082DE9F84366
:101280000C4628491E46174603F1080281FB02312D
:10129000092E4FEAE2730546C3EB610339DD4FF0D7
:1012A000010C00214FEA4C0C634501F10101F9DC0E
:1012B0002846FFF763FF014668B3089B4361092F87
:1012C0004FF00103036112DC0A340927BE420BDD33
:1012D000F61B264414F8013B0A22303B2846FFF750
:1012E0007DFFA6420146F5D10846BDE8F88304F12A
:1012F0000909C8463C4418F8013B0A22303B2846FD
:10130000FFF76CFFA0450146F5D1A7F108044C4456
:10131000DCE70021CCE70A46034B0448CE2101F06C
:1013200077FC00BF398EE338A4340108DC360108AD
:10133000020C12040346CAB90304102013F07F4FB5
:1013400004BF1B02083013F0704F04BF1B010430B0
:1013500013F0404F04BF9B000230002B05DB13F05D
:10136000804F00F1010008BF202070470020E5E712
:101370000368024613F0070007D0D9071DD4980769
:101380001FD55B0813600120704799B209B91B0C87
:101390001020D9B209B908301B0A190704BF1B096C
:1013A0000430990704BF9B080230D90703D45B08B7
:1013B00000F1010003D01360704700207047202027
:1013C00070479B0813600220704700BF38B5C36C9C
:1013D00004460D464BB15868B0B102685A6000220D
:1013E0000123C0E90435C26038BD2122042101F087
:1013F0002FFC0346E0640028EDD1094B0948002288
:101400004FF4A07101F004FC1C220121204601F0E0
:101410001FFC0028F1D001220223C0E90123DEE7EE
:10142000A4340108DC3601082DE9F04F0E69156976
:10143000AE4285B08846144605DB2A46234635462B
:101440000C4616469846A3686168AF19BB42B8BF00
:101450000131FFF793FE0190002800F08780019B87
:1014600003F1140909EB870AD14505D24B46002246
:1014700043F8042B9A45FBD808F1140808EB860BB7
:1014800004F11403D8451A4603EB85055FD22B1BE4
:10149000153B23F0030304331534A54238BF04235E
:1014A000CDE902A7AC461F46924605E0000C29D1C3
:1014B000C34509F1040948D958F8040B85B2002D39
:1014C000F4D056464C46002356F8040B216882B2ED
:1014D0001FFA81FE05FB02EE000C0A0C734405FBAB
:1014E000002202EB13429BB243EA0243B44544F8A4
:1014F000043B4FEA1243E7D849F8073058F8040C88
:10150000000CD5D0D9F80030544619464D4600227B
:101510002688090C00FB06110A449BB243EA0243E9
:1015200045F8043B54F8046B2968360C8BB200FB79
:10153000063303EB1243A4454FEA1342E8D8C345F0
:1015400049F8073009F10409B6D8DDE902A7002FF0
:1015500002DC05E0013F03D05AF8043D002BF9D02E
:10156000019B18461F6105B0BDE8F08F034B04488E
:10157000019A40F25D1101F04BFB00BFA434010859
:10158000DC36010812F003032DE9F041144606464B
:1015900032D10D46A41020D0D6F84880B8F1000F03
:1015A00033D0E3074FF0000707D4641015D0D8F804
:1015B0000000A8B18046E307F7D5424629463046E9
:1015C000FFF732FFB5B16968F36C641053F821205E
:1015D0002A6043F821500546E9D12846BDE8F0814C
:1015E000424641463046FFF71FFFC8F8000007603B
:1015F0008046E0E70546D8E7013B0F4A52F8232032
:101600000023FFF7EBFD0546C4E701213046FFF755
:10161000B5FD804640B1012340F27122C0E9043299
:101620000023B0640360BCE7044B054842464FF416
:10163000A07101F0EDFA00BF50380108A434010890
:10164000DC3601082DE9F0470C4690462669A36870
:10165000496806EB6216751C9D4207464FEA6219FF
:1016600004DD5B009D4201F10101FADC3846FFF721
:1016700085FD8446002851D0B9F1000F00F1140017
:101680000EDD09F105024FEA820E03460CEB8202E1
:10169000002143F8041B9342FBD1AEF1140318441C
:1016A000216904F1140318F01F0803EB81012DD008
:1016B000C8F1200986464FF0000A1A6802FA08F2BB
:1016C00042EA0A024EF8042B53F8042B994222FAFC
:1016D00009FAF2D80B1B153B23F00303043304F182
:1016E0001502914238BF0423BAF1000F18BF2E46ED
:1016F00040F803A0FB6C6268CCF8106053F822102D
:101700002160604643F82240BDE8F087043853F872
:10171000042B40F8042F9942F9D8EBE7034B044817
:10172000624640F2D91101F073FA00BFA4340108F7
:10173000DC3601080B6984460069C01A15D10CF12A
:10174000140C14310CEB830210B401EB830301E0A1
:10175000944508D252F8044D53F8041D8C42F7D03A
:1017600004D24FF0FF3010BC70477047012010BC0E
:10177000704700BF2DE9F84F0F691369FF1A002F5A
:101780000E4690467AD101F11405143202EB830221
:1017900005EB830301E09D4273D253F8041D52F818
:1017A000044DA142F7D064D37168FFF7E7FC81468E
:1017B000002872D03569D8F81020C76008F1140EDF
:1017C00006F1140009F1140A06F1100C0EEB820266
:1017D00000EB8507564600215EF8044B5CF804BF19
:1017E000A3B211FA8BF1CB1A210CC1EB1B4101EB17
:1017F00023419BB243EA0143724546F8043B4FEA5A
:101800002141E9D8A2EB0804153C08F1150842452E
:1018100024F0030606F1040638BF0426304424F001
:10182000030238BF002287425244B24416D95646BA
:10183000044654F8043B11FA83F10A1402EB1342F4
:1018400089B241EA0243A74246F8043B4FEA2241EB
:10185000EFD87A1E101A20F00302524423B952F82E
:10186000043D013D002BFAD0C9F810504846BDE8B0
:10187000F88F334601274646984695E7F9DB00275F
:1018800092E70021FFF77AFC814668B1012200232C
:10189000C9E904234846BDE8F88F074B07484A4684
:1018A0004FF4107101F0B4F9034B04484A4640F27A
:1018B000322101F0ADF900BFA4340108DC36010883
:1018C0000F4B0B40A3F15073002B02DD0020194693
:1018D00070475B42B3F1A07F4FEA235205DA4FF421
:1018E0000023002043FA02F17047143A1E2ADABF9F
:1018F0004FF0004323FA02F2012200211046704704
:101900000000F07F2DE9F843066900F1140808EBA8
:101910008606A6F1040956F8047C3846FFF708FD50
:10192000C0F120030A280B6036DDC8451ED2B0F195
:101930000B0356F8082C26D0C3F1200C22FA0CF128
:101940009F400F43A6F1080147F07F55884545F4B5
:1019500040153AD202FA03F056F80C3C23FA0CF385
:1019600003431C4620462946BDE8F883B0F10B032B
:1019700008D007FA03F343F07F55002345F44015E0
:101980001C46EFE71A4647F07F5545F440151446CC
:1019900020462946BDE8F883C0F10B0327FA03F27D
:1019A000C84542F07F553CBF56F8082CDA4000F19C
:1019B000150328BF002207FA03F345F4401543EA54
:1019C000020420462946BDE8F88302FA03F31C46C8
:1019D000C8E700BF70B5012182B016461D46FFF76B
:1019E000CDFB044600284BD02B46C5F30A55C3F364
:1019F00013030DB143F48013002E019322D06846E7
:101A00000096FFF7B5FC002836D0019B0099C0F185
:101A1000200203FA02F20A43C34001936261002BE1
:101A200014BF02210121A3612161ADB1069AA5F283
:101A3000334303441360079BC0F135001860204610
:101A400002B070BD01A8FFF793FC019B0121C4E91E
:101A500004132030002DE9D104EB8102A0F23243BF
:101A60001069069A1360FFF763FC079BC0EB4111F6
:101A70002046196002B070BDDDE900236261CEE747
:101A8000034B0448224640F20A3101F0C1F800BF7E
:101A9000A4340108DC3601082DE9F04383B00F4679
:101AA00069468046FFF72EFF04460D46384601A9D9
:101AB000FFF728FFD8F810303A690F469A1ADDE987
:101AC0000013CB1A03EB4213002B06460BDD05EB8C
:101AD00003594D4632463B4620462946EFF79AFECB
:101AE00003B0BDE8F083C3EB033307EB03510F46AC
:101AF000F0E700BF0139491101F1010C116902F150
:101B0000140303EB81018B4200EB8C0C16D210B551
:101B1000A0F1040E53F8044B4EF8044F9942F9D843
:101B20008B1A153B23F0030304331844844504D96E
:101B3000002340F8043B8445FBD810BD844505D9FB
:101B4000002340F8043B8445FBD87047704700BF32
:101B500003694A11934200F1140009DA00EB830390
:101B600002E053F8042DC2B98342FAD8002070472E
:101B700010DD11F01F010DD010B450F8224000EB21
:101B8000820324FA01F202FA01F18C420BD0012007
:101B900010BC704700EB8203E6E70120704753F862
:101BA000042D002AF3D18342F9D8002010BC7047DD
:101BB00038B50C46084D8446114620461A46002387
:101BC0002B606446F1F7AEF9431C00D038BD2B689A
:101BD000002BFBD0236038BD582B0024DFF860C0F9
:101BE000F8B521F000430027634504460D4616462C
:101BF000176022DC844653EA0C0C1ED0DFF844C088
:101C000001EA0C0C0A46BCF1000F09D10E4B002270
:101C1000EFF7D6FC6FF0350704460A4621F0004383
:101C200022F0FF421B1522F4E002A3F2FE3342F041
